:100000000C94D21A0C94031B0C94031B0C94031B2A
:100010000C94031B0C94031B0C94031B0C94031BE8
:100020000C94031B0C94031B0C94031B0C94031BD8
:100030000C94031B0C94031B0C94031B0C94031BC8
:100040000C94031B0C9440DA0C94031B0C94031BBC
:100050000C94031B0C94031B0C945EC10C94FEAC1B
:100060000C94031B0C9484560C947A560C94031B2A
:100070000C94031B0C94031B0C94031B0C94031B88
:100080000C9472340C94031B0C94031B0C94031BF0
:100090000C94031B0C94031B0C94031B0C94031B68
:1000A0000C94031B0C94031B0C9444340C94031BFE
:1000B0000C94031B0C94031B0C94031B0C94031B48
:1000C0000C94031B0C94031B0C94031B0C9480379F
:1000D0000C944A370C94031B0C94031B0C94031BC5
:1000E0000C94031B084AD73B3BCE016E84BCBFFD7A
:1000F000C12F3D6C74319ABD56833DDA3D00C77FF8
:1001000011BED9E4BB4C3E916BAAAABE0000008090
:100110003F05A84CCDB2D44EB93836A9020C50B91F
:10012000918688083CA6AAAA2ABE000000803F004B
:100130000C9471A80C94C2560C9438A60D94330DEF
:100140000D94B4170D94F40F0C947DA80D94FF0C2E
:100150000C947FA90C9486A80C940B380C9430A9AD
:100160000C9411AC0D9421130D9446070C94165762
:100170000C94BE370D94B00C0C94D2AB0C9451A9D6
:100180000C948AA80C941E380C9489A90C94F156EE
:100190000D949F040C9400570D94CA040D940313FE
:1001A0000C940F570C942E570C94A2A90C94C0A930
:1001B0000C942A570C943C380C947A420D945F0EA0
:1001C0000D940A140C9430AA0D94CF0D0C946BA9C5
:1001D0000C94ACAA0D94E4240D949F0F0D94D412AA
:1001E0000C9448570C94B5A50C9440570D94AD123F
:1001F0000C9402450D94A3100C943DA90C9479A87D
:100200000D94950E0C9426380D94DA120D946E0F01
:100210000C94B6A90D94C6240C94A6A80D946A0B50
:100220000C9480A80D948D0F0C941A380C9438A956
:100230000D948B020D94F5120C94C9420C9475A880
:100240000D94C7080D94DD140C9416380C9463A912
:100250000D94E30C0C9431380C9422570D94DD125C
:100260000C9498A80C941A570C9490A80C94FC37F2
:100270000D944F0F0C9439AB0C9437A60D94260FA8
:100280000C944DAA0C949EA80C9422380D940D1336
:100290000C94F5AA0C9435570C94B0A80C9475A93D
:1002A0000C945BA90C9494A80C9495440D94E10FC4
:1002B0000C9426570C9434AC0C941E570C9447A9FC
:1002C0000C94CAA90D942E130C9412380C94ACA95A
:1002D0000C9454AB0C94CD420C94C1440C943A450C
:1002E0000D94B5030D941A140C94ACA80C944438D6
:1002F0000C942A380D94030F0C94ED370D943506A9
:100300000C94E4AB0C945FA80C945AA80C9498A994
:100310000C94A2A84E414E494E495459494E46CDDF
:10032000CCCC3D0AD7233C17B7D13877CC2B3295AC
:1003300095E6241FB14F0A000020410000C842008A
:10034000401C4620BCBE4CCA1B0E5AAEC59D740054
:10035000407A10F35A00A0724E18090010A5D4E894
:100360000000E87648170000E40B54020000CA9A27
:100370003B000000E1F50500008096980000004079
:10038000420F000000A086010000001027000000BE
:1003900000E803000000006400000000000A000004
:1003A0000000000100000000002C76D888DC674FB8
:1003B0000823DFC1DFAE59E1B1B796E5E3E453C6E8
:1003C0003AE651997696E8E6C28426EB898C9B62E0
:1003D000ED407C6FFCEFBC9C9F40F2BAA56FA5F48A
:1003E00090055A2AF75C936B6CF9676DC11BFCE0B2
:1003F000E40D47FEF520E6B500D0ED902E03009405
:100400003577050080841E080000204E0A00000099
:10041000C80C333333330F986E12831141EF8D21A3
:1004200014893BE65516CFFEE6DB18D1844B381B0A
:10043000F77C1D901DA4BBE424203284725E2281CF
:1004400000C9F124ECA1E53D27434F4D4D554E49E0
:10045000434154494F4E0044525952554E00455263
:10046000524F525300494E464F004543484F0045B6
:1004700072726F722077726974696E6720746F2070
:10048000454550524F4D210A0053544F505045445A
:100490002E20005072696E7465722073746F7070D4
:1004A00065642064756520746F206572726F727365
:1004B0002E2046697820746865206572726F7220FC
:1004C000616E6420757365204D39393920746F2051
:1004D000726573746172742E202854656D70657234
:1004E00061747572652069732072657365742E205E
:1004F0005365742069742061667465722072657337
:1005000074617274696E67290A004E6F20436865D2
:10051000636B73756D2077697468206C696E6520F4
:100520006E756D6265722C204C617374204C696E1F
:10053000653A20004E6F20436865636B73756D20CC
:1005400077697468206C696E65206E756D6265727E
:100550002C204C617374204C696E653A20006368EE
:1005600065636B73756D206D69736D617463682C61
:10057000204C617374204C696E653A20004C696EA2
:1005800065204E756D626572206973206E6F7420F0
:100590004C617374204C696E65204E756D62657296
:1005A0002B312C204C617374204C696E653A20000D
:1005B0004D3131300053657269616C207374617420
:1005C0007573206D69736D617463680A0077616982
:1005D000740A0053442072656164206572726F7200
:1005E0000A002121204B494C4C20636175736564DE
:1005F00020627920746F6F206D75636820696E6169
:1006000063746976652074696D65202D2063757249
:1006100072656E7420636F6D6D616E643A20004880
:100620006F74656E642049646C652054696D656FF4
:10063000757400486F74656E642049646C6520545D
:10064000696D656F75740A003D3D6F6E46696C613A
:100650006D656E7452756E6F75743D3D0070617599
:100660007365004D363030002066696C616D656ED3
:10067000745F72756E6F7574200066696C616D656C
:100680006E745F72756E6F757420540046696C618C
:100690006D656E7452756E6F75742054002A2A2A27
:1006A000496E6974696E67206361726420697320A2
:1006B0004F4B2A2A2A004D6564696120496E736593
:1006C00072746564004D656469612052656D6F7672
:1006D0006564004D313030305300627573793A20D3
:1006E00070617573656420666F7220696E707574D1
:1006F0000A00627573793A207061757365642066CB
:100700006F7220757365720A00627573793A207092
:10071000726F63657373696E670A002A2A2A6B69B0
:100720006C6C2A2A2A00706F7765726F6666004BC0
:10073000494C4C45442E20005072696E74657220FD
:1007400068616C7465642E206B696C6C2829206369
:10075000616C6C6564210A0053544F505045442E1F
:1007600020005072696E7465722073746F707065CA
:10077000642064756520746F206572726F72732EC9
:100780002046697820746865206572726F722061F6
:100790006E6420757365204D39393920746F20726D
:1007A0006573746172742E202854656D7065726172
:1007B000747572652069732072657365742E205399
:1007C0006574206974206166746572207265737443
:1007D000617274696E67290A006563686F3A004543
:1007E00072726F723A0042696C696E656172204C78
:1007F0006576656C696E6720477269643A0A002104
:10080000212053544F502063616C6C6564206265F5
:100810006361757365206F6620424C546F75636821
:10082000206572726F72202D20726573746172740C
:100830002077697468204D3939390A002121205305
:10084000544F502063616C6C656420626563617510
:100850007365206F6620424C546F75636820657223
:10086000726F72202D2072657374617274207769C3
:100870007468204D3939390A002F2F616374696F0C
:100880006E3A0070726F6D70745F00656E64005335
:10089000656E64204D31303820746F207265737539
:1008A0006D650A00496E736572742066696C616DCE
:1008B000656E7420616E642073656E64204D313006
:1008C000380A005265686561742066696E697368EC
:1008D00065642E0052656865617420446F6E650022
:1008E000526568656174696E672E2E2E00526568C8
:1008F000656174004865617465722054696D656F47
:1009000075740053656E64204D31303820746F204B
:1009100068656174206E6F7A7A6C650A004E6F7A32
:100920007A6C65205061726B656400486F74656E07
:100930006420746F6F20636F6C640A00706175735C
:1009400065640050617573650044697361626C652C
:1009500052756E6F75740050757267654D6F726574
:10096000005061757365640073686F770062757419
:10097000746F6E00626567696E004C6F616420463B
:10098000696C616D656E74004C6F61642046696CC2
:10099000616D656E74205400496E736572742066D3
:1009A000696C616D656E7420616E642073656E6440
:1009B000204D3130380A00726573756D65640052E0
:1009C0006573756D696E670057616974696E67203C
:1009D000666F72206865617475702E0A004C6561DF
:1009E00076696E6720473236003F537065636966EB
:1009F00069656420582C5920636F6F7264696E6159
:100A00007465206F7574206F6620626F756E6473F5
:100A10002E0A003F28522965706561742076616C4A
:100A20007565206E6F7420706C61757369626C659A
:100A30003B206D757374206265206174206C656164
:100A4000737420312E0A003F285229657065617445
:100A5000206D7573742062652073706563696669C3
:100A60006564207768656E206E6F74207573696E9B
:100A70006720616E204C43442E0A003F537065632B
:100A80006966696564206E6F7A7A6C652074656D3D
:100A90007065726174757265206E6F7420706C6120
:100AA000757369626C652E0A003F537065636966F1
:100AB0006965642066696C616D656E742073697A1E
:100AC00065206E6F7420706C61757369626C652E41
:100AD0000A003F53706563696669656420707269D6
:100AE0006D65206C656E677468206E6F7420706C25
:100AF00061757369626C652E0A003F5072696D659D
:100B0000206C656E677468206D7573742062652053
:100B1000737065636966696564207768656E206EC9
:100B20006F74207573696E6720616E204C43442E8C
:100B30000A003F537065636966696564206E6F7A69
:100B40007A6C652073697A65206E6F7420706C61B1
:100B5000757369626C652E0A003F52657472616339
:100B600074696F6E204D756C7469706C6965722064
:100B70006D7573742062652073706563696669655D
:100B8000642E0A003F53706563696669656420528C
:100B9000657472616374696F6E204D756C746970F1
:100BA0006C696572206E6F7420706C617573696218
:100BB0006C652E0A003F5370656369666965642041
:100BC0006C6179657220686569676874206E6F74FE
:100BD00020706C61757369626C652E0A0043292E62
:100BE0000A003F53706563696669656420626564E5
:100BF0002074656D7065726174757265206E6F74B6
:100C000020706C61757369626C65202834302D002A
:100C1000473236207374617274696E672E2E2E0A05
:100C2000004F46460A00466164652048656967686A
:100C3000742000426564204C6576656C696E67209F
:100C4000004661696C656420746F20656E61626C3A
:100C50006520426564204C6576656C696E670A00A4
:100C6000496E76616C6964206D6573682E0A005068
:100C7000726F62696E6720506F696E740025532031
:100C800025692F2569002E0A002F0050726F6269B6
:100C90006E67206D65736820706F696E7420002028
:100CA0002844525952554E29004732392041757413
:100CB0006F20426564204C6576656C696E67003F05
:100CC00020284C2C522C462C4229206F7574206F02
:100CD0006620626F756E64732E0A003F2856296580
:100CE00072626F7365206C6576656C20696D706CDF
:100CF00061757369626C652028302D34292E0A00D5
:100D0000426164205A2076616C75650A004E6F203E
:100D100062696C696E65617220677269640A004479
:100D20006576696174696F6E0025533A20257300FA
:100D300046696E6973686564210A003A207A3A2030
:100D400000206F662000476F696E6720746F3A203D
:100D5000580043570A00206469723A0020616E67A8
:100D60006C653A00537461727420726164697573C2
:100D70003A004D343820506F696E740025533A2084
:100D800025642F256400506F736974696F6E696EF6
:100D900067207468652070726F62652E2E2E0A00BF
:100DA0003F4C656773206F66206D6F76656D656E6D
:100DB0007420696D706C61757369626C6520283090
:100DC0002D3135292E0A003F2028582C5929206F13
:100DD0007574206F6620626F756E64732E0A005002
:100DE000726F6265206F7574206F6620626F756E1A
:100DF0006473003F53616D706C652073697A652080
:100E00006E6F7420706C61757369626C6520283434
:100E10002D3530292E0A004D3438205A2D50726F4E
:100E20006265205265706561746162696C6974798C
:100E300020546573740A003F2856296572626F73E7
:100E400065206C6576656C20696D706C6175736981
:100E5000626C652028302D34292E0A005374616E8F
:100E60006461726420446576696174696F6E3A20CA
:100E7000002052616E67653A2000204D61783A206B
:100E800000204D696E3A2000205369676D613A2059
:100E9000004D65616E3A20005741524E494E472140
:100EA000204C6F77205A204A65726B206D61792043
:100EB0006C65616420746F20756E77616E74656413
:100EC000207061757365732E0A004F4646004F4EC1
:100ED0000020204D61783A2000200020204D696ECE
:100EE0003A2000536F667420656E6473746F70737C
:100EF0003A20003D3D4F6E506F7765724C6F7373B3
:100F0000526573756D653D3D004D32342053256C3F
:100F1000642054256C64004739322E3920452573EE
:100F200000473120462564004739322E39205A25A2
:100F300073004731205A302046323030004731208C
:100F400058257320592573204633303030004D34F6
:100F5000323020532569205A2573004D3130362018
:100F600050256920532569004D32303020442573C7
:100F70000047323852305859004739322E3920450F
:100F800030205A300A47315A2573004D313039200C
:100F9000532569004D31393020532569004D3432D5
:100FA00030205330205A300020496E76616C6964DD
:100FB000206578747275646572200047322F47335C
:100FC0002062616420706172616D65746572730A7C
:100FD00000536C6565702E2E2E005A2050726F6281
:100FE000652050617374204265640A005A20507273
:100FF0006F62652050617374204265640047323827
:101000004C30004D3131372050726F62652066617F
:10101000696C65642E0A4732380A0070726F626527
:101020005F72657769706500473239205265747266
:1010300079696E670050726F62696E6720466169F8
:101040006C6564004D31313720426564206C6576F3
:10105000656C696E67206661696C65642E0A47304D
:10106000205A31300A4D3330302050323520533839
:1010700038300A4D333030205035302053300A4D4F
:101080003330302050323520533838300A4D333029
:1010900030205035302053300A4D3330302050321C
:1010A0003520533838300A4D333030205035302019
:1010B00053300A47342053310070726F62655F66A7
:1010C00061696C6564004D31313720426564206C84
:1010D0006576656C696E6720646F6E652E00205AB8
:1010E0003A200020593A200042656420583A2000F6
:1010F0004D65736820706F696E74206F7574206F12
:10110000662072616E67650A004D302053746F70FF
:10111000004D312053746F7000436F6E74696E75AB
:101120006500436C69636B20746F20526573756D45
:10113000652E2E2E004E6F204D6F76652E00456E6B
:10114000642066696C65206C6973740A0042656787
:10115000696E2066696C65206C6973740A004E6F55
:10116000206D656469610A00526573756D696E670B
:1011700020534400286E6F2066696C652900437512
:101180007272656E742066696C653A2000507269EF
:101190006E742074696D653A20000A53746174732B
:1011A0003A2046696C616D656E7420757365643AAA
:1011B00020002C204C6F6E67657374206A6F623A52
:1011C0002000546F74616C2074696D653A2000537F
:1011D000746174733A20002C204661696C65643A2E
:1011E00020002C2046696E69736865643A200050BF
:1011F00072696E74733A200053746174733A2000FC
:10120000436F6F6C696E672E2E2E0048656174699E
:101210006E672E2E2E0045202553006F6B006F66E3
:1012200066006A0465045E04570449044445425557
:10123000473A004D31313320530042656420436FFB
:101240006F6C696E672E2E2E0042656420486561C2
:1012500074696E672E2E2E00544D33442045352080
:10126000506C7573204F46462E002F2F00205200E1
:10127000416363656C65726174696F6E3A205000FA
:101280004D32303620580046523A0020466C6F7777
:101290003A20003A200020536572766F2000206FBC
:1012A0007574206F662072616E67650A00536572FF
:1012B000766F200020643A0020693A0020703A00DE
:1012C000496E76616C6964206578747275646572C4
:1012D0000A0020643A0020693A0020703A006469EC
:1012E0007300656E0043290A0061626C6564202802
:1012F0006D696E2074656D702000436F6C642065AD
:101300007874727564657320617265200050494479
:10131000204175746F74756E6500504944204175A5
:10132000746F74756E65206661696C656421204216
:101330006164206865617465722069640A004669A9
:101340006C616D656E742072756E6F757420646962
:101350007374616E636520286D6D293A20004669BB
:101360006C616D656E742072756E6F757420004DC2
:1013700034323120696E636F7272656374207061FC
:1013800072616D657465722075736167650A004DE1
:1013900065736820706F696E74206F7574206F6656
:1013A0002072616E67650A004F666673657473200C
:1013B0004170706C696564004572723A20546F6FB9
:1013C000206661722100546F6F2066617220667220
:1013D0006F6D207265666572656E636520706F69FA
:1013E0006E740A00454550524F4D204F4B0A002E57
:1013F0000A002028302D313029002076616C756577
:10140000206F7574206F662072616E67650041649D
:1014100076616E6365204B3D00506F7765722D6C71
:101420006F7373207265636F766572792000436114
:10143000703A004D4541545041434B00434F4F4C8F
:1014400045525F54454D5045524154555245004315
:1014500048414D4245525F54454D504552415455C7
:10146000524500424142595354455050494E47005D
:1014700041524353004D4F54494F4E5F4D4F4445E9
:101480005300544845524D414C5F50524F544543D0
:1014900054494F4E004C4F4E475F46494C454E41D4
:1014A0004D45004155544F5245504F52545F53449F
:1014B0005F5354415455530053445F575249544568
:1014C000005245504541540053444341524400505A
:1014D000524F4D50545F535550504F525400454D4C
:1014E000455247454E43595F504152534552004380
:1014F0004153455F4C494748545F4252494748541D
:101500004E45535300544F47474C455F4C4947485D
:10151000545300534F4654574152455F504F57451F
:1015200052004255494C445F50455243454E540089
:101530004C4556454C494E475F44415441005A5F23
:1015400050524F42450052554E4F5554004155544C
:101550004F4C4556454C005052494E545F4A4F42FD
:101560000050524F4752455353004155544F524536
:10157000504F52545F54454D5000564F4C554D45B9
:101580005452494300454550524F4D0042494E4147
:1015900052595F46494C455F5452414E534645525D
:1015A0000053455249414C5F584F4E5F584F464695
:1015B000004649524D574152455F4E414D453A4DC7
:1015C00061726C696E20322E302E375F4457372E91
:1015D000332E3120544D334420453550534D444231
:1015E000422028417072203239203230323120318D
:1015F000333A35303A34362920534F555243455FFC
:10160000434F44455F55524C3A68747470733A2F97
:101610002F6769746875622E636F6D2F496E7361F1
:101620006E6974794175746F6D6174696F6E2F4D59
:1016300061726C696E2F747265652F437265616C9F
:101640006974794477696E5F322E302050524F545E
:101650004F434F4C5F56455253494F4E3A312E300F
:10166000204D414348494E455F545950453A544DE9
:10167000334420453520506C7573204558545255DD
:101680004445525F434F554E543A312055554944D5
:101690003A63656465326132662D343161322D34CE
:1016A0003734382D396231322D6335356336326641
:1016B00033363766660A0050726F6265204F666681
:1016C000736574205A0050726F6265204F666673AE
:1016D0006574205A00290A0020746F20003F5A20A8
:1016E0006F7574206F662072616E6765202800290F
:1016F0000A0020746F20003F59206F7574206F66B8
:101700002072616E676520282D00290A0020746F01
:1017100020003F58206F7574206F662072616E67DD
:101720006520282D0050726F6265204F66667365D4
:10173000742058004D383400446F6E652070726913
:101740006E74696E672066696C650A004D373700F4
:101750004D33310043616E6E6F74206F70656E2083
:1017600073756264697220002569730025696D20B4
:10177000256973002569682025696D202569730036
:10178000256964202569682025696D202569730015
:1017900025697920256964202569682025696D20DF
:1017A000256973003D3D4477696E20496E69742058
:1017B000436F6D706C6574653D3D002A2A2A4E6F3B
:1017C0007A7A6C6554656D705374617475735B32AD
:1017D0005D203D003D3D48656174696E6720446F42
:1017E0006E65204368616E67652046696C616D6552
:1017F0006E743D3D002020737461727470726F6767
:101800007265737320003D3D77616974776179205B
:10181000353D3D003D3D7761697477617920343D08
:101820003D003D3D7761697477617920333D3D002E
:101830003D3D7761697477617920313D3D003D3DE3
:101840006F6E5072696E7454696D657253746F7007
:101850007065643D3D003D3D6F6E466163746F721F
:101860007952657365743D3D00270A0A0000272000
:1018700027002027002D006E6F746966696361740C
:10188000696F6E200063616E63656C005072696EF3
:10189000742041626F72746564004469736D69738A
:1018A000730055492041626F7274656400726573FC
:1018B000756D65004D3234002A2A2A43506C6179D7
:1018C00020546F6E652A2A2A003D3D6F6E50726962
:1018D0006E7454696D65725061757365643D3D0049
:1018E000486F6D696E67204661696C6564006F7052
:1018F000656E00545249474745524544003A20001E
:1019000066696C616D656E74007A5F6D696E0079F1
:101910005F6D617800785F6D6178005265706F72FD
:1019200074696E6720656E6473746F702073746180
:101930007475730A0020746F6F206C6F6E6720657A
:101940007874727573696F6E2070726576656E74E7
:1019500065640A0020636F6C642065787472757327
:10196000696F6E2070726576656E7465640A0048F2
:101970006F6D652025732573257320466972737416
:10198000005761726E696E673A20486F6D696E67C5
:101990002042756D702044697669736F72203C2017
:1019A000310A000202040000B0430000B44300000A
:1019B00000000000B0430000B4430000C843000032
:1019C000004100000041000000400101FF00000054
:1019D0000100000001000080005555550000004046
:1019E0000033333300AAAA2A0049922400000020C1
:1019F00000C7711C0099991900D14517005555155C
:101A0000003BB11300244912001111110000001015
:101A1000000F0F0F00E3380E0043790D00CCCC0C03
:101A200000C3300C00E8A20B0064210B00AAAA0A34
:101A300000703D0A009DD80900427B0900922409EC
:101A400000DCD30800888808001042080000000865
:101A500000F0C107008787070075500700711C0759
:101A6000003EEB0600A1BC06006990060066660613
:101A700000703E06006118060017F4050074D105D9
:101A8000005BB00500B29005006272050055550577
:101A90000078390500B81E0500050505004EEC0468
:101AA0000087D40400A1BD040090A704004992045B
:101AB00000C17D0400EE690400C7560400444404DC
:101AC000005C3204000821040041100400000004FE
:101AD000003FF00300F8E0030026D20300C3C30375
:101AE00000CCB503003AA803000A9B0300388E031C
:101AF00000C08103009F750300D0690300505E039E
:101B0000001D53030034480300913D0300333303A9
:101B10000016290300381F030097150300300C033B
:101B200000030303000BFA020049F10200BAE802C5
:101B3000005CE002002DD802002DD0020059C8023E
:101B400000B0C0020031B90200DAB10200AAAA0254
:101B500000A0A30200BC9C0200FA9502005C8F0268
:101B600000DF88020082820200457C0200277602A4
:101B70000027700200436A02007C640200D05E020B
:101B8000003F590200C8530200FFFDFCFAF8F6F4CA
:101B9000F2F0EEECEAE9E7E5E3E1E0DEDCDAD9D702
:101BA000D5D4D2D0CFCDCBCAC8C7C5C3C2C0BFBDA4
:101BB000BCBAB9B7B6B4B3B2B0AFADACAAA9A8A617
:101BC000A5A4A2A1A09E9D9C9A9998979594939262
:101BD000908F8E8D8B8A8988878684838281807F8F
:101BE0007E7D7B7A797877767574737271706F6E9B
:101BF0006D6C6B6A696867666564636261605F5E8D
:101C00005D5C5B5A59585857565554535251505071
:101C10004F4E4D4C4B4A4A4948474646454443423D
:101C20004241403F3E3E3D3C3B3B3A3938383736F7
:101C30003535343332323130302F2E2E2D2C2B2BA4
:101C40002A29292827272625252423232221212044
:101C5000201F1E1E1D1C1C1B1B1A191918181716D5
:101C600016151514131312121111100F0F0E0E0D5D
:101C70000D0C0C0B0A0A09090808070706060505DA
:101C80000404030302020100003D3D6F6E507269BF
:101C90006E7454696D6572537461727465643D3D10
:101CA000000000B0430000B4430000C8430000003F
:101CB0000000000000000000003D3D6F6E53746F97
:101CC000726553657474696E67733D3D003D3D6F89
:101CD0006E436F6E66696775726174696F6E537477
:101CE0006F72655772697474656E3D3D005365741B
:101CF00074696E67732053746F726564000A20699B
:101D00006E6974207A70726F62655F7A6F6666734F
:101D10006574203D20003D3D6F6E436F6E666967C0
:101D200075726174696F6E53746F72655265616428
:101D30003D3D00454550524F4D20496E69746961E3
:101D40006C697A65640A003B20003A0A0020204D45
:101D5000363033200020440020204D3431322053CF
:101D60000046696C616D656E742072756E6F757476
:101D70002073656E736F723A002055004C004669FF
:101D80006C616D656E74206C6F61642F756E6C6F25
:101D90006164206C656E677468733A0020204D3969
:101DA0003030204B004C696E656172204164766171
:101DB0006E63653A0020204D3835312058005A2D89
:101DC00050726F6265204F66667365740020204D07
:101DD000343133205300506F7765722D4C6F73731D
:101DE000205265636F766572793A0020440020497D
:101DF0000020204D33303420500020440020490082
:101E000020204D33303120500050494420736574F8
:101E100074696E67733A00204A00202047323920E7
:101E20005720490020204D34323020530041757432
:101E30006F20426564204C6576656C696E673A0078
:101E400020204D323036205800486F6D65206F6677
:101E5000667365743A0020580020530020204D32EC
:101E60003035204200416476616E6365643A2042F9
:101E70003C6D696E5F7365676D656E745F74696DE7
:101E8000655F75733E20533C6D696E5F6665656482
:101E9000726174653E20543C6D696E5F7472617648
:101EA000656C5F66656564726174653E20583C6D63
:101EB00061785F785F6A65726B3E20593C6D61782E
:101EC0005F795F6A65726B3E205A3C6D61785F7A1C
:101ED0005F6A65726B3E20453C6D61785F655F6A45
:101EE00065726B3E0020540020520020204D32309D
:101EF00034205000416363656C65726174696F6E74
:101F00002028756E6974732F7332293A20503C7003
:101F100072696E745F616363656C3E20523C7265EA
:101F200074726163745F616363656C3E20543C74DA
:101F3000726176656C5F616363656C3E0020204D65
:101F40003230312058004D6178696D756D204163E4
:101F500063656C65726174696F6E2028756E697453
:101F6000732F7332293A0020204D3230332058002D
:101F70004D6178696D756D20666565647261746523
:101F8000732028756E6974732F73293A0053746532
:101F900070732070657220756E69743A0020440079
:101FA00020204D3230302053002044697361626C30
:101FB00065640A0046696C616D656E7420736574B2
:101FC00074696E67733A0020286D6D2900202047E0
:101FD0003231202020203B20556E69747320696EB9
:101FE000206D6D003D3D6F6E4C6F61645365747480
:101FF000696E67733D3D0000803B4400803B4400B8
:10200000002041000096420000A0420000A04200D3
:102010000048440080CC43D0070000D00700006493
:102020000000004B00000024F4D43050C38E20C2C6
:10203000A24017828B7011127A910D816CD90AA877
:1020400061E108C7586607615143061E4B5D05C133
:1020500045A7041A411104093D9803713931034021
:1020600036DB0265339102D4305402802E1D0263A8
:102070002CEE01752AC501B028A001102781018F1F
:102080002564012B244B01E0223401AC211F018D7A
:10209000200D01801FFC00841EED00971DDF00B89D
:1020A0001CD200E61BC600201BBC00641AB200B2A2
:1020B00019A8000A19A0006A189900D117910040C8
:1020C000178B00B516840031167E00B31579003ADF
:1020D000157300C7146F0058146A00EE1366008869
:1020E00013630025135E00C7125B006C12570015C6
:1020F000125400C111510070114F0021114B00D634
:102100001049008D1047004610440002104200C0E4
:102110000F4000800F3E00420F3C00060F3B00CBFB
:102120000E3800930E37005C0E3500270E3400F396
:102130000D3200C10D3100900D3000600D2E0032C7
:102140000D2D00050D2C00D90C2B00AE0C2900859F
:102150000C29005C0C2700350C27000E0C2600E82B
:102160000B2400C40B2400A00B23007D0B23005A7A
:102170000B2100390B2100180B2000F80A1F00D991
:102180000A1E00BB0A1E009D0A1D00800A1D006376
:102190000A1C00470A1B002C0A1B00110A1A00F730
:1021A000091A00DD091900C4091900AB09190092C8
:1021B0000917007B091800630917004C091600363F
:1021C000091600200916000A091500F5081500E097
:1021D000081400CC081400B8081400A408140090D7
:1021E0000813007D0812006B0813005808120046FF
:1021F0000812003408110023081100120811000110
:10220000081100F0071000E0071000D0071000C010
:10221000071000B0070F00A107100091070E008300
:10222000070F0074070F0065070E0057070E0049DF
:10223000070E003B070D002E070E0020070D0013B0
:10224000070D0006070D00F9060C00ED060D00E075
:10225000060C00D4060C00C8060C00BC060C00B02E
:10226000060C00A4060B0099060C008D060B0082DC
:10227000060B0077060B006C060B0061060A005780
:10228000060B004C060A0042060A0038060A002E19
:10229000060A0024060A001A060A001006090007AA
:1022A000060A00FD050900F4050900EB050900E236
:1022B000050900D9050900D0050900C7050900BEB8
:1022C000050900B5050800AD050800A50509009C35
:1022D000050800940508008C050800840508007CAA
:1022E000050800740508006C050700650508005D19
:1022F000050700560508004E050700470507004082
:1023000005080038050700310507002A05070023E6
:102310000507001C050600160507000F0507000845
:1023200005060002050700FB040600F5040700EEA1
:10233000040600E8040600E2040700DB040600D5FA
:10234000040600CF040600C9040600C3040600BD4D
:10235000040600B7040600B1040500AC040600A69C
:10236000040600A00405009B0406009504050090E7
:102370000406008A04050085040500800406007A2E
:1023800004050075040500700405006B0405006673
:10239000040500610405005C0405005704050052B3
:1023A0000405004D04050048040500430405003EF3
:1023B0000404003A04050035040500300404002C30
:1023C00004050027040400230405001E0404001A69
:1023D00004040016040500110404000D040400099F
:1023E0000405000404040000040400FC030400F8D5
:1023F000030400F4030400F0030400EC030400E809
:10240000030400E4030400E0030400DC030400D838
:10241000030400D4030400D0030400CC030400C868
:10242000030300C503030024F404D9201BC40C5C7F
:102430000E9804C4095F0265077101F405F900FBF9
:1024400004B30048048700C1036900580355000322
:10245000034500BE023A008402310053022A0029DB
:1024600002250004022000E4011C00C8011900AF8D
:10247000011700980114008401130071011000611C
:1024800001100051010E0043010D0036010B002B1D
:10249000010B0020010B00150109000C01090003CC
:1024A000010800FB000800F3000800EB000700E44F
:1024B000000600DE000600D8000600D2000600CCB0
:1024C000000500C7000500C2000500BD000400B9FA
:1024D000000400B5000400B1000400AD000400A930
:1024E000000400A5000300A20003009F0004009B5D
:1024F0000003009800030095000200930003009081
:102500000003008D0002008B00030088000200869B
:1025100000020084000300810002007F0002007DB1
:102520000002007B000200790002007700010076C3
:102530000002007400020072000100710002006FCE
:102540000002006D0001006C0002006A00010069D9
:1025500000020067000100660001006500010064E0
:102560000002006200010061000100600001005FE4
:102570000002005D0001005C0001005B0001005AE8
:1025800000010059000100580001005700010056E9
:1025900000010055000100540001005300000053E9
:1025A0000001005200010051000100500001004FE5
:1025B0000001004E0000004E0001004D0001004CE3
:1025C0000001004B0000004B0001004A00010049DF
:1025D00000010048000000480001004700010046DB
:1025E00000000046000100450000004500010044D5
:1025F00000010043000000430001004200000042CF
:102600000001004100000041000100400001003FC6
:102610000000003F0001003E0000003E0001003DC0
:102620000000003D0001003C0000003C0000003CB8
:102630000001003B0000003B0001003A0000003AAE
:1026400000010039000000390001003800000038A6
:10265000000000380001003700000037000100369C
:102660000000003600000036000100350000003593
:102670000000003500010034000000340000003488
:10268000000100330000003300000033000100327D
:102690000000003200000032000100310000003173
:1026A0000000003100010030000000300000003068
:1026B0000001002F0000002F0000002F0000002F5D
:1026C0000001002E0000002E0000002E0001002D51
:1026D0000000002D0000002D0000002D0001002C46
:1026E0000000002C0000002C0000002C0001002B3A
:1026F0000000002B0000002B0000002B0001002A2E
:102700000000002A0000002A0000002A0001002921
:102710000000002900000029000000290000002915
:102720000001002800000028000000280000002808
:1027300000000028000100270000002700000027FB
:1027400000000027000000270001002600000026EE
:1027500000000026000000260000002600010025E1
:1027600000000025000000250000002500000025D5
:1027700000000025000100240000002400000024C7
:1027800000000024000000240001002300000023BA
:1027900000000023000000230000002300000023AD
:1027A000000000230001002200000022000000229F
:1027B0000000002200000022000000220001002191
:1027C0000000002100000021000000210000002185
:1027D0000000002100000021000100200000002076
:1027E0000000002000000020000000200000002069
:1027F00000000020000000200001001F0000001F5A
:102800000000001F0000001F0000001F0000001F4C
:102810000000001F0001001E0000001E0000001E3E
:102820000000001E000000232C0000B8220000560B
:102830001800003A0F0000B8080000B10400007151
:102840000200003E01000020436F756E7420583A6C
:102850000023646566696E652044454641554C54C5
:102860005F0000626564004B6420004B6920004BF0
:10287000702000504944204175746F74756E652056
:1028800066696E6973686564212050757420746888
:1028900065206C617374204B702C204B6920616E35
:1028A00064204B6420636F6E7374616E7473206672
:1028B000726F6D2062656C6F7720696E746F204354
:1028C0006F6E66696775726174696F6E2E680A0053
:1028D000504944204175746F74756E652066616956
:1028E0006C6564212074696D656F75740A005049C8
:1028F00044204175746F74756E65206661696C65FE
:1029000064212054656D7065726174757265207400
:102910006F6F20686967680A00204B643A200020C6
:102920004B693A2000204B703A200020436C6173C1
:1029300073696320504944200A00204E6F206F764F
:10294000657273686F6F740A002054753A20002016
:102950004B753A2000206D61783A2000206D696E39
:102960003A200020643A200020626961733A200016
:10297000504944204175746F74756E65207374619D
:1029800072740A00504944204175746F74756E6505
:10299000206661696C6564212054656D70657261A3
:1029A0007475726520746F6F20686967680A0042E9
:1029B000656400453100626564002C20737973748E
:1029C000656D2073746F7070656421204865617453
:1029D00065725F49443A200048656174696E6720FA
:1029E0004661696C65640048656174696E6720665C
:1029F00061696C6564004D313132205368757464CF
:102A00006F776E001000C90210012C0140012201F5
:102A100070011801B0010E01F00104015002FA002A
:102A2000B002F0003003E600D003DC009004D200D6
:102A30007005C800A006BE000008B400B009AA00D6
:102A4000D00BA000600E960060118C000015820073
:102A500020197800C01D6E00A0226400B0275A0023
:102A6000902C500000314600E0343C001038320019
:102A7000903A2800603C1E00A03D1400803E0A00F1
:102A8000203F0000544845524D414C2052554E4184
:102A900057415900546865726D616C2052756E61C2
:102AA000776179004572723A204D415854454D5036
:102AB000004D415854454D502074726967676572E6
:102AC0006564004572723A204D494E54454D5000A0
:102AD0004D494E54454D5020747269676765726563
:102AE0006400202F002042403A0020403A00205746
:102AF0003A0020573A00496E76616C696420657827
:102B00007472756465720A007C3C3E5E2B3D3F2FFB
:102B10005B5D3B2C2A225C0043616E6E6F74206FFC
:102B200070656E2073756264697220005344204999
:102B30006E6974204661696C00534420636172645D
:102B4000206F6B0A006F70656E526F6F7420666144
:102B5000696C65640A00766F6C756D652E696E69C7
:102B600074206661696C65640A004E6F20534420CE
:102B7000636172640A000A4D3234004D32332025FD
:102B800073002E0A006F70656E206661696C656463
:102B90002C2046696C653A200046696C6520736597
:102BA0006C65637465640A002053697A653A200095
:102BB00046696C65206F70656E65643A2000454E0D
:102BC0004420535542524F5554494E450A00222045
:102BD000706F73002220706172656E743A22005328
:102BE0005542524F5554494E452043414C4C207458
:102BF00061726765743A220053756263616C6C2080
:102C00004F766572666C6F770045786365656465BD
:102C100064206D617820535542524F5554494E45BA
:102C20002064657074683A002E0A0044656C65740F
:102C3000696F6E206661696C65642C2046696C65FD
:102C40003A200046696C652064656C657465643A79
:102C5000005344207072696E74696E6720627974E3
:102C60006520004E6F74205344207072696E746941
:102C70006E670A0057726974696E6720746F206608
:102C8000696C653A2000667265736800646F696EEE
:102C900067002066696C653A20004E6F7720002F30
:102CA0006175746F25632E67002020506C616E6E15
:102CB000657242756666657242797465733A200082
:102CC0002046726565204D656D6F72793A2000432C
:102CD0006F6D70696C65643A2041707220323920E2
:102CE000323032310A00204C6173742055706461B7
:102CF0007465643A20323032312D30342D31382031
:102D00007C20417574686F723A2054696E794D6108
:102D10006368696E657333440A00322E302E375F64
:102D20004457372E332E310A004D61726C696E00A4
:102D300020536F6674776172652052657365740AFB
:102D400000205761746368646F672052657365740F
:102D50000A002042726F776E206F7574205265737F
:102D600065740A002045787465726E616C20526546
:102D70007365740A00506F77657255700A0073743A
:102D80006172740A004739310A47315A350A4739A6
:102D9000300A4D38340A4D31303453300A4D313415
:102DA000305330004D31303031006572726F722017
:102DB00077726974696E6720746F2066696C650A42
:102DC00000446F6E6520736176696E672066696C7A
:102DD000652E0A004D323900456E6473746F70734E
:102DE00000255320256320256320256320256300CB
:102DF000205A3A0020593A0020583A00656E647310
:102E0000746F7073206869743A200000000A0B0226
:102E1000090C0D0E0807030401000000000000006B
:102E200000000000000000000000000000000000A2
:102E3000000000000000001211100000000000005F
:102E40000000000000000000000000000000000082
:102E50000070012C0190012701B0012201C0011D69
:102E600001F00118011002130130020E0160020985
:102E70000190020401C002FF000003FA004003F5C4
:102E8000008003F000D003EB002004E6007004E1B2
:102E900000E004DC004005D700C005D2004006CDAC
:102EA00000D006C8008007C3003008BE00F008B993
:102EB00000C009B400B00AAF00B00BAA00D00CA546
:102EC00000000EA000500F9B00C010960050129101
:102ED0000000148C00C0158700B0178200B0197D67
:102EE00000D01B7800001E730040206E0090226905
:102EF00000F024640040275F0090295A00E02B5521
:102F000000102E500020304B0010324600E03341BC
:102F10000090353C001037370070383200A0392D52
:102F200000B03A2800A03B2300603C1E00103D1971
:102F300000903D1400103E0F00703E0A00C03E0598
:102F400000003F0000403FFBFF803FF6FFC03FF125
:102F5000FF50726F62696E67204661696C6564003C
:102F6000205A3A200020593A200042656420583AFD
:102F700020003D3D6F6E55736572436F6E666972DA
:102F80006D52657175697265643D3D00220A005598
:102F90006E6B6E6F776E20636F6D6D616E643A203D
:102FA00022002042002050006F6B00204500205A74
:102FB00000205900204D393220580020453A002089
:102FC0005A3A0020593A00583A0020746F6F206C2A
:102FD0006F6E6720657874727573696F6E2070729A
:102FE0006576656E7465640A0020636F6C642065A5
:102FF0007874727573696F6E2070726576656E7421
:1030000065640A0043616E6E6F7420656E7465724C
:10301000207375626469723A20004D323520500A7F
:103020004D323400526573756D650055492050610D
:10303000757365004E6F204D61746368203A004DD2
:1030400032320A4D32310052656672657368005043
:10305000675570005067446F776E0049732046696A
:103060006C6520004973204469722000476F5570D9
:1030700044697200486173204D6564696100466966
:103080006C656E616D652053656C65637465640085
:103090004D3130303043004D313030300046696CB6
:1030A000616D656E7420537461742030202D20335F
:1030B0000046696C616D656E7420537461742030D4
:1030C000202D20320046696C616D656E742053744A
:1030D00061742030202D2031002046696C616D65BF
:1030E0006E7420526573706F6E7365204E6F005260
:1030F0006573756D652059657320647572696E67B7
:10310000207072696E74000A204E6F2046696C61EF
:103110006D656E7400496E76616C6964204F7074E1
:10312000696F6E004D3530300053746F72652053F7
:10313000657474696E677300426564205049442069
:1031400053746172746564004D3939390A4D3238EF
:103150003050305331363000424C546F7563682024
:103160005265736574004D3530320A4D353030008C
:10317000496E697420454550524F4D00486F746543
:103180006E64205049442053746172746564004534
:103190006E676C69736820416C7265616479205355
:1031A0006574004368696E657365204E6F742053C3
:1031B0007570706F7274656400496E4C616E674320
:1031C000686F696365000A202A2A2A726563646150
:1031D000742E646174615B305D203D004732380AB3
:1031E0004731204631303030205A313000556E732F
:1031F0007570706F72746564204F7074696F6E20A3
:1032000053656C65637465640047323652323535F8
:10321000004D3139305335350A4732380A47323993
:103220000A4D3430300A4D313034533231350A478B
:1032300032380A4D313039533231350A4D3432305B
:1032400053310A47315831303059313030463530FA
:1032500030300A47315A300A4D3530300A4D31315D
:103260003720536574205A204F6666736574004793
:1032700031204631303030205A302E30004732383D
:103280000A4731204631303030205A302E30004D40
:10329000353030005A204F6666736574203A202519
:1032A00073004D353030005A204F666673657420C8
:1032B0003A202573004732380A47314631353030DD
:1032C0005A302E30004732385A0A473146313530AD
:1032D000305A302E30004D383400473146313030CE
:1032E000305A302E30004732380A473146313030BC
:1032F000305A302E30004D616E75616C53657454D8
:10330000656D7000526571756573746564204F66F4
:1033100066736574204265796F6E64204C696D69CF
:103320007473005A204F6666736574203A202573C3
:1033300000526F756E64696E6720746F20737465D8
:103340007000526571756573746564204F666673AD
:103350006574200053746F702054726967676572DA
:1033600065640053746F70204E6F0053746F70501B
:1033700072696E740048616E646C652044617461AA
:103380002041646A75737420322053657474696EC9
:10339000672053637265656E200048616E646C65DA
:1033A0002044617461205072696E7446696C6520B6
:1033B000332053657474696E672053637265656E5C
:1033C000200048616E646C65204461746120507215
:1033D000696E7446696C6520322053657474696E39
:1033E000672053637265656E20004D383400486174
:1033F0006E646C652044617461205072696E74461D
:10340000696C6520506F73740048616E646C652050
:1034100044617461205072696E7446696C65205015
:10342000726500426567696E537769746368003D31
:103430003D20436865636B6B65793D3D0072656354
:103440006461742E61646472203D3D007265636442
:1034500061742E646174615B305D203D3D00776175
:103460006974776179203D3D0020202A2A2A2A2A82
:103470002A2A5254535F48616E646C6544617461DA
:103480002A2A2A2A2A2A2A2A2000526573656E646B
:103490003A200000002200250028002B002E0031D9
:1034A00000340002010000050108010B01000021A9
:1034B00000240027002A002D003000330001010005
:1034C00000040107010A01050505050705080808AC
:1034D00008020202020A0A080804040404010101A5
:1034E00001010101010303030303030303040707AD
:1034F000070C0C0C0C0C0C0C0C020202020606064B
:1035000006060606060B0B0B0B0B0B0B0B01021032
:1035100020200808102040102040800201020108ED
:10352000040201010204081020408080402010089D
:1035300004020180040201804020100804020108F6
:103540000402010102040810204080010204081056
:10355000204080544D334420453520506C757320F5
:1035600052656164792E005072696E74696E672EBF
:103570002E2E005072696E74205061757365640060
:103580006E6F74696669636174696F6E200050497B
:10359000442054756E652046696E697368656400E1
:1035A000EA000A0111241FBECFEFD1E2DEBFCDBF7A
:1035B00000E00CBF14E0A0E0B2E0EEEEFBE602E0BB
:1035C0000BBF02C007900D92A431B107D9F726E1D5
:1035D000A4E1B4E001C01D92A73AB207E1F71AE1F5
:1035E000C1EDDAE100E006C021970109802FFE015C
:1035F0000F942432C03DD10780E00807A9F70F944B
:103600007C1F0D94E5350C9400009F92AF92BF9201
:10361000CF92DF92EF92FF920F931F93CF93DF939E
:1036200000D01F921F92CDB7DEB7E9E8FBE100277B
:10363000BB27462F572FA82FAA2341F4A52F542F7D
:10364000B85FAA2319F4A52F5527B85FA03138F425
:103650005295A295452F4F70507FA42BBC5FA0348C
:1036600028F4550FAA1F550FAA1FBE5FA03818F4E3
:10367000550FAA1FB395550FAA1FEA0FF01F4491CB
:1036800051E0AA27B85081F1C8F0B0FF02C0440F42
:10369000551FB1FF04C0440F551F440F551FB2FF03
:1036A00006C052954295142F1F70407F512BB3FFD7
:1036B0001BC0A52F542F44270C94741BB195B0FF49
:1036C00002C055954795B1FF04C05595479555954E
:1036D0004795B2FF05C05295407F4295452B5F70DC
:1036E000B3FF02C0452F5527DD24CC24BB24B2E014
:1036F000649FD018C108B00AB00B749FC018B108FD
:10370000B00B849FB018B109659FC018B108B00B09
:10371000759FB018B109859FB0196A9FB018B1099B
:103720007A9FB0194D9DA12C9924332799272227E0
:103730005D9DA00C911C301F901F201FAD9D900C13
:10374000311D901F201F4C9DA00C911C301F901FFD
:10375000201F5C9D900C311D901F201FAC9D300DD3
:10376000911D201F4B9D900C311D901F201F5B9DB4
:10377000300D911D201FAB9D900D211D4B9F300DD5
:10378000911D201F5B9F900D211DAB9F200DB1E06F
:10379000BB24CC24DD24639FD018C108B00AB00B31
:1037A000739FC018B108B00B839FB018B109699F0F
:1037B000C018B108B00B799FB018B109899FB01932
:1037C000629FB018B109729FB019D61AC70AB80A19
:1037D00020F0B1E03B0F901F201F1124792F632FA1
:1037E00090E0822F0F900F900F900F900F90DF912D
:1037F000CF911F910F91FF90EF90DF90CF90BF90EE
:10380000AF909F900895AF92BF92CF92DF92EF92C8
:10381000FF920F931F93CF93DF93C1EADCE008EF91
:1038200018E081EBA82E8CE0B82EC12CD12C7601AB
:10383000C39469917991899199910F94622B288908
:1038400039894A895B890F94C32B0F94A033F801FF
:1038500061937193819391938F01C616D706E80601
:10386000F90610F46B017C01AC16BD0611F76FEF81
:103870007FEFCB01A70196010F94A1312093080996
:103880003093090940930A0950930B09DF91CF91B6
:103890001F910F91FF90EF90DF90CF90BF90AF906E
:1038A0000895CF92DF92EF92FF92809114088823BF
:1038B00009F457C0C0901008D0901108E090120889
:1038C000F090130820E030E0A901C701B6010F9481
:1038D0005D2B882309F445C020E030E040E05FE341
:1038E000C701B6010F94C32B9B01AC010F94C32BEE
:1038F0002BED3FE049E450E40F94C32B9B01AC0156
:1039000060E070E080E89FE30F9427336B017C0157
:10391000C092E90CD092EA0CE092EB0CF092EC0C25
:1039200060917D0270917E02072E000C880B990B2E
:103930000F94642B2AE037ED43E25CE30F94C32B32
:10394000A70196010F94C32B6093790270937A02BA
:1039500080937B0290937C02FF90EF90DF90CF905A
:103960000895C12CD12C80E8E82E8FE3F82ED0CF1B
:103970000F931F93CF93DF9350E0FC01E40FF51FEB
:103980008081440F551F440F551F4E545A4FEA0172
:10399000882329F188819981AA81BB81EB01088163
:1039A00019812A813B810097A105B10569F40C5961
:1039B0001F4F2F4F3F4FDA010D931D932D933C93D3
:1039C00013978FEF808306C0081B190B2A0B3B0B44
:1039D00037FDF7CFDF91CF911F910F910895188296
:1039E00019821A821B82F6CFCF93DF9324E0829F45
:1039F000C0011124EC01C551D74FFC01EF5DF74F19
:103A00008B5E974FDC012D913D914D915C916081D2
:103A10007181828193810F942D32688379838A83A7
:103A20009B83DF91CF9108958091AD059091AE0574
:103A3000A091AF05B091B0058093490290934A02DE
:103A4000A0934B02B0934C028091AB059091AC05D2
:103A50009093800280937F02089580914902909113
:103A60004A02A0914B02B0914C028093AD05909315
:103A7000AE05A093AF05B093B00580917F02909101
:103A800080029093AC058093AB0584E690E0909320
:103A9000800280937F0208958091F1129091F2123A
:103AA000891B877089F48091F90D81110DC0809177
:103AB000ED0C9091EE0C892B39F481E09091BB06CE
:103AC000911103C080E0089581E00895CF93DF93C2
:103AD000DB01F9019C919130C1F0943080F0945059
:103AE0009C938830D1F480819181009771F0019787
:103AF00091838083480F591FEA01188206C08C35D4
:103B000039F49C5F9C93943041F4DF91CF910895F8
:103B10008B3339F781E08C93F8CF20813181B90163
:103B20006F5F7F4F71836083420F531FEA01888369
:103B3000808191818F3591056CF7E7CF0F931F93AB
:103B400081E00091A5141091A6142091A714309142
:103B5000A8144091A1145091A2146091A3147091E3
:103B6000A414041715072607370708F480E01F91EF
:103B70000F91089590E080E00895282F90910F080C
:103B8000833021F495FD0FC094FD0FC0892F90E084
:103B9000B0E0A0E004C0B695A795979587952A95C3
:103BA000D2F78170089581E0089580E00895FC01C6
:103BB000659175918591949108958F929F92AF929E
:103BC000BF92CF92DF92EF92FF92CF93DF93EC01FF
:103BD0008090E7089090E808A090E908B090EA0883
:103BE00020E030E0A901C501B4010F945D2B8823CA
:103BF00009F454C0C880D980EA80FB80A7019601EF
:103C0000C501B4010F945D2B18160CF04CC0209127
:103C1000DF083091E0084091E1085091E208C701C7
:103C2000B6010F945D2B882331F1C092DF08D0924A
:103C3000E008E092E108F092E2082091E308309178
:103C4000E4084091E5085091E608688179818A810D
:103C50009B810F94C32B9B01AC0160E070E080E876
:103C60009FE30F942C3260930F02709310028093A5
:103C700011029093120260910F02709110028091D4
:103C8000110290911202DF91CF91FF90EF90DF909F
:103C9000CF90BF90AF909F908F90089560E070E0BC
:103CA00080E89FE3F0CF60E070E0CB01ECCFCF92F3
:103CB000DF92EF92FF92CF93DF93EC01CC80DD8017
:103CC000EE80FF8027E137EB41ED58EBC701B601ED
:103CD0000F948D3487FD23C023E030E044EB53E4A0
:103CE000C701B6010F945D2B1816CCF0C880D9809F
:103CF000EA80FB8027E137EB41ED58EBC701B601C5
:103D00000F948D3487FD0BC0C1E023E030E040EB21
:103D100053E4C701B6010F945D2B18160CF4C0E0F4
:103D20008C2FDF91CF91FF90EF90DF90CF9008958F
:103D30002FEB280F2A3108F047C0E22FF0E08091E6
:103D4000470590914805A0914905B0914A0504C0E6
:103D5000B695A795979587952A95D2F780FD02C0CD
:103D600081700895E75DFA4FE081EE2341F1809183
:103D7000A1079091A207E80FF92FF11D808190ED26
:103D8000980F9A3030F08E3251F4818180538A300E
:103D900098F4F0931805E093170581E008958D32AB
:103DA00011F08B3249F4818190ED980F9A3088F3AD
:103DB0008E3211F48281EACFF0E0E0E0EACF109297
:103DC000180510921705E9CF80E008950E94981E0B
:103DD000882341F081E02091170530911805232BAD
:103DE00009F480E008958F929F92AF92BF92CF9294
:103DF000DF92EF92FF92C090E905D090EA05E09043
:103E0000EB05F090EC0520E030E0A901C701B60118
:103E10000F945D2B8823E1F1A701960160E070E02B
:103E200080E89FE30F9427336B017C018090ED05C0
:103E30009090EE05A090EF05B090F00520E030E006
:103E4000A901C501B4010F945D2B882329F1A501B7
:103E5000940160E070E080E89FE30F942733C09204
:103E6000F004D092F104E092F204F092F304609333
:103E7000F4047093F5048093F6049093F704FF9094
:103E8000EF90DF90CF90BF90AF909F908F9008956C
:103E9000C12CD12C7601CACF60E070E0CB01DFCF1E
:103EA000129A08955F9A80919F0C8E7F80939F0C49
:103EB0008A9A80919F0C8D7F80939F0C809108013E
:103EC000809581708093060180919F0C8B7F8093F9
:103ED0009F0C0C94501F269A2E9A08958C3221E044
:103EE000920714F08CE291E0909356128093551251
:103EF0000C9495E9E5E2F6E01082118212821382B9
:103F000014820C9495E94F925F926F927F928F92F8
:103F10009F92AF92BF92CF92DF92EF92FF920F9358
:103F20001F93CF93DF93EC012091E1053091E205DF
:103F30004091E3055091E405688179818A819B81F4
:103F40000F942C326B017C012091E5053091E60540
:103F50004091E7055091E8056C817D818E819F81BC
:103F60000F942C324B015C01A70196016091030272
:103F70007091040280910502909106020F945D2BCE
:103F8000882309F450C0C0920302D0920402E09248
:103F90000502F09206022091F0043091F104409164
:103FA000F2045091F304C701B6010F94C32B2B0107
:103FB0003C010F94CF336B017C0120E030E0A9017C
:103FC0000F945D2B87FD70C020E030E040E450E4AA
:103FD000C701B6010F948D3418162CF4C12CD12CC6
:103FE000C0E4EC2EFE2CA7019601C301B2010F9490
:103FF0002C326093E8047093E9048093EA04909370
:10400000EB04C701B6010F9499336093E604062EC2
:10401000000C770B6F5F7F4F6430710514F064E024
:1040200070E06093E404D09101021091E604A501D0
:1040300094016091070270910802809109029091A9
:104040000A020F945D2B811133C0D11381C02091DE
:10405000CC043091CD044091CE045091CF046091B6
:10406000E8047091E9048091EA049091EB040F94C4
:10407000C32B2091D0043091D1044091D2045091AF
:10408000D3040F942D32DF91CF911F910F91FF90A8
:10409000EF90DF90CF90BF90AF909F908F907F90E8
:1040A0006F905F904F900895C12CD12C76019BCFDB
:1040B0008092070290920802A0920902B0920A022E
:1040C0002091F4043091F5044091F6045091F704E6
:1040D000C501B4010F94C32B4B015C010F94CF3386
:1040E0006B017C0120E030E0A9010F945D2B87FD7E
:1040F000F3C020E030E040E450E4C701B6010F9483
:104100008D3418162CF4C12CD12CB0E4EB2EFE2CDF
:10411000A7019601C501B4010F942C326093EC0401
:104120007093ED048093EE049093EF04C701B60101
:104130000F9499336093E704062E000C770B6F5FA2
:104140007F4F6430710514F064E070E06093E50423
:10415000C091E704D11305C0809102028C1709F4C5
:1041600070C08091E6049091E704909302028093DE
:1041700001020C2E000CDD0B25E01203C0011124FE
:10418000FC01EC0FFD1FEE0FFF1FEE0FFF1FE555AB
:10419000F84F20813181428153812093E004309394
:1041A000E1044093E2045093E3040091E504002EFF
:1041B000000C110BFC01E00FF11FEE0FFF1FEE0FC3
:1041C000FF1FE555F84F60817181828193810F94C3
:1041D0002C326093DC047093DD048093DE049093B2
:1041E000DF042091E40435E02303F0011124CE0F15
:1041F000DF1FCC0FDD1FCC0FDD1FC555D84F288129
:1042000039814A815B812093D8043093D90440934B
:10421000DA045093DB04E00FF11FEE0FFF1FEE0FE7
:10422000FF1FE555F84F60817181828193810F9462
:104230002C326093D4047093D5048093D604909369
:10424000D7048090EC049090ED04A090EE04B09020
:10425000EF042091DC043091DD044091DE045091A4
:10426000DF04C501B4010F94C32B2091E004309109
:10427000E1044091E2045091E3040F942D326B016C
:104280007C01C092D004D092D104E092D204F0928A
:10429000D3042091D4043091D5044091D604509198
:1042A000D704C501B4010F94C32B2091D8043091D9
:1042B000D9044091DA045091DB040F942D32A70108
:1042C00096010F942C326093CC047093CD048093AC
:1042D000CE049093CF04BBCEC12CD12C760118CF45
:1042E000CF92DF92EF92FF92CF93DF93EC0108968B
:1042F0000E94DD1D6B017C0120E030E0A9010F94DC
:104300005D2B20E030E0A901882359F0CE010E9406
:10431000831F9B01AC01C701B6010F94C32B9B0106
:10432000AC01688579858A859B850F942C326887D6
:1043300079878A879B87DF91CF91FF90EF90DF90FD
:10434000CF9008952F923F924F925F926F927F92FB
:104350008F929F92AF92BF92CF92DF92EF92FF9295
:104360000F931F93CF93DF93D62FC72FFC0180802D
:104370009180A280B380C501B40120E831E541E01D
:1043800050E00F94A131C9016DE671E00F94103235
:104390006B017C01C501B40120E13EE040E050E04A
:1043A0000F94A131CA01B90128E130E040E050E0AA
:1043B0000F94A131362E272E062F172F8CE3482E6F
:1043C000512C612C712CC501B401A30192010F94F1
:1043D000A131B62EA72ECA01B901A30192010F94F3
:1043E000A131CB01C114D10479F1AF92BF927F9377
:1043F0006F932F923F92FF92EF92DF92CF9280E9DC
:1044000097E19F938F93CF93DF930F94F42A8DB707
:104410009EB70E960FB6F8949EBF0FBE8DBF8D2F20
:104420009C2FDF91CF911F910F91FF90EF90DF9024
:10443000CF90BF90AF909F908F907F906F905F9044
:104440004F903F902F900895E114F104C9F0AF927E
:10445000BF927F936F932F923F92FF92EF9280E8EB
:1044600097E19F938F93CF93DF930F94F42AEDB747
:10447000FEB73C960FB6F894FEBF0FBEEDBFCFCF90
:10448000012BB9F0AF92BF927F936F932F923F921F
:1044900084E797E19F938F93CF93DF930F94F42A50
:1044A0008DB79EB70A960FB6F8949EBF0FBE8DBF0C
:1044B000B6CF892BA9F0AF92BF927F936F938CE612
:1044C00097E19F938F93CF93DF930F94F42AEDB7E7
:1044D000FEB738960FB6F894FEBF0FBEEDBF9FCF64
:1044E000AF92BF9288E697E19F938F93CF93DF932C
:1044F0000F94F42A0F900F900F900F900F900F9041
:104500008ECFEF92FF920F931F93CF93DF93CDB790
:10451000DEB78C01EDB6FEB60F94AA2A01962DB730
:104520003EB7281B390B0FB6F8943EBF0FBE2DBF08
:104530008DB79EB70196B8010F94A32A0F94861CDD
:104540000FB6F894FEBE0FBEEDBEDF91CF911F9166
:104550000F91FF90EF9008958C38910514F08CE83E
:1045600090E09093EB118093EA110C9496C1AB010B
:10457000BC014093A5145093A6146093A7147093A4
:10458000A8148DE096E10C944EB22F923F924F9278
:104590005F926F927F928F929F92AF92BF92CF92D3
:1045A000DF92EF92FF920F931F93CF93DF93CDB7DC
:1045B000DEB760970FB6F894DEBF0FBECDBF8B8716
:1045C0006C87042F122F282F30E03E872D87462F2F
:1045D00050E05A87498785E0982E929EC001939EAD
:1045E000900D1124988B8F87FA01E80FF91FEE0FB9
:1045F000FF1FEE0FFF1FE555F84F6081718182812B
:1046000093819B01AC010F941F35882309F445C1A8
:104610004B85400F6C85610F949EC0011124E98584
:10462000FA85E80FF91FEE0FFF1FEE0FFF1FE5558C
:10463000F84FC080D180E280F380040F909EA001EB
:104640001124E985FA85E40FF51FEE0FFF1FEE0F29
:10465000FF1FE555F84F0081918082807380262FDF
:1046600030E0EF85F889E20FF31FEE0FFF1FEE0F2A
:10467000FF1FE555F84F20807181798372817A831D
:1046800073817B83610F70E0EF85F889E60FF71F78
:10469000EE0FFF1FEE0FFF1FE555F84FF88BEF876A
:1046A000F081FC83EF85F889F181FD83EF85F8893E
:1046B000F281FE83EF85F889F381FF83FC01E20F2D
:1046C000F31FEE0FFF1FEE0FFF1FE555F84F208180
:1046D0002887A180B2806380FA01E60FF71FEE0FF2
:1046E000FF1FEE0FFF1FE555F84F408051803280CD
:1046F0001381202F392D482D572D602F792D882D8E
:10470000972D0F941F35882321F000E0912C812CE8
:10471000712C9601A701B601C7010F941F3588239C
:1047200021F0C02ED92CE82CF72C2C813D814E8114
:104730005F816C817D818E819F810F941F358823DD
:1047400021F01C821D821E821F82222D39814A8106
:104750005B81622D79818A819B810F941F3588232B
:1047600039F02C803D8139834E814A835F815B83A0
:104770009201432D512FB201832D912F0F941F359C
:10478000882321F0412C512C312C10E028853A2D22
:104790004B2D562D68857A2D8B2D962D0F941F3518
:1047A000882321F04886A52CB32C612E85E02D8529
:1047B0003E85829FF001839FF00D112449855A8523
:1047C000E40FF51FEE0FFF1FEE0FFF1FE555F84F2B
:1047D000FA87E9879601A701B601C7010F942D3228
:1047E000202F392D482D572D0F942C326B017C0131
:1047F000222D39814A815B81622D79818A819B8159
:104800000F942D322C813D814E815F810F942C328B
:104810009B01AC01C701B6010F942D326B017C01E5
:1048200028853A2D4B2D562D68857A2D8B2D962D6A
:104830000F942D329201432D512F0F942C329B0156
:10484000AC01C701B6010F942D3220E030E040E406
:1048500050E40F942733E985FA856083718382835E
:1048600093836C858B8560960FB6F894DEBF0FBE80
:10487000CDBFDF91CF911F910F91FF90EF90DF900F
:10488000CF90BF90AF909F908F907F906F905F90F0
:104890004F903F902F900D94C61A60960FB6F894E3
:1048A000DEBF0FBECDBFDF91CF911F910F91FF9063
:1048B000EF90DF90CF90BF90AF909F908F907F90C0
:1048C0006F905F904F903F902F90089580911705C3
:1048D00090911805009731F04AE050E070E060E0F8
:1048E0000D94782960E070E0CB0108958091170560
:1048F00090911805009731F04AE050E070E060E0D8
:104900000D944A2860E070E0CB010895CF93DF93C7
:10491000EB010E94E61E882319F00E947624EB0129
:10492000CE01DF91CF9108950E94762497FD0CC0AF
:104930000E9476246F3F71058105910509F034F4DA
:104940000E947624862F089580E008958FEF0895C1
:10495000CF93C62F0E94E61E882319F0CF910C94A6
:1049600094248C2FCF91089580911705909118056C
:10497000892B41F00E94942491E0811101C090E0C4
:10498000892F089591E0FCCFCF93DF93C82FD62FC6
:104990000E94E61E882321F0DF91CF910C94B4246D
:1049A0008C2F0E94981E811101C08D2FDF91CF9115
:1049B00008950E947624CB010895CF93DF93EB01F5
:1049C0000E94E61E882321F0DF91CF910C94D92418
:1049D000CE01DF91CF9108950F931F93CF938091D4
:1049E0001705909118050097E9F0FC018F01C1911E
:1049F0002C2F2F7D81F0C53411F0C536B9F7F801A1
:104A0000108270E060E00F94EC26F801C083CF9133
:104A10001F910F91089570E060E0CF911F910F9169
:104A20000D94EC2660E070E0CB01F1CFCF92DF92E5
:104A3000EF92FF926A017B010E94E61E882331F00B
:104A4000FF90EF90DF90CF900C94EC24C701B6015B
:104A5000FF90EF90DF90CF9008954F925F926F920A
:104A60007F928F929F92AF92BF92CF92DF92EF92FE
:104A7000FF921F93CF93DF9300D01F92CDB7DEB785
:104A800019821A821B821C82CE0101964C018FE88A
:104A9000C82E87E0D82E99E6E92E92E0F92E2BEE6B
:104AA000A22E28E0B22E10E088E5810F0E94E61EBB
:104AB000F40181934F01882309F4E0C00E94EC24A3
:104AC0002B013C01812F0E94BD1D882309F4CCC01D
:104AD000F7012081318142815381C301B2010F94DA
:104AE0002D32F60160837183828393831F5FF4E02C
:104AF000CF0ED11C84E0E80EF11C94E0A90EB11C8D
:104B0000133091F685E40E94E61E8C83882309F415
:104B1000C0C00E94EC246B017C0183E00E94BD1D9B
:104B2000882371F0209175023091760240917702CE
:104B300050917802C701B6010F942D326B017C01B0
:104B4000C0929B07D0929C07E0929D07F0929E072F
:104B50008091E005882359F18091A91482FF27C034
:104B60008C81882321F18981811103C08A81882366
:104B7000F1F02DEC3CEC4CE45DE360913608709173
:104B8000370880913808909139080F942D329B0195
:104B9000AC016091710270917202809173029091E8
:104BA00074020F948D34181614F40F940C1A40E00C
:104BB00050E0BA0186E40E94162520E030E0A90109
:104BC0000F948D34181684F40E94EC2420E030E019
:104BD00040E752E40F9427336093490270934A02EE
:104BE00080934B0290934C0280915D0C83FD28C012
:104BF0008091A606882321F12091750230917602DA
:104C0000409177025091780260919B0770919C07C8
:104C100080919D0790919E070F942C322091B306AE
:104C20003091B4064091B5065091B6060F942D32DE
:104C30006093B3067093B4068093B5069093B6065E
:104C40000F900F900F900F90DF91CF911F91FF90D9
:104C5000EF90DF90CF90BF90AF909F908F907F901C
:104C60006F905F904F900895F501208131814281CE
:104C70005381C301B2010F942C3233CFF7018081ED
:104C80009181A281B381F60180839183A283B38352
:104C90002DCF8091750290917602A0917702B0910C
:104CA000780280939B0790939C07A0939D07B093F5
:104CB0009E074ECFCF92DF92EF92FF926B017C0165
:104CC00083E3C816D104E104F10470F082E3C81A4A
:104CD000D108E108F10862E370E080E090E00E9412
:104CE000CFA90E9410C5ECCFC701B6010E94CFA981
:104CF000FF90EF90DF90CF900C9410C5CF92DF9291
:104D0000EF92FF920F931F93CF93DF936B017A0182
:104D1000EC01C455DB4F28813CE0389F8001399F6E
:104D2000100D112427FF24C0FB01118210828881FD
:104D30008F5F888388819801280F311D87FD3A9500
:104D4000C9012091DC12F6012817190629F024F078
:104D500088818C300CF43CC0808191810496803431
:104D60009C4908F475C0F60180819181049672C057
:104D700088819801280F311D87FD3A95C90120913E
:104D8000DC122817190699F294F28881A801480FBD
:104D9000511D87FD5A95FA01EE0FFF1FE40FF51F15
:104DA000EC56FD4E808187FFC2CF8881F801E80F65
:104DB000F11D87FDFA95CF01EE0FFF1FE80FF91FD8
:104DC000EC56FD4E808160E08F770E942AA8AFCF1D
:104DD000808191812881A801420F511D27FD5A959C
:104DE0009A01FA01EE0FFF1FE20FF31FEC56FD4E82
:104DF00021813281820F931FF70191838083888103
:104E00009801280F311D87FD3A95F901EE0FFF1F1C
:104E1000E20FF31FEC56FD4E808187FF20C0888192
:104E2000080F111D87FD1A95F801EE0FFF1FE00F07
:104E3000F11FEC56FD4E808161E08F77DF91CF91BD
:104E40001F910F91FF90EF90DF90CF900C942AA8C4
:104E500080E49CE9F701918380838FEF8883DF9161
:104E6000CF911F910F91FF90EF90DF90CF90089519
:104E70000F931F93CF93DF9305EB1CE0CEECD1E1B2
:104E8000F80121913191419151918F0160E070E0E1
:104E900080E89FE30F9427336993799389939993DB
:104EA000F1E1CE3DDF0761F70F944B18DF91CF9111
:104EB0001F910F910C94031CCF92DF92EF92FF92FF
:104EC000CF93DF932091A00C222329F1EC010896C7
:104ED0000E94DD1D6B017C0120E030E0A9010F94F0
:104EE0005D2B20E030E0A901882359F0CE010E941B
:104EF000831F9B01AC01C701B6010F94C32B9B011B
:104F0000AC01688579858A859B850F942D326887E9
:104F100079878A879B87DF91CF91FF90EF90DF9011
:104F2000CF9008952F923F924F925F926F927F920F
:104F30008F929F92AF92BF92CF92DF92EF92FF92A9
:104F40000F931F93CF93DF93CDB7DEB76C970FB658
:104F5000F894DEBF0FBECDBF8C015B015A8349833D
:104F6000FC01EF5AFF4F2081318142815381298713
:104F70003A874B875C87CA01B9010F94622B6B019A
:104F80007C01D5012D913D914D915C910F94C32BE6
:104F90000F940B332B013C01E981FA81208131818F
:104FA00042815381C701B6010F94C32B0F940B3379
:104FB0004B015C01C301B2010F94A033698B7A8B62
:104FC0008B8B9C8B683771058105910540F428E730
:104FD00030E040E050E0298B3A8B4B8B5C8BC50175
:104FE000B4010F94A0336D877E878F87988B6837C5
:104FF00071058105910540F448E750E060E070E0FC
:105000004D875E876F87788BF801E35AFF4F4080AA
:10501000518062807380C301B2010F94642B698355
:105020007A838B839C8369897A898B899C890F9485
:10503000622B6D8B7E8B8F8B988F20E030E0A901E7
:1050400069817A818B819C810F945D2B882309F47F
:10505000E1C1A7019601C701B6010F94C32B4B0113
:105060005C012D893E894F89588DCA01B9010F9481
:10507000C32B9B01AC01C501B4010F942C324B0131
:105080005C0129813A814B815C81CA01B9010F948D
:105090002D329B01AC01C501B4010F9427330F944D
:1050A0000B330F94A0336D837E838F83988766279D
:1050B0007727CB0164197509860997090F94642B2A
:1050C0004B015C016D857E858F8598890F94622BDD
:1050D0002B013C0120E030E0A901C501B4010F948F
:1050E0005D2B882309F49AC1A3019201C301B20187
:1050F0000F94C32B698F7A8F8B8F9C8FA70196019A
:10510000C701B6010F94C32B9B01AC01698D7A8D49
:105110008B8D9C8D0F942C326B017C01A501940129
:10512000C501B4010F942D329B01AC01C701B6013A
:105130000F9427330F94CF33D80195968D909D907F
:10514000AD90BC909897750164012D813E814F818F
:105150005885C21AD30AE40AF50A0F94A033C61A76
:10516000D70AE80AF90AF7FE8EC02D893E894F89D1
:10517000588DCA01B9010F94C32B6B017C012981A1
:105180003A814B815C81CA01B9010F942D32698744
:105190007A878B879C8720E030E0A90169817A813A
:1051A0008B819C810F945D2B882309F43BC1C50141
:1051B000B4010F94622B29853A854B855C850F9449
:1051C000C32BA70196010F942C326D837E838F83AE
:1051D0009887A3019201C301B2010F94C32B9B01D5
:1051E000AC016D817E818F8198850F942D322B01CA
:1051F0003C0120E030E040E850E469817A818B8115
:105200009C810F94C32B9B01AC01C301B2010F948D
:1052100027330F940B332B013C0120E030E0A90130
:105220000F948D3418161CF0412C512C3201C301FF
:10523000B2010F94A0336D837E838F839887861687
:105240009706A806B90620F48D829E82AF82B886A2
:105250006D817E818F8198850F94622B29853A8597
:105260004B855C850F94C32BA70196010F942D32BB
:105270000F94DB340F94A03369877A878B879C87E0
:10528000C12CD12C760169857A858B859C852989ED
:105290003A894B895C89621B730B840B950B0F94C5
:1052A000622B29813A814B815C810F94273320E066
:1052B00034E244EF59E40F94C32B0F94A0334B0115
:1052C0005C0169857A858B859C852D853E854F851A
:1052D0005889621B730B840B950B0F94622B2981E9
:1052E0003A814B815C810F94273320E034E244EF14
:1052F00059E40F94C32B0F94A0332B013C013FE6DC
:1053000083169104A104B10408F090C0F401EE0FDB
:10531000FF1FEE0FFF1FE353F64E85919591A59168
:10532000B4918983292E3A2EBD8B4FE64416510441
:105330006104710408F083C0F201EE0FFF1FEE0F4D
:10534000FF1FE353F64E45915591659174919A0173
:10535000CB014D815E816F817885D80199964D93FF
:105360005D936D937C939C974C0D5D1D6E1D7F1D11
:10537000F80145A756A767A770ABEB5AFF4F4989BD
:105380005A896B897C894083518362837383D59664
:105390008D929D92AD92BC92D897F80141AE52AEDB
:1053A00063AE74AEFD9649814083218232825D896D
:1053B00053833496208331838283938369857A85EE
:1053C0008B859C85D1966D937D938D939C93D4977B
:1053D00078962D853E854F85588920833183428379
:1053E00053836C960FB6F894DEBF0FBECDBFDF912E
:1053F000CF911F910F91FF90EF90DF90CF90BF90D2
:10540000AF909F908F907F906F905F904F903F9064
:105410002F90089560E070E0CB0141CE60E070E035
:10542000CB0188CE60E070E0CB01F3CEC501B401C2
:105430000E94051B6983272E382E9D8B76CFC301D2
:10544000B2010E94051B9B0184CF8091F1129091C3
:10545000F212891B877019F490E080E00895909112
:10546000EE12992351F0833030F48FEF890F19F049
:105470008093EE12F1CF1092EE128091F21227E695
:10548000829FC00111248B5D964FFC01208120FD7D
:10549000E3CF2091F2122F5F27702093EF1230910B
:1054A000F2122091F012321304C02091EF122093D7
:1054B000F012089590916F0081E091FD02C080E0AC
:1054C000089590916F009D7F90936F00089580FFE5
:1054D00004C090919F0C90FD8E7F81FF05C090913C
:1054E0009F0C969590FD8D7F82FF06C090919F0C3A
:1054F0009695969590FD8B7F08958F929F92AF928F
:10550000BF92CF92DF92EF92FF92CF93DF932091E1
:105510004D02222309F49EC0EC018091B105C82EF2
:10552000D12CF12CE12C80FF2CC080904F02909068
:105530005002A0905102B0905202288139814A81D4
:105540005B81C501B4010F948D34181624F4888250
:105550009982AA82BB8280905B0290905C02A090AC
:105560005D02B0905E02288139814A815B81C5016C
:10557000B4010F945D2B87FF04C088829982AA82B0
:10558000BB82D701C601B695A7959795879580FFF1
:105590002CC08090530290905402A0905502B0907D
:1055A00056022C813D814E815F81C501B4010F946B
:1055B0008D34181624F48C829D82AE82BF82809036
:1055C0005F0290906002A0906102B09062022C8114
:1055D0003D814E815F81C501B4010F945D2B87FF32
:1055E00004C08C829D82AE82BF8282E0F694E794F2
:1055F000D794C7948A95D1F7C0FE2CC0C0905702AB
:10560000D0905802E0905902F0905A0228853985CE
:105610004A855B85C701B6010F948D34181624F4B2
:10562000C886D986EA86FB86C0906302D090640261
:10563000E0906502F0906602288539854A855B8591
:10564000C701B6010F945D2B87FF04C0C886D986B9
:10565000EA86FB86DF91CF91FF90EF90DF90CF90AD
:10566000BF90AF909F908F900895CF92DF92EF926E
:10567000FF920F931F93C12CD12C76018C0125E74B
:1056800032E041E752E06DE672E089E692E00F9485
:1056900068001F910F91FF90EF90DF90CF900895D9
:1056A0000D944B1880919E05659B6EC08061809320
:1056B0009E059091030180919E0591FF67C08062D5
:1056C00080939E0580919E054B9B62C08460809371
:1056D0009E0580919E0590919D05981709F45AC0EA
:1056E00092E090939C0580939D058091B80681116E
:1056F00005C080919F07882309F459C08091050651
:1057000080FF10C08091B90680FD0CC080919B0580
:1057100084FF08C08091FB0680618093FB0680E0D7
:105720000E949ACD80910506869580FF11C08091D8
:10573000B906869580FD0CC080919B0585FF08C049
:105740008091FB0680628093FB0681E00E949ACDE7
:10575000809105068695869580FF29C08091B906BF
:105760008695869580FF23C080919F078823F9F056
:1057700080919B0582FF1BC08091FB068460809313
:10578000FB0682E00C949ACD8F7E91CF8F7D98CFCF
:105790008B7F9DCF80919C05882309F4A6CF8150F3
:1057A00080939C058111A1CF90939B059ECF089576
:1057B0008091B806811104C080919F07882331F041
:1057C00062E070E080E090E00C945A2608950F9318
:1057D0001F9380918C11813019F50E9402AA0091CB
:1057E000BA051091BB052091BC053091BD05601B29
:1057F000710B820B930B28EE33E040E050E00F94E6
:10580000A1316091BE057091BF058091C005909156
:10581000C105620F731F841F951F1F910F9108957B
:105820006091C2057091C3058091C4059091C50532
:10583000D6CF10928C111092BA051092BB0510921F
:10584000BC051092BD051092C2051092C3051092BE
:10585000C4051092C5051092BE051092BF051092A6
:10586000C0051092C1050895CF92DF92EF92FF928A
:10587000CF93DF93C62FFC01C080D180E280F380FC
:1058800020E030E0A901C701B6010F945D2B20E0B4
:1058900030E0A90187FD14C020E030E048EC52E47C
:1058A000C701B6010F948D3424E630E040E050E0AB
:1058B000181634F0C701B6010F9499339B01AC015F
:1058C000C230A0F4D0E0C05ED64FAFEFB0E00F948E
:1058D000E23124E630E040E050E00F94C3312F3F46
:1058E000310519F010F02FEF30E02883DF91CF91D0
:1058F000FF90EF90DF90CF9008958091090180FD97
:1059000006C08091A91483FB882780F9089580E060
:105910000895CF92DF92EF92FF92FC01C080D18078
:10592000E280F380663019F510922A0610922B0659
:1059300010922C0610922D0610922E060E9496C1EF
:1059400020E030E0A901C701B6010F945D2B87FF6D
:105950001DC0C12CD12C7601C701B6010F949A3419
:10596000CB01FF90EF90DF90CF900C94AC220E947F
:105970007A1F20E030E0A901C701B6010F945D2B2A
:1059800087FF15C0C12CD12C760121C020E030E06A
:105990004CE053E4C701B6010F948D341816E4F6B9
:1059A000C12CD12C9CE0E92E93E4F92ED5CF20E038
:1059B00030E046E953E4C701B6010F948D34181660
:1059C00034F4C12CD12C86E9E82E83E4F82EC701EB
:1059D000B6010F949A34CB01FF90EF90DF90CF90F7
:1059E0000C946E1F90919F0C977081E0973009F096
:1059F00080E008952091990520FF14C020E83EE33F
:105A0000629FA001639F500D729F500D1124CA0127
:105A10009695879596958795009731F08A95000021
:105A2000E9F708950C945A260895CF93DF931092C6
:105A30005E0C1092EF0C1092F10C1092F00C109280
:105A4000980510929705CFEFDFEF8091A91485FD9F
:105A500007C00E94AFADD0932813C0932713F5CF92
:105A60008FEF9FEF9093281380932713DF91CF91AF
:105A700008958F929F92AF92BF92CF92DF92EF9252
:105A8000FF920F931F93CF93DF9310924C051092C8
:105A90004B052FE3209346051092450510924405CF
:105AA000109243051092470510924805109249053F
:105AB00010924A059C01F90190812F5F3F4F90326F
:105AC000D1F39E34C9F4818190ED980F9A3020F083
:105AD0008D3211F08B3281F432969F012F5F3F4F50
:105AE000808180538A3008F47BC09F012F5F3F4F35
:105AF0008081803209F476C0F093A207E093A10779
:105B00008F010F5F1F4FC0816AE270E0C8010F94E0
:105B10007B35009731F0FC01319780818032E1F3D1
:105B20001182CD3429F0C43519F0C73409F04BC0C7
:105B3000F80180810F5F1F4F8032D1F380538A308C
:105B400008F041C0C093460530E020E04AE0DF01A4
:105B50001196429FC001439F900D11249C01205338
:105B600031098081280F311D87FD3A95818190EDA3
:105B7000980F9A30C8F130934505209344058E3232
:105B800061F4329690E04AE0DF0131968C9150ED5D
:105B9000580F5A3058F190934305CD01DC0101961E
:105BA0004C914032D9F3CD3489F52E31310539F09D
:105BB00018F52731310519F02C31310539F5B0933D
:105BC0004C05A0934B05DF91CF911F910F91FF9052
:105BD000EF90DF90CF90BF90AF909F908F900895FF
:105BE000F9017BCFF90181CFFD01B1CF949F800DE9
:105BF000112490ED980FC8CF2537310538F027379D
:105C00003105E8F2203A83E03807C9F2D091A107C4
:105C100040E050E0BA0110E000E0C12CD12C760148
:105C2000C394FD0131968C91882309F47FC08132A1
:105C3000E1F4CD34D1F420323105B9F44093470575
:105C4000509348056093490570934A05F0934C05BD
:105C5000E0934B0563E270E0CF010F947B35009732
:105C600009F4B1CFFC011082AECF81548A3108F023
:105C700058C0DF019D91903291F0A0EDA90FAA309C
:105C8000E8F09E3271F4918190539A30B8F001158A
:105C9000110519F48F010150110990E013C0FD01A5
:105CA000E8CF9D3211F09B3291F79181A0EDA90FC1
:105CB000AA3020F09E3259F79281E6CF9E2F9D1B8D
:105CC000309759F3A82FB0E04601570104C0880C63
:105CD000991CAA1CBB1C8A95D2F7482959296A2904
:105CE0007B29A75DBA4F9C9380818154DF018A3163
:105CF00008F497CFDF018191882309F492CF90EDCA
:105D0000980F9A30B8F393ED980F923098F38B3246
:105D100089F3CD010196EC91E03209F082CFDC01EC
:105D2000F8CF0115110501F78D01DECF10934C0559
:105D300000934B05409347055093480560934905F0
:105D400070934A0540CF4F925F926F927F928F92ED
:105D50009F92AF92BF92CF92DF92EF92FF92CF933A
:105D6000DF9300D000D01F921F92CDB7DEB75C0149
:105D7000DB01CD90DD90ED90FC90E091EC12F09184
:105D8000ED12FE83ED8384819581A681B78189839D
:105D90009A83AB83BC839C01AD01C701B6010F940C
:105DA0002C322B013C01F50180809180A280B380D0
:105DB000AD81BE818D919D910D90BC91A02D8D8363
:105DC0009E83AF83B88727E137EB41ED58EBC301E2
:105DD000B2010F948D3487FDD1C023E030E044EB55
:105DE00053E4C301B2010F945D2B18160CF4C6C026
:105DF0002D813E814F815885C501B4010F942C320D
:105E00002B013C0127E137EB41ED58EB0F948D342A
:105E100087FDB4C023E030E040EB53E4C301B2019E
:105E20000F945D2B18160CF4A9C020E030E0A901F6
:105E30006D817E818F8198850F942D322B013C01DD
:105E400020E030E040E450E40F945D2B87FF05C074
:105E5000412C512C30E4632E762C27E137EB41EDB9
:105E600058E3C301B2010F942C329B01AC01C50170
:105E7000B4010F948D3487FD81C020E030E040EB09
:105E800053E46D817E818F8198850F942D322B0193
:105E90003C0120E030E84EEA53E40F948D341816AC
:105EA0003CF4412C20E8522E2EEA622E23E4722E7E
:105EB00027E137EB41ED58E3C301B2010F942D32D6
:105EC0009B01AC01C501B4010F945D2B18160CF4B5
:105ED00055C020E030E0A90169817A818B819C81E5
:105EE0000F942D324B015C0120E030E040EE51E494
:105EF0000F945D2B87FF06C0812C912C90EEA92E6C
:105F000091E4B92E27E137EB41ED58E3C501B40127
:105F10000F942C329B01AC01C701B6010F948D3454
:105F200087FD2CC020E030E044EB53E469817A81A6
:105F30008B819C810F942D324B015C0120E030E07D
:105F400046EA53E40F948D34181634F4812C912CC6
:105F500086EAA82E83E4B82E27E137EB41ED58E31B
:105F6000C501B4010F942D329B01AC01B1E0B9839E
:105F7000C701B6010F945D2B18160CF419828981A4
:105F800028960FB6F894DEBF0FBECDBFDF91CF913C
:105F9000FF90EF90DF90CF90BF90AF909F908F9049
:105FA0007F906F905F904F900895EDE2F8E082EB64
:105FB000DF011D928A95E9F708958091E00581112E
:105FC00004C00E94D52F0C9410BB8091A91482FDAF
:105FD0000D940C1A089580912D08882361F09091FA
:105FE000DE08891308C08091A91483FF04C08BE6E2
:105FF00098E00C94DAB980E00895FC012381211126
:106000000C940FB60895EFE6F0E080818260808303
:106010000895CF92DF92EF92FF92CF93DF93C82F34
:106020000E945A2A94E0C99FE0011124FE01ED5E0E
:10603000F94FC080D180E280F38081110E9403304B
:10604000C253DE4EC701B6010F94642B28813981FB
:106050004A815B810F94C32BDF91CF91FF90EF902A
:10606000DF90CF9008958F929F92AF92BF92CF9280
:10607000DF92EF92FF921F93CF93DF93CDB7DEB7FE
:1060800060970FB6F894DEBF0FBECDBF182F80E02B
:106090000E9409304B015C0180929F059092A005FF
:1060A000A092A105B092A20581E00E9409306B0187
:1060B0007C01C092A305D092A405E092A505F092C0
:1060C000A60582E00E9409306093A7057093A80599
:1060D0008093A9059093AA051D861E861F86188A9F
:1060E00089829A82AB82BC82CD82DE82EF82F88680
:1060F00069877A878B879C8783E00E9409306D8748
:106100007E878F87988B8091A00C882321F0CE0109
:1061100001960E9470211E3FD9F480E1FE01319664
:10612000A9E6B2E001900D928A95E1F760960FB66C
:10613000F894DEBF0FBECDBFDF91CF911F91FF90CE
:10614000EF90DF90CF90BF90AF909F908F90089589
:1061500084E0189FF0011124DF01A759BD4F81E0B1
:1061600090E08C0F9D1FE80FF91F408151816281E3
:1061700073814D935D936D937C931397D7CFCF929B
:10618000DF92EF92FF92CF93DF93C82F0E945A2A9B
:1061900094E0C99FE0011124FE01E95FF94FC0803E
:1061A000D180E280F38081110E940330C253DE4E21
:1061B000C701B6010F94642B288139814A815B8124
:1061C0000F94C32BDF91CF91FF90EF90DF90CF9092
:1061D00008950E945A2A9091F2129093F11290938E
:1061E000F0129093EF1294E69093EE1220ED33E0CC
:1061F000309324092093230981110E94033081E008
:10620000809306060895CF93DF93CDB7DEB72C9722
:106210000FB6F894DEBF0FBECDBF0F9429190E94B0
:106220005A2A9CE0E3E1F6E0DE01119601900D921E
:106230009A95E1F781110E940330CE0101960E94E8
:106240007ACD2C960FB6F894DEBF0FBECDBFDF918E
:10625000CF9108952F923F924F925F926F927F92CB
:106260008F929F92AF92BF92CF92DF92EF92FF9266
:106270000F931F93CF93DF9300D0CDB7DEB78090FD
:10628000690290906A02A0906B02B0906C024090FC
:106290006D0250906E0260906F0270907002C0901C
:1062A0007102D0907202E0907302F09074020E942A
:1062B000031C0E94511C0DEA1CE18FE492E09B83B9
:1062C0008A8381EA282E8CE1382E198289810E94E6
:1062D000F41CC8010E94D71DEA81FB816193719370
:1062E00081939193FB83EA83C1010E94D71DEA81C8
:1062F000FB816087718782879387F981FF5FF983CC
:106300000C5F1F4F84E0280E311CF330F9F681EF4B
:1063100095E00F948E190E94F31E0E943827A50164
:1063200094016091690270916A0280916B02909170
:106330006C020F945D2B81111CC0A301920160912E
:106340006D0270916E0280916F02909170020F94B5
:106350005D2B81110EC0209171023091720240912B
:10636000730250917402C701B6010F945D2B88230C
:10637000B9F00F900F900F90DF91CF911F910F9177
:10638000FF90EF90DF90CF90BF90AF909F908F9055
:106390007F906F905F904F903F902F900C940331BF
:1063A0000F900F900F90DF91CF911F910F91FF9061
:1063B000EF90DF90CF90BF90AF909F908F907F90A5
:1063C0006F905F904F903F902F9008958091E211D1
:1063D0009091E311892B79F48091E2119091E3116E
:1063E000892B49F42091E2113091E31181E0232BB4
:1063F00019F480E0089581E008951092FD048091E1
:10640000220290912302A0912402B0912502809350
:10641000FD059093FE05A093FF05B0930006089537
:106420009091F9111092F911923071F0943079F045
:10643000913099F4813089F48091FD04882369F0CA
:10644000109226020C94FD3110929E0C089584EB5C
:1064500098E19093EE0C8093ED0C08959091A9141F
:1064600093FB882780F993FF06C081E09091101676
:10647000911101C080E00895CF93C0919A05CF7724
:1064800039F50E942E32882319F18091A114909140
:10649000A214A091A314B091A4140097A105B10572
:1064A000B9F0BC01CD016D597F4F8F4F9F4F24E64E
:1064B00030E040E050E00F94A1316091A51470915C
:1064C000A6148091A7149091A8140F94A131C22F03
:1064D0008C2FCF910895E0E2F9E0108211820895A7
:1064E00081E00895DC01EC918E2F90E0FC01EE0F2D
:1064F000FF1FE80FF91FEC56FD4E80818F778083D8
:1065000008958F929F92AF92BF92CF92DF92EF92B7
:10651000FF920F93CF93DF931F92CDB7DEB75C014D
:106520007B0149016B01C40ED51EF501808191816B
:106530000F947B318983002311F0F7018083BE0122
:106540006F5F7F4FC4010E947FE9F50180819181D7
:10655000019691838083FFEFEF1AFF0AEC14FD048C
:1065600021F780E00F90DF91CF910F91FF90EF9096
:10657000DF90CF90BF90AF909F908F9008950F9332
:10658000AB010091F50521E0022726EF35E0BC01C3
:1065900086ED95E00E9481320F910895009781F475
:1065A0001092900082E080939100109295001092DA
:1065B0009400C19A80917100826080937100089567
:1065C000019761F41092A00082E08093A1001092E4
:1065D000A5001092A40089BB8093720008957F9259
:1065E0008F929F92AF92BF92CF92DF92EF92FF92E3
:1065F0000F931F93CF93DF93EC017B018881883148
:1066000008F0C3C090E0FC01EE0FFF1FE80FF91F78
:10661000EC56FD4E80818F770E946FF019821A82AE
:1066200088812CE0622F0F940432829FB0011124E4
:1066300030E020E0AB01420F531FFA01EE0FFF1FC5
:10664000E40FF51FEC56FD4E908197FD08C02F5FBB
:106650003F4F2C30310571F790E00E94CE327880A8
:10666000072D10E06801CC0CDD1CF601E00FF11FD6
:10667000EC56FD4E80818068808377FC86C080E286
:10668000E81682E0F8060CF03FC08A8128E532E087
:10669000281B310987FD3395220F331F220F331F2B
:1066A000032E000C440B550B898178E8872E912C22
:1066B000881A910887FD9394880C991C880C991C62
:1066C000092C000CAA08BB0860E070E0CB01F7FCC5
:1066D0000AC0B701653B710514F064EB70E0072E4A
:1066E000000C880B990B281939094A095B090F948A
:1066F000913124EB30E040E050E00F94C331820E42
:10670000931EA41EB51E740187E18715D8F0298158
:1067100088E890E0821B910927FD9395880F991FC7
:10672000880F991FE816F90604F502972FB7F89419
:10673000E601C00FD11FCC56DD4E880F991F9A83FA
:1067400089832FBF62E370E080E090E0DF91CF911A
:106750001F910F91FF90EF90DF90CF90BF90AF907F
:106760009F908F907F900C945A262A8188E592E022
:10677000821B910927FD9395880F991F880F991FF8
:10678000E816F90694F6C701D0CFDF91CF911F919B
:106790000F91FF90EF90DF90CF90BF90AF909F90C0
:1067A0008F907F900895CF93DF93EB01682F70E077
:1067B0008DED92E10E94EF32688179818A819B811F
:1067C000643F21E072078105910520F464EF71E0D8
:1067D00080E090E00E945A2689B183FB882780F9E7
:1067E000DF91CF910895CF93DF9300D01F92CDB763
:1067F000DEB78EEE92E0A0E0B0E089839A83AB83AF
:10680000BC83BE016F5F7F4F8AE50E94D3330F9038
:106810000F900F900F90DF91CF910895CF93DF935A
:1068200000D01F92CDB7DEB78EEE92E0A0E0B0E0D0
:1068300089839A83AB83BC83BE016F5F7F4F8AE0FD
:106840000E94D3330F900F900F900F90DF91CF9154
:106850000895CF93DF9300D01F92CDB7DEB784EFBA
:1068600091E0A0E0B0E089839A83AB83BC83BE0152
:106870006F5F7F4F80EA0E94D3330F900F900F908D
:106880000F90DF91CF9108951F920F920FB60F9244
:1068900011240BB60F922F933F934F935F936F93F7
:1068A0007F938F939F93AF93BF93EF93FF9348EAA8
:1068B00050E064EA70E081E090E00E947E26FF9163
:1068C000EF91BF91AF919F918F917F916F915F9168
:1068D0004F913F912F910F900BBE0F900FBE0F90D5
:1068E0001F9018951F920F920FB60F9211240BB69E
:1068F0000F922F933F934F935F936F937F938F9359
:106900009F93AF93BF93EF93FF9348E950E064E9FF
:1069100070E090E080E00E947E26FF91EF91BF91B1
:10692000AF919F918F917F916F915F914F913F9127
:106930002F910F900BBE0F900FBE0F901F901895C8
:106940009091D10095FD0CC09091D00095FF08C0AA
:106950008093D6008091D00080648093D000089509
:1069600020912A042F5F2F770FB607FC27C0909144
:106970002B04921328C09091D00095FF1EC09091D7
:106980002B0440912A04941306C09091D1009F7D5E
:106990009093D10012C0E92FF0E0E65DFB4F328109
:1069A0009F5F9F773093D60090932B043091D00057
:1069B00030643093D000491741F3D9CF90912B0424
:1069C000921301C0FBCFE0912A04F0E0E65DFB4F9B
:1069D000828320932A048091D10080628093D10029
:1069E00008958F929F92AF92BF92CF92DF92EF92D3
:1069F000FF920F931F93CF93DF937C0121E5E20E6B
:106A0000F11CD7014C914A3509F0A4C06C01B2E5E4
:106A1000CB0ED11CF6013081353A09F09BC0EC0158
:106A2000C05BDF4F2881233008F494C08C010056EE
:106A30001F4FD8014C93E15BFF4F30833196208389
:106A4000EF54F1093081E05BFF4F30833038B1F40F
:106A50003196AC54B1093C913083E854F109AF5AF6
:106A6000BF4F50E040E02250330B42175307CCF4A5
:106A7000808132968D934F5F5F4FF7CF233031F592
:106A8000313809F074C0FC01EC55FF4FDC01AC5A01
:106A9000BF4F2C9120833196885A9F4FDC018C91F7
:106AA00080834801B12CA12C888190E002968A1540
:106AB0009B050CF43FC0F40181914F010E94A0346A
:106AC0000E94C2E9FFEFAF1ABF0AEECF323821F5BC
:106AD000FC01EC5AFF4F30814181E05BFF4F408366
:106AE00031963083DC01AA55BF4F50E040E023507F
:106AF000330B42175307ACF6FA01EE7FE45AFF4F0F
:106B0000E80FF91F608171817C9311966C93119746
:106B10004E5F5F4F1296EDCF243019F6333809F6E9
:106B2000FC01EC5AFF4F20813181E05BFF4F308345
:106B30003196B0CF80E5DE011D928A95E9F78AE1B2
:106B4000F80111928A95E9F78AE5D7018C9385EAD5
:106B5000F6018083DF91CF911F910F91FF90EF900D
:106B6000DF90CF90BF90AF909F908F900895323874
:106B700009F097CFADCFAF92BF92CF92DF92EF9255
:106B8000FF920F931F93CF93DF93EC0184E6C82EFF
:106B900080E2D82EE12CF12C02E8A12C90E2B92E53
:106BA00015E000933614C0923714D0923814E09256
:106BB0003914F0923A14B0924014A0923F141093FA
:106BC000331483EE93E10E94F1348FEFC81AD80A90
:106BD000E80AF80A88E7C81680E2D806E104F1045A
:106BE00001F724E630E240E050E0BE0183EE93E19D
:106BF000DF91CF911F910F91FF90EF90DF90CF9099
:106C0000BF90AF900C94C7E9CF92DF92EF92FF92C2
:106C10000F931F93CF93DF93CDB7DEB77C01CDB633
:106C2000DEB60F94AA2A01962DB73EB7281B390B62
:106C30000FB6F8943EBF0FBE2DBF0DB71EB70F5F46
:106C40001F4FB701C8010F94A32AC8010E94BB358A
:106C50000FB6F894DEBE0FBECDBEDF91CF911F916F
:106C60000F91FF90EF90DF90CF9008958F929F92B9
:106C7000AF92BF92CF92DF92EF92FF920F931F934A
:106C8000CF93DF930E94152D3AE0C32E30E2D32E2E
:106C9000E12CF12C15E002E846015701CAE0D0E0F2
:106CA0001092401410923F14109333140093361432
:106CB0008092371490923814A0923914B0923A14FA
:106CC00083EE93E10E94F13421978FEF881A980A9E
:106CD000A80AB80A209721F78AE0C80ED11CE11C47
:106CE000F11C82EDC81680E2D806E104F104A1F699
:106CF000C12C20E2D22EE12CF12CD5E0C2E810927A
:106D0000401410923F14D0933314C0933614C092A1
:106D10003714D0923814E0923914F0923A1483EE7A
:106D200093E10E94F1341092401410923F14D093DA
:106D30003314C0933614D701C6018C529F4FAF4F06
:106D4000BF4F8093371490933814A0933914B093A5
:106D50003A1483EE93E10E94F1348FEFC81AD80AF7
:106D6000E80AF80A8AE0C81680E2D806E104F104CD
:106D700031F69EEDC92E90E2D92EE12CF12CD5E012
:106D8000C2E81092401410923F14D0933314C09371
:106D90003614C0923714D0923814E0923914F0921D
:106DA0003A1483EE93E10E94F1348FEFC81AD80AA7
:106DB000E80AF80A86EEC81680E2D806E104F10473
:106DC00001F7CC24C39482E1D82EE12CF12C0AE007
:106DD00010E0D5E0C2E81093401400933F14D09324
:106DE0003314C0933614C0923714D0923814E09202
:106DF0003914F0923A1483EE93E10E94F134109327
:106E0000401400933F14D0933314C0933614D70129
:106E1000C6018096A11DB11D80933714909338143C
:106E2000A0933914B0933A1483EE93E10E94F134A5
:106E30008FEFC81AD80AE80AF80A85E1C81682E175
:106E4000D806E104F10439F682E190E09093401411
:106E500080933F14D0933314C093361484E190E1AF
:106E6000A0E0B0E08093371490933814A0933914C5
:106E7000B0933A1483EE93E1DF91CF911F910F917C
:106E8000FF90EF90DF90CF90BF90AF909F908F904A
:106E90000C94F1341F920F920FB60F9211240BB67F
:106EA0000F922F938F939F93EF93FF9380912B04D7
:106EB00020912A04821306C08091D1008F7D809397
:106EC000D10012C0E82FF0E0E65DFB4F92818F5FAA
:106ED0008F779093D60080932B049091D00090648C
:106EE0009093D000281741F3FF91EF919F918F91DC
:106EF0002F910F900BBE0F900FBE0F901F90189503
:106F00001F920F920FB60F9211240BB60F920F9390
:106F10001F932F933F934F935F936F937F938F9321
:106F20009F93AF93BF93CF93DF93EF93FF93C09162
:106F3000D60000914E05D0914D0511E01D0F1F7335
:106F400090912904913108F09FC0E92FF0E0882743
:106F5000E355F84C8F4F0D942432BE37ED37FC3794
:106F60000B3812384438163844381A381E3844382A
:106F7000223826382A38313844383C38C03229F093
:106F800028F5CA3011F0CD3031F5011731F0ED2F71
:106F9000F0E0E35BFA4FC283D12FD0934D05FF9110
:106FA000EF91DF91CF91BF91AF919F918F917F91A1
:106FB0006F915F914F913F912F911F910F910F9082
:106FC0000BBE0F900FBE0F901F901895CD3481F01F
:106FD00081E0CE3471F080E10CC0CA3338F4C033A4
:106FE000A0F6C03291F2CD32B1F7CFCFCD3499F7C0
:106FF00082E080932904C9CFC13359F018F4C0321C
:1070000021F2E9CF88E0C433A1F38BE0C83389F3E0
:10701000E2CF83E0EECF84E0C03359F386E0C133A2
:1070200041F3D9CF85E0C833B1F6E3CF87E0C2336F
:1070300091F6DFCF89E0C13371F6DBCF8AE0C03350
:1070400051F6D7CF8CE0C73331F6D3CF8DE0C633BE
:1070500011F6CFCFC03209F498CF8EE0C33549F294
:10706000BACF80ED8C0F8A3008F08FCF9FE09093DD
:1070700029048093280489CFCA3019F0CD3009F053
:1070800084CF1092290481CFCA3019F0CD3009F095
:107090007CCF80919D148823A1F3973089F038F438
:1070A000953079F71092440210929E0CEACF9A30F4
:1070B00059F09F3031F7809128040E941032E1CFBF
:1070C00081E080932406DDCF81E080932306D9CF31
:1070D0009091C00095FFFCCF8093C6000895CF9398
:1070E000DF93EC018991882319F00E946838FACF68
:1070F0008DE00E9468388AE0DF91CF910C94683867
:10710000CF92DF92EF92FF92CF936B017C01C42F5D
:107110004A3069F4F7FE0BC0F094E094D094C09428
:10712000C11CD11CE11CF11C8DE20E9468384C2F5F
:10713000C701B601CF91FF90EF90DF90CF900C94F4
:1071400048ADCF93DF93EC01FE0184912196882313
:1071500019F00E946838F8CFDF91CF910895CF934E
:10716000DF93D0918C1189E89CE10E94A1388AE0DC
:107170000E94683880910B0D873009F449C083E084
:107180008093060D81E08093860280E190E09093E9
:10719000401480933F1485E080933314C2E8C09379
:1071A000361484E190E1A0E0B0E08093371490932E
:1071B0003814A0933914B0933A1483EE93E10E94EB
:1071C000F13461E070E080E090E00E94FA2C81E010
:1071D0009AE59093401480933F1485E390E0909358
:1071E00042148093411487E080933314C093361483
:1071F00084E890E0A0E0B0E08093371490933814D6
:10720000A0933914B0933A1483EE93E10E94F134C1
:1072100080918C11813089F1823061F50E94E72BD9
:107220006093BE057093BF058093C0059093C10520
:1072300081E080938C110E9402AA6093BA0570933A
:10724000BB058093BC059093BD05D23089F0809139
:10725000A7069091A80601969093A8068093A7068A
:107260001092C6051092C7051092C8051092C90564
:1072700081E004C00E94192CDBCF80E0DF91CF9128
:107280000895CF93C82FCB010E94A1388DEF98E1CC
:107290000E94A1388EEE98E1CC2311F083EF98E1A3
:1072A0000E94A1388AE0CF910C946838CF93DF9385
:1072B00000D01F92CDB7DEB784EF91E0A0E0B0E040
:1072C00089839A83AB83BC83BE016F5F7F4F8CE35E
:1072D0000E94D3338BE199E10E94A1388CB165E122
:1072E00079E185FB882780F90E944139809103016B
:1072F0006FE079E1869581700E94413989B169E03A
:1073000079E183FB882780F90E9441398CB160E0E4
:1073100079E1829581700E9441394B9909C00E94A0
:107320000E340F900F900F900F90DF91CF91089532
:107330000E94F3330F900F900F900F90DF91CF9139
:10734000089580918C118130C1F589EC98E10E94FB
:10735000A1388AE00E94683881E09AE59093401451
:1073600080933F1487E590E09093421480934114FA
:1073700087E08093331482E88093361484E890E0A9
:10738000A0E0B0E08093371490933814A0933914A0
:10739000B0933A1483EE93E10E94F13482E080933B
:1073A0008C110E9402AA6093C2057093C30580935A
:1073B000C4059093C50581E0089580E008950F937A
:1073C0001F930E9402AA0091A2061091A306209189
:1073D000A4063091A506011511052105310509F016
:1073E00067C020911513222309F45FC0E0911313A5
:1073F00021502093151321E02E0F20931313309169
:107400001613231302C01092131324E0E29FF0011D
:107410001124E95EFC4E00811181228133810093A9
:107420009E0610939F062093A0063093A106600F3E
:10743000711F811D911D6093A2067093A306809316
:10744000A4069093A5068091A0069091A106892B91
:1074500061F11FB7F89488EB98E10E94A1388AE0A7
:107460000E94683884E096E09093401480933F1423
:1074700080EA90E8909342148093411487E08093CF
:10748000331482E88093361480EA90E0A0E0B0E004
:107490008093371490933814A0933914B0933A140E
:1074A00083EE93E10E94F1341FBF1F910F91089565
:1074B000601B710B820B930B97FDF7CF40981092D6
:1074C000A2061092A3061092A4061092A506EDCF74
:1074D0000F931F93CF93DF938C01EB0190911513C2
:1074E00020911613921305C00E94DF390E9410C527
:1074F000F5CF8091141334E0839FF0011124E95EED
:10750000FC4E11830083D383C2839F5F9093151336
:107510008F5F281739F080931413DF91CF911F915B
:107520000F91089510921413F8CFCF92DF92EF923B
:10753000FF921F93CF93DF93182F662351F0109281
:10754000FC041092F8041092F9041092FA041092BC
:10755000FB040E9402AA6B017C018091F8049091C7
:10756000F904A091FA04B091FB04A7019601281B2D
:10757000390B4A0B5B0BDA01C901B7FD3DC0209105
:10758000FC0417FD13C0412F012E000C550B4C5F5E
:107590005F4F822F022E000C990B4817590764F198
:1075A00084EF91E0A0E0B0E0211724F488EE93E0AE
:1075B000A0E0B0E08C0D9D1DAE1DBF1D8093F804B2
:1075C0009093F904A093FA04B093FB042170C22FA6
:1075D00030E0D32F84E28C9FB0018D9F700D7C1B17
:1075E000112460597C4F82E390E00E94683A8091B8
:1075F000FC048F5F8093FC04DF91CF911F91FF907B
:10760000EF90DF90CF900895CF93DF9300D01F923B
:10761000CDB7DEB78EE398E10E94A1388AE00E94E0
:10762000683880910B0D8330D9F119821A821B8240
:107630001C8260E0CE0101960E94342C19821A82CD
:107640001B821C8261E0CE0101960E94342C81E0F5
:10765000809385021092050D8093860281E09AE561
:107660009093401480933F1483E390E090934214EE
:107670008093411487E08093331482E8809336141A
:1076800084E890E0A0E0B0E0809337149093381441
:10769000A0933914B0933A1483EE93E10E94F1342D
:1076A0000F900F900F900F90DF91CF9108956F92F0
:1076B0007F928F929F92AF92BF92CF92DF92EF9282
:1076C000FF920F931F93CF93DF93CDB7DEB76497ED
:1076D0000FB6F894DEBF0FBECDBF1092D0008091E0
:1076E000D00082608093D0001092D50080E180931A
:1076F000D4008091D10080618093D1008091D1002D
:1077000088608093D1008091D10080688093D100FF
:107710008091D1008F7D8093D1008AE580933414CD
:107720008093E41385EA809335148093E513E3E8AE
:10773000F4E18AE1DF011D928A95E9F78091040D59
:10774000882309F474C283E090E0909340148093FE
:107750003F1485E08093331482E8809336148FE1E0
:1077600090E1A0E0B0E08093371490933814A09398
:107770003914B0933A1483EE93E10E94F13484E615
:1077800090E09093401480933F1405E000933314ED
:1077900012E81093361486E090E1A0E0B0E0809308
:1077A000371490933814A0933914B0933A1483EE9D
:1077B00093E10E94F1348BE090E090934014809329
:1077C0003F14009333141093361480E092E1A0E04C
:1077D000B0E08093371490933814A0933914B09389
:1077E0003A1483EE93E10E94F13410924014109207
:1077F0003F14009333141093361484E390E1A0E017
:10780000B0E08093371490933814A0933914B09358
:107810003A1483EE93E10E94F134109240141092D6
:107820003F1400933314109336148AE390E1A0E0E0
:10783000B0E08093371490933814A0933914B09328
:107840003A1483EE93E10E94F134809153129091A7
:1078500054129093401480933F1400933314109368
:10786000361486E390E1A0E0B0E080933714909363
:107870003814A0933914B0933A1483EE93E10E9424
:10788000F1348091E8119091E91190934014809324
:107890003F1400933314109336148CE390E1A0E06E
:1078A000B0E08093371490933814A0933914B093B8
:1078B0003A1483EE93E10E94F13482E090E09093D9
:1078C000401480933F1400933314109336148EE1C8
:1078D00090E1A0E0B0E08093371490933814A09327
:1078E0003914B0933A1483EE93E10E94F13481E0AD
:1078F0008093850270E6C72E70E1D72EE12CF12C23
:107900001092401410923F140093331410933614C5
:10791000C0923714D0923814E0923914F0923A148D
:1079200083EE93E10E94F134BFEFCB1ADB0AEB0A3E
:10793000FB0AE4E7CE16E0E1DE06E104F10401F71C
:10794000CE0101967C0184E1D7011D928A95E9F769
:1079500081E08F9390E99F938F9390E69F938F930D
:1079600088E68F9383EA93E09F938F93FF92EF9241
:107970000F94B53520E630E140E050E060EB73E075
:1079800083EE93E10E94C7E92AE630E140E050E04F
:107990006DEB73E083EE93E10E94C7E924E730E1E9
:1079A00040E050E0B70183EE93E10E94C7E92EE783
:1079B00030E140E050E06BEC73E083EE93E10E9435
:1079C000C7E91092401410923F140093331410939F
:1079D00036148EE090E1A0E0B0E0809337149093ED
:1079E0003814A0933914B0933A1483EE93E10E94B3
:1079F000F1341092401410923F14009333141093FA
:107A000036148FE090E1A0E0B0E0809337149093BB
:107A10003814A0933914B0933A1483EE93E10E9482
:107A2000F1340FB6F894DEBF0FBECDBF4AE0C42ECE
:107A300040E2D42EE12CF12C55E0752E62E8662E42
:107A4000460157010AE010E01092401410923F14D2
:107A500070923314609236148092371490923814D6
:107A6000A0923914B0923A1483EE93E10E94F1345B
:107A700001501109FFEF8F1A9F0AAF0ABF0A0115C3
:107A8000110511F78AE0C80ED11CE11CF11C92ED22
:107A9000C91690E2D906E104F10491F6C12C30E256
:107AA000D32EE12CF12C05E012E810924014109234
:107AB0003F140093331410933614C0923714D092AD
:107AC0003814E0923914F0923A1483EE93E10E9454
:107AD000F1341092401410923F1400933314109319
:107AE0003614D701C6018C529F4FAF4FBF4F8093C2
:107AF000371490933814A0933914B0933A1483EE4A
:107B000093E10E94F134AFEFCA1ADA0AEA0AFA0ADC
:107B1000BAE0CB16B0E2DB06E104F10431F62EED5B
:107B2000C22E20E2D22EE12CF12C05E012E81092B8
:107B3000401410923F140093331410933614C092E3
:107B40003714D0923814E0923914F0923A1483EE3C
:107B500093E10E94F134EFEFCE1ADE0AEE0AFE0A3C
:107B6000F6EECF16F0E2DF06E104F10401F7CC24D3
:107B7000C39482E1D82EE12CF12C9AE0A92EB12CED
:107B800005E012E8B0924014A0923F140093331421
:107B900010933614C0923714D0923814E0923914EE
:107BA000F0923A1483EE93E10E94F134B0924014C3
:107BB000A0923F140093331410933614D701C601DA
:107BC0008096A11DB11D8093371490933814A09313
:107BD0003914B0933A1483EE93E10E94F1348FEF9D
:107BE000C81AD80AE80AF80A95E1C91692E1D90636
:107BF000E104F10439F684EA97E10E94A1388AE0B1
:107C00000E94683864960FB6F894DEBF0FBECDBFF1
:107C1000DF91CF911F910F91FF90EF90DF90CF9068
:107C2000BF90AF909F908F907F906F90089582E06B
:107C300090E08BCD0E94573B1092960581E0809397
:107C4000860286E598E10E94A1388AE00C946838A3
:107C50000F931F93CF938C01C62F8EE294E10E9465
:107C6000A138C8010E94A1388AE30E94683880E3E5
:107C70008C0F0E9468388AE0CF911F910F910C946D
:107C8000683881EB95E10E94A13860E081EA95E1D6
:107C90000E94283E60E08CE895E10E94283E61E069
:107CA00085E895E10E94283E61E08AE795E10E941F
:107CB000283E61E08AE695E10E94283E60E081E688
:107CC00095E10E94283E61E087E595E10E94283E0B
:107CD00061E08DE495E10E94283E61E086E495E153
:107CE0000E94283E61E08EE395E10E94283E61E01B
:107CF00080E395E10E94283E61E082E295E10E94E6
:107D0000283E60E083E195E10E94283E60E085E046
:107D100095E10E94283E60E08FEE94E10E94283EAB
:107D200061E08EED94E10E94283E61E08FEC94E1E9
:107D30000E94283E61E088EC94E10E94283E60E0C9
:107D400081EC94E10E94283E61E088EB94E10E947E
:107D5000283E61E083EA94E10E94283E61E085E9E3
:107D600094E10E94283E61E082E894E10E94283E6E
:107D700060E085E794E10E94283E61E080E794E1BD
:107D80000E94283E61E083E694E10E94283E60E084
:107D90008FE494E10E94283E60E08CE394E10E942D
:107DA000283E60E08CEA94E10E94BA1D682F617061
:107DB00083E394E10C94283E80914705827149F455
:107DC000809149058C7829F480914A05837009F4E3
:107DD00075C082E40E94981E882351F00E94662498
:107DE0006093B10C7093B20C8093B30C9093B40C6D
:107DF00083E50E94981E882351F00E94EC24609332
:107E0000E10C7093E20C8093E30C9093E40C84E516
:107E10000E94981E882351F00E94EC246093E50C88
:107E20007093E60C8093E70C9093E80C88E50E9431
:107E3000981E882351F00E94EC2460930C097093E3
:107E40000D0980930E0990930F0989E50E94981EF1
:107E5000882351F00E94EC2460931009709311095B
:107E600080931209909313098AE50E94981E882333
:107E7000B1F00E94EC24609314097093150980936B
:107E80001609909317092DEC3CEC4CEC5DE30F9434
:107E90005D2B181624F088E99EE00E94A13885E445
:107EA0000E94981E882351F00E94EC2460931809C8
:107EB0007093190980931A0990931B090895AF9242
:107EC000BF92CF92DF92EF920F931F93CF93DF93E6
:107ED0005B01EA016901882309F463C081E99EE03E
:107EE0000E94A138F501608171818281938146E011
:107EF0000E9450BDE1100BC088E89EE00E94A138AE
:107F0000688179818A819B8146E00E9450BD81E829
:107F10009EE00E94A138F601608171818281938187
:107F200043E00E9450BD8AE79EE00E94A138F8011C
:107F3000608171818281938143E00E9450BD81E71D
:107F40009EE00E94A138F601208131814281538157
:107F5000F80160817181828193810F942C3243E01A
:107F60000E9450BDEE20F9F08AE00E9468388CE54E
:107F70009EE00E94A138688179818A819B8146E0D8
:107F80000E9450BD8AE00E9468388AE0DF91CF915C
:107F90001F910F91EF90DF90CF90BF90AF900C9416
:107FA0006838E110E4CFDF91CF911F910F91EF90EE
:107FB000DF90CF90BF90AF9008950F931F93CF9312
:107FC0008C01C62F89E798E00E94A138C8010E9461
:107FD000A138CC2331F08AE0CF911F910F910C94FE
:107FE0006838CF911F910F9108950E94D7ED10929C
:107FF0009E0C109244020E942E32882351F08091F0
:10800000A91482FD06C084EB98E19093EE0C809356
:10801000ED0C61E08DEA98E10E94DD3F0C94AF38F1
:108020000F931F93CF93DF938C016F3F19F410923E
:10803000CD1160E02091CD11862F062E000C990BFA
:108040002817190609F08CF56093CD1160E087E7D9
:1080500098E10E94DD3FC8010E94A1388AE00E9499
:108060006838C8010F94AA2A800F911FEC01C01B29
:10807000D10BC034D1053CF00197FC012491207C48
:108080002038D1F3F3CFDD27AE01B8018DE891E1BF
:108090000F94CB2AC357DE4E18828DE891E1DF9111
:1080A000CF911F910F910C94BB35DF91CF911F9110
:1080B0000F91089510929E0C109244028091A91481
:1080C00080648093A91461E085E898E10E94DD3F17
:1080D0004AE958E162EA78E185E00E94E5EB60E078
:1080E0008CE898E10C9410400F931F93CF938C0170
:1080F000C62F60E083E898E00E94DD3FC8010E943F
:10810000A138CC2331F08AE0CF911F910F910C94CC
:108110006838CF911F910F91089561E08BE898E046
:108120000C947440EF92FF920F931F93CF937C01B6
:108130008B01C42F60E083E898E00E94DD3FC70117
:108140000E94A13880E20E946838C8010E94A138CC
:10815000CC2319F08C2F0E9468388AE0CF911F91B0
:108160000F91FF90EF900C946838DF92EF92FF929E
:108170000F931F93CF93DF93D82E7B018A01E901E0
:108180000E948D40D092F91140E0B70184E799E058
:108190000E9492400115110531F040E0B8018DE6D2
:1081A00099E00E949240209731F040E0BE018DE6B8
:1081B00099E00E94924061E088E699E0DF91CF91DA
:1081C0001F910F91FF90EF90DF900C947440AF924D
:1081D000BF92CF92DF92EF92FF920F931F93CF93B4
:1081E000DF9386EE97E00E94A138C0E0D7E0D1503F
:1081F00021F080E20E946838FACF8C2F0E941EEA9C
:10820000CF5FC53099F78AE00E9468380BEA17E023
:10821000C0E080E20E9468388C2F0E941EEA58015C
:10822000D5E080E20E946838F501C080D180E2800C
:10823000F380A7019601C701B6010F941F3588236B
:1082400069F180E20E9468388DE30E9468388DE30E
:108250000E9468388DE30E9468388DE30E94683878
:108260008DE30E946838D150F4E1AF0EB11CD111FA
:10827000D8CF8AE00E946838CF5F0C5F1F4FC530AF
:1082800041F68AE0DF91CF911F910F91FF90EF901F
:10829000DF90CF90BF90AF900C94683820E030E032
:1082A000A901C701B6010F948D3487FD03C08BE28D
:1082B0000E94683843E0C701B6010E9450BDD3CF89
:1082C000811107C08AEC9EE00E94A1388AE00C94DC
:1082D00068388EEC9EE0F8CFCF93DF93EB010E94DD
:1082E000A138CE01DF91CF910C94DCEACF93C62F59
:1082F0000E94A1388C2FCF910C941EEACF92DF926E
:10830000EF92FF926A017B010E94A13842E0C7010F
:10831000B601FF90EF90DF90CF900C9450BDCF92BC
:10832000DF92EF92FF926A017B010E94A1384AE03E
:10833000C701B601FF90EF90DF90CF900C9480388A
:10834000CF93DF93EB010E94A138CE01DF91CF9153
:108350000C9425EA4F925F926F927F928F929F9238
:10836000AF92BF92CF92DF92EF92FF920F931F9343
:10837000CF93DF9300D000D01F921F92CDB7DEB70E
:108380008091950581110AC480919305909194057F
:108390009C012F5F3F4F30939405209393058E3EB1
:1083A000924008F4FBC38091531290915412909321
:1083B000401480933F1405E00093331412E81093A7
:1083C000361486E390E1A0E0B0E0809337149093F8
:1083D0003814A0933914B0933A1483EE93E10E94B9
:1083E000F1348091E8119091E911909340148093B9
:1083F0003F1400933314109336148CE390E1A0E003
:10840000B0E08093371490933814A0933914B0934C
:108410003A1483EE93E10E94F134809155129091C9
:1084200056129093401480933F140093331410938A
:10843000361484E390E1A0E0B0E080933714909389
:108440003814A0933914B0933A1483EE93E10E9448
:10845000F1348091EA119091EB1190934014809344
:108460003F1400933314109336148AE390E1A0E094
:10847000B0E08093371490933814A0933914B093DC
:108480003A1483EE93E10E94F13481E080939505E4
:10849000109294051092930580910B0D882339F169
:1084A0000E944C1D811123C0809192058F5F8093A3
:1084B000920580919205853620F0109292051092D7
:1084C0000B0DE0910B0DE150E73008F06AC00E2E65
:1084D000000CFF0B8827E059FD4B8F4F0D94243281
:1084E0007A42C9429544C14402453A45CD42109270
:1084F0009205DFCF0E94F22C882309F452C081E05C
:108500008093860280E398E10E94A1388AE00E946D
:10851000683880E190E09093401480933F1485E0A8
:108520008093331412E81093361484E190E1A0E0B4
:10853000B0E08093371490933814A0933914B0931B
:108540003A1483EE93E10E94F13481E09AE590932E
:10855000401480933F1486E390E0909342148093FC
:10856000411487E0809333141093361484E890E02C
:10857000A0E0B0E08093371490933814A09339149E
:10858000B0933A1483EE93E10E94F13410920B0DF4
:1085900008C00E94F22C882321F00E944C1D8823E1
:1085A000A9F380918602882309F433C78091960548
:1085B0008111C0C284E096E09093401480933F14F0
:1085C00080EA90E8909342148093411417E010934E
:1085D000331402E80093361480EA90E0A0E0B0E0A3
:1085E0008093371490933814A0933914B0933A14AD
:1085F00083EE93E10E94F134809181029091820296
:10860000A0918302B09184020097A105B10509F001
:108610003FC21092401410923F1415E0109333148F
:10862000009336148AE890E1A0E0B0E0809337141C
:1086300090933814A0933914B0933A1483EE93E1D5
:108640000E94F13489E090E09093401480933F14AD
:1086500010933314009336148CE890E1A0E0B0E05E
:108660008093371490933814A0933914B0933A142C
:1086700083EE93E10E94F134809181029091820215
:10868000A0918302B09184020097F1E0AF07B10599
:1086900008F441C2B0934014A0933F149093421445
:1086A0008093411487E08093331482E880933614DA
:1086B00088E890E1A0E0B0E08093371490933814FC
:1086C000A0933914B0933A1483EE93E10E94F134ED
:1086D0008091810290918202A0918302B0918402E4
:1086E000BA2FA92F982F8827009721E0A207B1055C
:1086F00008F417C2B0934014A0933F14909342140F
:108700008093411487E08093331412E81093361459
:1087100081EA90E0A0E0B0E08093371490933814A1
:10872000A0933914B0933A1483EE93E10E94F1348C
:108730008091A00C882309F4FAC183E090E0909323
:10874000401480933F1485E08093331410933614C3
:1087500085E490E1A0E0B0E0809337149093381462
:10876000A0933914B0933A1483EE93E10E94F1344C
:1087700080919605875E8093960520919605822FBD
:1087800090E0253608F021C29093401480933F1466
:1087900085E08093331482E88093361480E090E182
:1087A000A0E0B0E08093371490933814A09339146C
:1087B000B0933A1483EE93E10E94F1340E944C1D71
:1087C000811114C20E942E32811105C09091990529
:1087D00091FD0E944C1D9091990580FB91F9909319
:1087E000990591FD03C28091A91482FDFFC180917A
:1087F0008C118150823008F4F9C16091EA117091B6
:10880000EB11072E000C880B990B0F94642B6B0156
:108810007C0120E030E0A9010F945D2B882309F44E
:10882000BBC66091E8117091E911072E000C880B0E
:10883000990B0F94642B2B013C0120E030E040E0C9
:1088400050E4C701B6010F942C32A30192010F949A
:108850008D3418160CF4C2C66091531270915412E4
:10886000072E000C880B990B0F94642B6D837E836D
:108870008F8398876091551270915612072E000CC5
:10888000880B990B0F94642B4B015C0120E030E0C6
:1088900040E251E40F942C322D813E814F81588566
:1088A0000F948D3418160CF499C620E030E040E0A7
:1088B00050E4C701B6010F942D32A30192010F9429
:1088C0005D2B87FD10C020E030E040E251E4C5019F
:1088D000B4010F942D322D813E814F8158850F9424
:1088E0005D2B87FF6AC684E190E0909340148093EB
:1088F0003F1485E08093331482E88093361484E13A
:1089000090E1A0E0B0E08093371490933814A093E6
:108910003914B0933A1483EE93E10E94F1348091BC
:10892000060D81117CC682E07AC682E298E10E943F
:10893000A1388AE00E94683881E09AE5909340145B
:1089400080933F1480E490E090934214809341140C
:1089500017E01093331482E88093361484E890E093
:10896000A0E0B0E08093371490933814A0933914AA
:10897000B0933A1483EE93E10E94F13410930B0DFF
:1089800010CE8091F50C882309F40BCE0E94F22CB6
:10899000882309F406CE0E944C1D811102CE84E189
:1089A00098E10E94A1388AE00E9468388091F60C14
:1089B00090E0B0E0A0E0895B9F4FAE4FB54A21E068
:1089C0003AE53093401420933F14909342148093DF
:1089D000411487E08093331482E88093361484E84E
:1089E00090E0A0E0B0E08093371490933814A09307
:1089F0003914B0933A1483EE93E10E94F13410924B
:108A0000F50CC4CD0E94F22C882309F4CACD0E9433
:108A10004C1D8111C6CD81E08093860210920B0D12
:108A200086E098E10E94A1388AE00E94683881E0DF
:108A30009AE59093401480933F148EE490E09093D5
:108A400042148093411487E08093331482E880932A
:108A5000361484E890E0A0E0B0E08093371490935F
:108A60003814A0933914B0933A1483EE93E10E9422
:108A7000F13497CD0E944C1D811193CD19821A8239
:108A80001B821C8262E0CE0101960F94CA007ECD4B
:108A90000196A11DB11D35E0B695A79597958795CF
:108AA0003A95D1F70197A109B1090097E1E0AE0726
:108AB000B10548F1B0934014A0933F149093421431
:108AC000809341141093331412E8109336148AE8FB
:108AD00090E1A0E0B0E08093371490933814A09315
:108AE0003914B0933A1483EE93E10E94F13488E094
:108AF00090E09093401480933F1485E0809333146A
:108B000010933614A9CD9093401480933F1485E0C0
:108B100080933314D9CF9093401480933F1485E011
:108B2000C2CD9093401480933F1485E0ECCD82E059
:108B300090E005CE8A3F08F020CE8EEF8093960518
:108B400085EF97E10E94A1388AE00E94683881E0B1
:108B50008093860281E09AE59093401480933F14BD
:108B60008DE290E0909342148093411487E08093CB
:108B7000331482E88093361484E890E0A0E0B0E0FB
:108B80008093371490933814A0933914B0933A1407
:108B900083EE93E10E94F1341092950528960FB66A
:108BA000F894DEBF0FBECDBFDF91CF911F910F9123
:108BB000FF90EF90DF90CF90BF90AF909F908F90FD
:108BC0007F906F905F904F90089584569109909395
:108BD000401480933F1485E08093331482E880939F
:108BE000361481E090E1A0E0B0E0DCCD8CE090E0D4
:108BF0009093401480933F1415E01093331482E84F
:108C00008093361484E190E1A0E0B0E080933714C3
:108C100090933814A0933914B0933A1483EE93E1EF
:108C20000E94F1340E94E72B20E13EE040E050E05A
:108C30000F94A1312115310581E04807510508F451
:108C400070C05093401440933F14309342142093CB
:108C5000411487E08093331412E81093361480E1B6
:108C600090E1A0E0B0E08093371490933814A09383
:108C70003914B0933A1483EE93E10E94F1340E94C8
:108C8000E72B20E13EE040E050E00F94A1312CE3DF
:108C900030E040E050E00F94A13130934014209335
:108CA0003F1405E0009333141093361482E190E1F1
:108CB000A0E0B0E08093371490933814A093391457
:108CC000B0933A1483EE93E10E94F1340E943C3257
:108CD000882309F45CC48F5F80939105E82EF12C02
:108CE000833330F5EE0CFF1CF0924014E0923F14F9
:108CF00000933314109336148EE090E1A0E0B0E0BE
:108D00008093371490933814A0933914B0933A1485
:108D100083EE93E10E94F1341092401410923F14BC
:108D20002BC03093401420933F141093331494CFEE
:108D300084E690E09093401480933F1400933314A2
:108D4000109336148EE090E1A0E0B0E080933714E9
:108D500090933814A0933914B0933A1483EE93E1AE
:108D60000E94F134A2E3EA1AA0E8FA0AEE0CFF1C12
:108D7000F0924014E0923F14009333141093361491
:108D80008FE090E1A0E0B0E0809337149093381426
:108D9000A0933914B0933A1483EE93E10E94F13416
:108DA0000E943C3290E09093401480933F1485E001
:108DB0008093331482E88093361486E190E1A0E03A
:108DC000B0E08093371490933814A0933914B09383
:108DD0003A1483EE93E10E94F13420E030E0A901DF
:108DE0006091E8127091E9128091EA129091EB1271
:108DF0000F942D3220E030E048EC52E40F94C32B66
:108E00000F9499337093401460933F1405E00093DE
:108E1000331412E81093361486E290E1A0E0B0E03B
:108E20008093371490933814A0933914B0933A1464
:108E300083EE93E10E94F13480917D0290917E0255
:108E40009093401480933F1400933314109336147E
:108E500080E093E1A0E0B0E0809337149093381461
:108E6000A0933914B0933A1483EE93E10E94F13445
:108E700020E030E040E251E46091B50C7091B60C16
:108E80008091B70C9091B80C0F94C32B0F94A03322
:108E90007093401460933F1400933314109336146E
:108EA00082E492E1A0E0B0E080933714909338140C
:108EB000A0933914B0933A1483EE93E10E94F134F5
:108EC00020E030E040E251E46091B90C7091BA0CBE
:108ED0008091BB0C9091BC0C0F94C32B0F94A033CA
:108EE0007093401460933F1400933314109336141E
:108EF00086E492E1A0E0B0E08093371490933814B8
:108F0000A0933914B0933A1483EE93E10E94F134A4
:108F100020E030E040E251E46091BD0C7091BE0C65
:108F20008091BF0C9091C00C0F94C32B0F94A03371
:108F30007093401460933F140093331410933614CD
:108F40008AE492E1A0E0B0E0809337149093381463
:108F5000A0933914B0933A1483EE93E10E94F13454
:108F600020E030E040E251E46091C10C7091C20C0D
:108F70008091C30C9091C40C0F94C32B0F94A03319
:108F80007093401460933F1400933314109336147D
:108F90008EE492E1A0E0B0E080933714909338140F
:108FA000A0933914B0933A1483EE93E10E94F13404
:108FB00020E030E048EC52E46091E0127091E11260
:108FC0008091E2129091E3120F94C32B0F94993386
:108FD0007093401460933F1400933314109336142D
:108FE00086E392E1A0E0B0E08093371490933814C8
:108FF000A0933914B0933A1483EE93E10E94F134B4
:1090000020E030E048EC52E46091E4127091E51207
:109010008091E6129091E7120F94C32B0F9499332D
:109020007093401460933F140093331410933614DC
:109030008AE392E1A0E0B0E0809337149093381473
:10904000A0933914B0933A1483EE93E10E94F13463
:1090500080918D0290918E029093401480933F14E2
:10906000009333141093361482E592E1A0E0B0E04F
:109070008093371490933814A0933914B0933A1412
:1090800083EE93E10E94F13480918B0290918C02E7
:109090009093401480933F1400933314109336142C
:1090A00084E592E1A0E0B0E0809337149093381407
:1090B000A0933914B0933A1483EE93E10E94F134F3
:1090C00020E030E040E251E4609158127091591272
:1090D00080915A1290915B120F94C32B0F94A0337E
:1090E0007093401460933F1400933314109336141C
:1090F00086E592E1A0E0B0E08093371490933814B5
:10910000A0933914B0933A1483EE93E10E94F134A2
:109110002CEA35EC47E25EE360915C1270915D12DF
:1091200080915E1290915F120F94273320E030E01F
:1091300040E251E40F94C32B0F94A033709340147A
:1091400060933F1400933314109336148AE592E130
:10915000A0E0B0E08093371490933814A0933914B2
:10916000B0933A1483EE93E10E94F1342CEA35EC8B
:1091700047E25EE360916012709161128091621229
:10918000909163120F94C32B20E030E040E251E451
:109190000F94C32B0F94A0337093401460933F142B
:1091A00000933314109336148EE592E1A0E0B0E002
:1091B0008093371490933814A0933914B0933A14D1
:1091C00083EE93E10E94F13420E030E040E251E48C
:1091D0006091ED117091EE118091EF119091F0116D
:1091E0000F94C32B0F94A0337093401460933F14DB
:1091F000009333141093361482E692E1A0E0B0E0BD
:109200008093371490933814A0933914B0933A1480
:1092100083EE93E10E94F1342CEA35EC47E25EE301
:109220006091F1117091F2118091F3119091F4110C
:109230000F94273320E030E040E251E40F94C32B39
:109240000F94A0337093401460933F140093331431
:109250001093361486E692E1A0E0B0E080933714D4
:1092600090933814A0933914B0933A1483EE93E199
:109270000E94F1342CEA35EC47E25EE36091F5118F
:109280007091F6118091F7119091F8110F94C32B02
:1092900020E030E040E251E40F94C32B0F94A03360
:1092A0007093401460933F1400933314109336145A
:1092B0008AE692E1A0E0B0E08093371490933814EE
:1092C000A0933914B0933A1483EE93E10E94F134E1
:1092D0008091FF0C811105C08091010D882309F454
:1092E0006DC06091531270915412072E000C880BC0
:1092F000990B0F94642B20E030E048EC52E40F947B
:10930000C32B6B017C016091551270915612072E90
:10931000000C880B990B0F94642B9B01AC01C701C7
:10932000B6010F9427330F94A0336536710510F002
:1093300064E670E07093401460933F1405E000937E
:10934000331412E81093361484E290E1A0E0B0E008
:109350008093371490933814A0933914B0933A142F
:1093600083EE93E10E94F134609153127091541294
:10937000072E000C880B990B0F94642B6B017C015A
:1093800020E030E04AE253E40F948D34181624F4C0
:109390008091FF0C811146C1609155127091561257
:1093A000072E000C880B990B0F94642B9B01AC01CA
:1093B000C701B6010F948D3487FFAFC18091F50CC2
:1093C000882339F18091F40C91E0980F9093F40C7C
:1093D00090E09093401480933F1485E08093331481
:1093E00082E88093361482E490E1A0E0B0E08093BC
:1093F000371490933814A0933914B0933A1483EE31
:1094000093E10E94F1348091F40C8A3010F01092B4
:10941000F40C0E947D2C882309F4B5C16091090DDC
:1094200070910A0DEE24E394F12C61157105A9F0F9
:1094300090E080E00F94622B20E030E040E85EE3B3
:109440000F94C32B0F940B3320E030E040E85FE330
:109450000F942D320F94A0337B0101E010E0809136
:10946000EF0C811102C010E000E080912713909171
:1094700028138F3F980711F40E94A5B690932813E4
:1094800080932713080F191FB80190E080E00F9414
:10949000622B20E030E040E85EE30F94C32B0F9492
:1094A0000B334B015C01F0924014E0923F1405E055
:1094B0000093331412E81093361480E193E1A0E096
:1094C000B0E08093371490933814A0933914B0937C
:1094D0003A1483EE93E10E94F134C501B4010F9474
:1094E000A0337093401460933F140093331410938F
:1094F000361482E193E1A0E0B0E0809337149093BA
:109500003814A0933914B0933A1483EE93E10E9477
:10951000F13403E814E1AAE1FA2E80914D0590910F
:109520004E0520918F0530919005891B8F7309F4AA
:1095300049C12A3131050CF0DBC190914D05809174
:109540004E054FEF5FEF981749F0E82FF0E0E35B2F
:10955000FA4F42818F5F8F7380934E05F901ED576B
:10956000FB4E4083809183148A3509F0B3C162E0D9
:1095700070E080E090E00E94FA2C80918F0590913D
:10958000900501969093900580938F05C6CF109219
:10959000401410923F14ACCB60915512709156124A
:1095A000072E000C880B990B0F94642B20E030E001
:1095B000A9010F945D2B811134C98CE090E0909348
:1095C000401480933F1485E08093331482E88093A5
:1095D000361484E190E1A0E0B0E0F3CB8DE090E0C0
:1095E0009093401480933F1485E08093331482E875
:1095F0008093361484E190E1A0E0B0E080933714CA
:1096000090933814A0933914B0933A1483EE93E1F5
:109610000E94F1348091060D811101C081E0809398
:10962000060DDBCB1092FF0C20E030E040E251E46D
:109630006091F70C7091F80C8091F90C9091FA0CF4
:109640000F94C32B0F9499337093401460933F147D
:10965000009333141093361484E590E1A0E0B0E059
:109660008093371490933814A0933914B0933A141C
:1096700083EE93E10E94F13420E030E040E251E4D7
:109680006091FB0C7091FC0C8091FD0C9091FE0C94
:109690000F94C32B0F9499337093401460933F142D
:1096A000009333141093361488E590E1A0E0B0E005
:1096B0008093371490933814A0933914B0933A14CC
:1096C00083EE93E10E94F13484ED97E10E94A1388A
:1096D0008AE00E94683881E09AE590934014809374
:1096E0003F1481E490E0909342148093411487E00A
:1096F000809333141093361484E890E0A0E0B0E037
:109700008093371490933814A0933914B0933A147B
:1097100083EE93E10E94F13451CE6091010D6623F6
:1097200009F44CCE062E000C770B8BEB97E10E94D0
:10973000A0418AE00E9468381092010D84E090E018
:109740009093401480933F1485E08093331412E883
:10975000109336148EE890E1A0E0B0E080933714C7
:1097600090933814A0933914B0933A1483EE93E194
:109770000E94F13481E09AE59093401480933F1465
:1097800083E590E0B0CF1092401410923F1405E0B2
:109790000093331412E81093361480E193E1A0E0B3
:1097A000B0E08093371490933814A0933914B09399
:1097B0003A1483EE93E10E94F13410924014109217
:1097C0003F1493CE121613060CF492C08091E71347
:1097D0009091E813A091E913B091EA138C34E0E181
:1097E0009E07A105B10509F4D7C98A349041A105A6
:1097F000B10509F4D1C920E030E040E251E46091C4
:10980000690270916A0280916B0290916C020F94D0
:10981000C32B0F9499337093401460933F1405E069
:109820000093331412E81093361488E490E1A0E01A
:10983000B0E08093371490933814A0933914B09308
:109840003A1483EE93E10E94F13420E030E040E2EC
:1098500051E460916D0270916E0280916F0290915F
:1098600070020F94C32B0F9499337093401460933C
:109870003F1400933314109336148AE490E1A0E06F
:10988000B0E08093371490933814A0933914B093B8
:109890003A1483EE93E10E94F13420E030E040E29C
:1098A00051E4609171027091720280917302909103
:1098B00074020F94C32B0F949933709340146093E8
:1098C0003F1400933314109336148CE490E1A0E01D
:1098D000B0E056C9121613060CF01FCEF8012F2D5A
:1098E00011922A95E9F71092900510928F0515CEE6
:1098F0009091E41380918314981321C09091E51303
:109900008091841498131BC023303105C4F09091CA
:1099100085149093E313809186148093E61393301B
:10992000D1F4982F9D7F9038B1F4909187149F3493
:1099300009F059C0909188149B3409F054C0E3E8B1
:10994000F4E18AE1DF011D928A95E9F71092900512
:1099500010928F053BCF833809F045C08091871462
:1099600090918814982789279827B0E0A0E08093E9
:10997000E7139093E813A093E913B093EA13C09010
:109980008914D12CF12CE12CC092EB13D092EC1362
:10999000E092ED13F092EE132AE834E140E050E05B
:1099A000BA014C155D056E057F0508F04AC0DB0164
:1099B000CA01B695A795979587950696880F991F22
:1099C000FC01ED51FC4ED9018C9111969C91892797
:1099D00098278927918380834E5F5F4F6F4F7F4F1A
:1099E0002E5F3F4FDECF813861F58091871490E084
:1099F000B0E0A0E08093E7139093E813A093E913FD
:109A0000B093EA1380918814482F50E070E060E032
:109A10004093EB135093EC136093ED137093EE139C
:109A2000A9E8B4E1EFEEF3E190E030E020E0821746
:109A3000930739F04D9150E0419351932F5F3F4F81
:109A4000F6CFE3E8F4E18AE1DF011D928A95E9F7B8
:109A50001092900510928F050F946C01B7CE3F9233
:109A60004F925F926F927F928F929F92AF92BF922E
:109A7000CF92DF92EF92FF920F931F93CF93DF93DA
:109A80008091490587FD38C080914A058370A1F512
:109A9000C091EC12D091ED12488159816A817B818D
:109AA00085E297E10E947E414C815D816E817F81DC
:109AB00081EB9FE20E947E414091E8125091E912B1
:109AC0006091EA127091EB128EEA9FE20E947E4151
:109AD0008AE0DF91CF911F910F91FF90EF90DF907F
:109AE000CF90BF90AF909F908F907F906F905F903E
:109AF0004F903F900C9468386090E0127090E112A3
:109B00008090E2129090E312A090E412B090E512DF
:109B10000091E6121091E712C090E812D090E9127D
:109B2000E090EA12F090EB1288E50E94E61EC82F42
:109B3000882309F49AC00E94EC24362E472E582E12
:109B4000D92F20E030E040EB53EC0F948D3487FDAB
:109B50000DC020E030E040EB53E4632D742D852DE3
:109B60009D2F0F945D2B18160CF081C060E671E0FC
:109B700082E197E10E94A04160E671E08DE097E10B
:109B80000E94A0418AE097E10E94A138C0E089E5E7
:109B90000E94E61E882361F10E94EC24362E472E97
:109BA000582ED92F20E030E044EB53EC0F948D3445
:109BB00087FD0DC020E030E044EB53E4632D742DAD
:109BC000852D9D2F0F945D2B18160CF055C068E65F
:109BD00071E087EF96E10E94A04168E671E082EFB4
:109BE00096E10E94A0418FEE96E10E94A138C0E06C
:109BF0008AE50E94E61E882309F443C00E94EC24F3
:109C00006B017C0120E030E040E151EC0F948D3499
:109C100087FD0AC020E030E040E151E4C701B60111
:109C20000F945D2B18166CF567EF7FEF8DED96E1C5
:109C30000E94A04169E070E088ED96E10E94A04199
:109C400085ED96E1DF91CF911F910F91FF90EF90FD
:109C5000DF90CF90BF90AF909F908F907F906F904C
:109C60005F904F903F900C94A138C1E090CF632C4F
:109C7000742C852C9D2E8BCFA32CB42C052D1D2F41
:109C8000B7CFCC23E1F0C301D4018093E0129093CD
:109C9000E112A093E212B093E312C501D8018093C0
:109CA000E4129093E512A093E612B093E712C092EB
:109CB000E812D092E912E092EA12F092EB12DF91F0
:109CC000CF911F910F91FF90EF90DF90CF90BF90B9
:109CD000AF909F908F907F906F905F904F903F904C
:109CE00008958FED97E00C94A13889ED97E00C94DE
:109CF000A13884E690E09093D7058093D605109222
:109D0000F7051092F6050C9474E4EF92FF920F930E
:109D10001F93CF93DF93CDB7DEB762970FB6F8945A
:109D2000DEBF0FBECDBF0E94672A882309F43FC063
:109D30004AEF53E082FF02C04EED53E02AEF33E0DA
:109D400081FF02C020EE33E080FD2EC08AEF93E059
:109D50005F934F933F932F939F938F938FE699E158
:109D60009F938F938E010F5F1F4F1F930F930F943D
:109D7000F42A0E94754EC8010E946F38C8010E94E3
:109D80009FED0FB6F894DEBF0FBECDBF81E06296A7
:109D90000FB6F894DEBF0FBECDBFDF91CF911F91FC
:109DA0000F91FF90EF90089582EE93E0D1CF80E085
:109DB000EECFCF92DF92EF92FF928AE50E94E61EED
:109DC000882309F45AC00E94EC2420E030E040E0EF
:109DD00050EC0F945D2BC12CD12CE12C90ECF92E82
:109DE00087FD0FC00E94EC2420E030E040E050E40A
:109DF0000F948D3418160CF462C00E94EC246B0191
:109E00007C012091BD0C3091BE0C4091BF0C509153
:109E1000C00CC701B6010F94C32B0F949933CB012B
:109E20000E9428ED80E50E94981E81114EC0A70176
:109E300096016091E8127091E9128091EA12909176
:109E4000EB120F942D326093E8127093E912809315
:109E5000EA129093EB120E94754E4091E8125091D5
:109E6000E9126091EA127091EB1286EC96E10E9481
:109E70007E418AE00E94683805C083E50E94E61EA4
:109E80008111A1CF8091490587FD24C080914A05A9
:109E9000837001F50E94754E4091E8125091E912CD
:109EA0006091EA127091EB1287EB96E10E947E417D
:109EB0008AE0FF90EF90DF90CF900C946838C12C2F
:109EC000D12CE12C80E4F82E9CCF0E94B424811187
:109ED000AECFD8CF82E50E94981E8111DBCFFF90D4
:109EE000EF90DF90CF900895CF9384E50E94E61E17
:109EF000C0E08823D9F00E949424C82F1816B4F427
:109F00000E94754E8DE40E946838809144059091BE
:109F100045050E94DCEA6C2FCC0F770B88EA9FE0A6
:109F20000E94A0418AE00E946838CFEF8C2FCF9129
:109F300008954F925F926F927F928F929F92AF920D
:109F4000BF92CF92DF92EF92FF92CF93DF93CDB784
:109F5000DEB72C970FB6F894DEBF0FBECDBF409092
:109F6000EB085090EC086090ED087090EE0820919E
:109F70004F02309150024091510250915202C30160
:109F8000B2010F942D3269837A838B839C838090F6
:109F9000EF089090F008A090F108B090F20820919E
:109FA0005302309154024091550250915602C5011E
:109FB000B4010F942D326D837E838F839887C09078
:109FC000F308D090F408E090F508F090F60820919E
:109FD0005702309158024091590250915A02C701DC
:109FE000B6010F942D3269877A878B879C872091E1
:109FF0005B0230915C0240915D0250915E02C301B0
:10A00000B2010F942D322B013C0120915F0230915F
:10A0100060024091610250916202C501B4010F9447
:10A020002D324B015C01209163023091640240911A
:10A03000650250916602C701B6010F942D326B0183
:10A040007C010E94754E83EE9EE00E94A13883E55C
:10A050000E94981E882321F00E94B42480934D0210
:10A0600080914D02811151C08AEC9EE00E94A1387E
:10A070008BED9EE00E94A13849815A816B817C81E1
:10A0800086E59EE10E947E414D815E816F817885EB
:10A0900081EB9FE20E947E4149855A856B857C85D4
:10A0A0008EEA9FE20E947E4189ED9EE00E94A138E7
:10A0B00081ED9EE00E94A138B301A20186E59EE1F8
:10A0C0000E947E41B501A40181EB9FE20E947E4186
:10A0D000B701A6018EEA9FE20E947E418AE02C969B
:10A0E0000FB6F894DEBF0FBECDBFDF91CF91FF90CA
:10A0F000EF90DF90CF90BF90AF909F908F907F9028
:10A100006F905F904F900C9468388EEC9EE0AECFCD
:10A110005F926F927F928F929F92AF92BF92CF92F7
:10A12000DF92EF92FF920F931F93CF93DF931F92D3
:10A13000CDB7DEB77C0139018B015B01A40EB51EE2
:10A14000D12CC12CA016B10609F450C0F7018080B3
:10A150009180F80151908F015982C4010F947B3195
:10A160005816B9F1652DC4010F948331FFEFCF1A52
:10A17000DF0AC6018F779927892B21F162E070E011
:10A1800080E090E00E94CFA9C4010F947B319981B7
:10A190008917F9F00E94754E8FE694E00E94A1386D
:10A1A00081E00F90DF91CF911F910F91FF90EF9081
:10A1B000DF90CF90BF90AF909F908F907F906F90E7
:10A1C0005F90089562E070E080E090E00E945A267F
:10A1D000DBCFBE016F5F7F4FC3010E947FE9F701B4
:10A1E00080819181019691838083ACCF80E0D9CF2B
:10A1F000DF92EF92FF920F931F93CF93DF93CDB730
:10A20000DEB7CA5AD1090FB6F894DEBF0FBECDBF74
:10A21000CF55DF4F188219821A821B82C15AD04053
:10A220008091E4039091E503A091E603B091E703E8
:10A23000CB55DF4F88839983AA83BB83C55AD0400F
:10A2400084E690E09093D7058093D6051092F705A9
:10A250001092F6051092F80526EF35E044E050E044
:10A26000BE016B557F4F86ED95E00E94885080912E
:10A27000D6059091D70502969093D7058093D60581
:10A280001092F7051092F60581E0C655DF4F8883DE
:10A29000CA5AD040CE0186559F4F0E949BDA26EFC6
:10A2A00035E048E450E061EA7CE086ED95E00E940C
:10A2B000885026EF35E040E150E06CE079E086ED33
:10A2C00095E00E9488508AE097EDA3EABCE3CF5561
:10A2D000DF4F88839983AA83BB83C15AD040CE01C4
:10A2E0008F559F4F0E9492DA81E298E00E94ADDA8A
:10A2F00086E292E00E94A4DA82E292E00E9492DA80
:10A300008091E7089091E808A091E908B091EA08E7
:10A3100089839A83AB83BC838E010F5F1F4FC80173
:10A320000E9492DACF55DF4F188219821A821B825F
:10A33000C15AD0407E018DE6E80EF11C83E0D701C2
:10A340008C938983CE018F559F4F0E9492DAC7016B
:10A350000E949BDAC8010E949BDA4AE0D42EDA946C
:10A36000DD2031F0CE018F559F4F0E9492DAF7CF5A
:10A3700080EE92E10E94ADDACF55DF4F188219824C
:10A380001A821B82C15AD0403AE0D32EDA94DD20E3
:10A3900031F0CE018F559F4F0E9492DAF7CF85E0C2
:10A3A000D82ED982F701D082C8010E949BDAC7015A
:10A3B0000E949BDA26EF35E048E050E069EE75E058
:10A3C00086ED95E00E94885026EF35E048E050E0A9
:10A3D00061EE75E086ED95E00E94885026EF35E04D
:10A3E00044E650E06BEA77E086ED95E00E94885005
:10A3F00019828FEFD7018C93C8010E94A4DAC7019C
:10A400000E949BDA26EF35E044E050E06CEF72E00A
:10A4100086ED95E00E9488508091BA068983C80134
:10A420000E94A4DA198A1A8A1B8A1C8A80E090E0AA
:10A43000A0E8BFE38D879E87AF87B88B80915812C5
:10A4400090915912A0915A12B0915B1289839A830C
:10A45000AB83BC832CEA35EC47E25EE360915C128F
:10A4600070915D1280915E1290915F120F9427336C
:10A470006D837E838F8398872CEA35EC47E25EE319
:10A4800060916012709161128091621290916312DA
:10A490000F94C32B69877A878B879C8726EF35E0DB
:10A4A00044E150E0B80186ED95E00E94885084E1D7
:10A4B00090E09A838983C8010E9480DA8091ED112F
:10A4C0009091EE11A091EF11B091F01189839A83D0
:10A4D000AB83BC832CEA35EC47E25EE36091F1117B
:10A4E0007091F2118091F3119091F4110F94273330
:10A4F0006D837E838F8398872CEA35EC47E25EE399
:10A500006091F5117091F6118091F7119091F81109
:10A510000F94C32B69877A878B879C87C8010E9419
:10A5200089DA8CE0E3E9F2E0D80101900D928A9596
:10A53000E1F7C8010E9489DA1982C8010E949BDAFA
:10A540008FE790E09A838983C8010E9480DAEFE95F
:10A55000F2E0D80101900D92DA94E1F726EF35E0B0
:10A5600045E050E0B80186ED95E00E94885080916A
:10A57000E0058983C8010E94A4DA80E2E4EAF2E0FF
:10A58000D80101900D928A95E1F726EF35E040E27F
:10A5900050E0B80186ED95E00E948850F7011082E6
:10A5A000C7010E94A4DA84E198E00E94A4DA80E165
:10A5B00098E00E9492DACF55DF4F188219821A82F2
:10A5C0001B82C15AD040CE018F559F4F0E9492DA14
:10A5D00080E2D8011D928A95E9F726EF35E040E246
:10A5E00050E0B80186ED95E00E948850FE01F99692
:10A5F00088E0DF011D928A95E9F744E650E060E0CB
:10A6000070E049835A836B837C834D835E836F83C1
:10A61000788783E090E0A0E0B0E089879A87AB87F5
:10A62000BC874D875E876F87788B498B5A8B6B8B86
:10A630007C8B8D8B9E8BAF8BB88F898F9A8FAB8FD6
:10A64000BC8F8D8F9E8FAF8FB8A38EE190E0A0E07E
:10A65000B0E089A39AA3ABA3BCA38DA39EA3AFA391
:10A66000B8A789A79AA7ABA7BCA78DA79EA7AFA796
:10A67000B8AB89AB9AABABABBCAB8DAB9EABAFAB66
:10A68000B8AF26EF35E040E450E0B80186ED95E044
:10A690000E94885090E1D92EF8018D2D11928A9553
:10A6A000E9F726EF35E040E150E0B80186ED95E0AE
:10A6B0000E948850D8011D92DA94E9F726EF35E020
:10A6C00040E150E0B80186ED95E00E9488508CE1B1
:10A6D00099E00E9492DA2CE0D22EF8018D2D119291
:10A6E0008A95E9F726EF35E04CE050E0B80186EDB9
:10A6F00095E00E9488508CE6D8011D928A95E9F772
:10A7000026EF35E04CE650E0B80186ED95E00E947A
:10A7100088508AEC95E00E9489DA26EF35E048E01F
:10A7200050E068ED75E086ED95E00E948850F701F5
:10A730001192DA94E9F7C755DF4F1882C95AD04011
:10A7400080E090E0A0E4B0E4C356DF4F88839983B3
:10A75000AA83BB83CD59D040C7010E94ADDACE0198
:10A7600087559F4F0E949BDACE0183569F4F0E94D0
:10A7700092DA80E3D7011D928A95E9F789EB9CE193
:10A780000E94A1388AE00E94683826EF35E040E355
:10A7900050E0B70186ED95E00E9488508091F80561
:10A7A000811128C00091D6051091D7058091F6053A
:10A7B0009091F705F7019183808384E690E0909370
:10A7C000D7058093D60526EF35E044E050E060E001
:10A7D00073E086ED95E00E948850C7010E9480DA00
:10A7E00091E00536134009F490E08091F805892B3B
:10A7F0008093F8058091F805811105C060E08DEE29
:10A800009CE10E9410408DEC9CE10E94A1388AE0FE
:10A810000E9468389091F80581E08927C655DF4F7E
:10A820000FB6F894DEBF0FBECDBFDF91CF911F9161
:10A830000F91FF90EF90DF900895CF93DF9300D0BA
:10A840001F92CDB7DEB78091A6068823C1F083E3BF
:10A8500090E09C838B831A8219829E012F5F3F4F69
:10A8600040E150E067EA76E0CE0103960E9488500E
:10A870008DEC9CE10E94A1388AE00E9468380F901C
:10A880000F900F900F90DF91CF910895CF92DF92AC
:10A89000EF92FF92CF93C82F80918C11815082301C
:10A8A00008F069C00E94043B10928C110E9402AA19
:10A8B0006093C2057093C3058093C4059093C5054A
:10A8C000C090C605D090C705E090C805F090C905B6
:10A8D0000E94E72BAB01BC014093C6055093C7050E
:10A8E0006093C8057093C9058091AB069091AC0642
:10A8F000A091AD06B091AE068C199D09AE09BF09B5
:10A90000840F951FA61FB71F8093AB069093AC06CC
:10A91000A093AD06B093AE06C1110AC0C1E00E947B
:10A920001D548C2FCF91FF90EF90DF90CF90089522
:10A930008091A9069091AA0601969093AA06809309
:10A94000A9060E94E72BC090AF06D090B006E09019
:10A95000B106F090B206C616D706E806F906F0F67C
:10A960000E94E72B6093AF067093B0068093B10608
:10A970009093B206D3CFC0E0D2CF81E00C9446547E
:10A980000E94C3C10E94BD5480E00F94D31B8091EC
:10A99000FC068130A1F40E94714E82E697E00E948D
:10A9A000A13860E088E597E00E9410406EE571E014
:10A9B00080E090E00E945A2688E08093FC0608958B
:10A9C000CF92DF92EF92FF921F93CF93DF9300D04D
:10A9D0001F92CDB7DEB78EEEC82E82E0D82EE12CC6
:10A9E000F12CC982DA82EB82FC82BE016F5F7F4F5D
:10A9F0008AE50E94D33381110EC010E0812F0F90A1
:10AA00000F900F900F90DF91CF911F91FF90EF90DB
:10AA1000DF90CF9008950E942934C982DA82EB82B8
:10AA2000FC82BE016F5F7F4F8AE50E94D333182FEF
:10AA3000882319F30E94714E8CE398E00E94A1389C
:10AA40000E94C054DBCFCF92DF92EF92FF921F9310
:10AA5000CF93DF9300D01F92CDB7DEB78EEEC82E16
:10AA600082E0D82EE12CF12CC982DA82EB82FC82C2
:10AA7000BE016F5F7F4F8AE00E94D33381110EC009
:10AA800010E0812F0F900F900F900F90DF91CF91DA
:10AA90001F91FF90EF90DF90CF9008950E9429348E
:10AAA0000E94F3330E940E340E94F333C982DA828B
:10AAB000EB82FC82BE016F5F7F4F8AE00E94D3333E
:10AAC000182F8823E9F20E94714E8FEF97E00E94C1
:10AAD000A1380E94C054D5CFCF93DF9300D01F92EE
:10AAE0001F92CDB7DEB781E08093A60680E1E7EA4A
:10AAF000F6E0DF011D928A95E9F70E941D5486E178
:10AB00008D8382E390E09C838B831A8219829E015D
:10AB10002F5F3F4F41E050E0BE016B5F7F4FCE01A2
:10AB200003960E9488500F900F900F900F900F90F7
:10AB3000DF91CF910895CF93DF93CDB7DEB7A8977C
:10AB40000FB6F894DEBF0FBECDBF8C01F42E0E946D
:10AB5000C3C10E94714E88E397E00E94A13801159D
:10AB6000110511F40FE217E08091990580FD79C07D
:10AB70008160809399058BE197E00E94A1388AE07B
:10AB80000E946838CC24C3948AE5D82ED092401411
:10AB9000C0923F148FE090E0909342148093411450
:10ABA00097E0792E7092331422E8E22EE092361468
:10ABB00034E8832E912CA12CB12C809237149092E2
:10ABC0003814A0923914B0923A1483EE93E10E94A3
:10ABD000F134D0924014C0923F1488E590E09093F5
:10ABE00042148093411470923314E0923614809290
:10ABF000371490923814A0923914B0923A1483EE1C
:10AC000093E10E94F1348AE289838A838B838C8367
:10AC1000F801DE011596BE016F5F7F4FCD01861BE7
:10AC2000970B2491319621110CC0FB01E80FF91FFD
:10AC30008AE29F01261B370B2832310524F48193C9
:10AC4000F8CF2D93EBCF20E630E140E050E083EEEB
:10AC500093E10E94C7E96AE070E080E090E00E9422
:10AC6000FA2C61E086E297E00E94DD3F89EE93E0F6
:10AC700030E6019729F0232F2A950000E9F7F9CF54
:10AC8000F89489EE93E038EE019729F0232F2A9566
:10AC90000000E9F7F9CF0E94C3C1FF2031F00E9404
:10ACA000521F0E946B1FA895FECF0E94501FF9CF24
:10ACB0008091FB06882319F01092FB06089540E06E
:10ACC00070E060E080EE98E10E949B5580910C0D51
:10ACD00090910D0D2FEF3FEF981751F0E92FF0E015
:10ACE000E45FF24F228130E09F5F9F7790930D0DDC
:10ACF000C90108951F920F920FB60F9211240F9061
:10AD00000FBE0F901F9018951F920F920FB60F92C3
:10AD100011240BB60F920F931F932F933F934F93D2
:10AD20005F936F937F938F939F93AF93BF93CF93D3
:10AD3000DF93EF93FF93C091C60000910D0DD0916A
:10AD40000C0D11E01D0F1F7790912704913108F031
:10AD50009FC0E92FF0E08827EF54F94A8F4F0D94F8
:10AD60002432C256F15600570F57165748571A57F4
:10AD700048571E572257485726572A572E57355798
:10AD800048574057C03229F028F5CA3011F0CD306D
:10AD900031F5011731F0ED2FF0E0E45FF24FC2839F
:10ADA000D12FD0930C0DFF91EF91DF91CF91BF91F7
:10ADB000AF919F918F917F916F915F914F913F9153
:10ADC0002F911F910F910F900BBE0F900FBE0F9000
:10ADD0001F901895CD3481F081E0CE3471F080E180
:10ADE0000CC0CA3338F4C033A0F6C03291F2CD3271
:10ADF000B1F7CFCFCD3499F782E080932704C9CF44
:10AE0000C13359F018F4C03221F2E9CF88E0C433DD
:10AE1000A1F38BE0C83389F3E2CF83E0EECF84E087
:10AE2000C03359F386E0C13341F3D9CF85E0C8334D
:10AE3000B1F6E3CF87E0C23391F6DFCF89E0C133CB
:10AE400071F6DBCF8AE0C03351F6D7CF8CE0C73341
:10AE500031F6D3CF8DE0C63311F6CFCFC03209F42F
:10AE600098CF8EE0C33549F2BACF80ED8C0F8A308F
:10AE700008F08FCF9FE0909327048093280489CF18
:10AE8000CA3019F0CD3009F084CF1092270481CF59
:10AE9000CA3019F0CD3009F07CCF80919D14882301
:10AEA000A1F3973089F038F4953079F71092440285
:10AEB00010929E0CEACF9A3059F09F3031F7809172
:10AEC00028040E941032E1CF81E080932406DDCF78
:10AED00081E080932306D9CF8EBD0DB407FEFDCF50
:10AEE00008958FEF8EBD0DB407FEFDCF8EB508958A
:10AEF000909164009B7F90936400982F906A969540
:10AF00009CBD80FD03C091E0863009F490E09DBDBA
:10AF10000895CF93DF93EB010E94A138CE01DF911A
:10AF2000CF910C940DB22F923F924F925F926F92FD
:10AF30007F928F929F92AF92BF92CF92DF92EF92C9
:10AF4000FF920F931F93CF93DF93009709F0AAC14D
:10AF50001092F10C1092F00C909398058093970545
:10AF6000BAE0CB2EB0E2DB2EE12CF12C15E002E8AA
:10AF700046015701C4E1D0E0109286131092851368
:10AF80001093791300937C1380927D1390927E131B
:10AF9000A0927F13B092801389E293E10E94F13472
:10AFA00021972FEF821A920AA20AB20A209721F75C
:10AFB00044E1C40ED11CE11CF11C8AE5C81680E2F4
:10AFC000D806E104F104A1F6C12CA0E2DA2EE12CAE
:10AFD000F12CD5E0C2E81092861310928513D0931D
:10AFE0007913C0937C13C0927D13D0927E13E092AC
:10AFF0007F13F092801389E293E10E94F134109262
:10B00000861310928513D0937913C0937C13D701C4
:10B01000C6018C529F4FAF4FBF4F80937D139093CB
:10B020007E13A0937F13B093801389E293E10E9473
:10B03000F134EFEFCE1ADE0AEE0AFE0AFAE0CF167E
:10B04000F0E2DF06E104F10431F6FEEDCF2EF0E28E
:10B05000DF2EE12CF12CD5E0C2E81092861310927D
:10B060008513D0937913C0937C13C0927D13D09233
:10B070007E13E0927F13F092801389E293E10E94A5
:10B08000F1342FEFC21AD20AE20AF20A46EEC416CF
:10B0900040E2D406E104F10401F7CC24C394E2E1D8
:10B0A000DE2EE12CF12C0AE010E0D5E0C2E810938E
:10B0B000861300938513D0937913C0937C13C092A9
:10B0C0007D13D0927E13E0927F13F092801389E279
:10B0D00093E10E94F1341093861300938513D0936B
:10B0E0007913C0937C13D701C6018096A11DB11DB1
:10B0F00080937D1390937E13A0937F13B09380135E
:10B1000089E293E10E94F1348FEFC81AD80AE80A65
:10B11000F80AE5E0CE16E2E1DE06E104F10439F6D4
:10B120000091F00C1091F10C0115110509F0D6C039
:10B130008091EF0C882309F4E1C02AE030E240E07E
:10B1400050E068EE73E089E293E10E94C7E9C1E054
:10B15000D0E003E010E0E090F00CF090F10C35E06E
:10B16000332E42E8242E44244A94542C64E0662E64
:10B17000712C7FE1C72E74E0D72E8091F00C909156
:10B18000F10C800F911FE816F90608F0D5C0C70131
:10B190000E94E2EA882309F481C0809107126AEFD5
:10B1A00071E1882311F067E072E1FB01019000205A
:10B1B000E9F7CF010197861B970BF4E1FC9F900103
:10B1C000FD9F300D1124265F3F4D50E040E0459734
:10B1D00010F0FB01128A89E293E10E94C7E9CE01D7
:10B1E0008F5F9D4EB0E0A0E021964E0124E0880CD8
:10B1F000991C2A95E1F7FDEF8F1AFFE99F0AB12C00
:10B20000A12C2091A91424FF7EC070928613609215
:10B2100085133092791320927C1380937D13909341
:10B220007E13A0937F13B093801389E293E10E9471
:10B23000F134D0928613C092851330927913209204
:10B240007C1380927D1390927E13A0927F13B09214
:10B25000801389E293E10E94F134B70185E798E118
:10B260000E946C418091071267E072E1811102C077
:10B270006AEF71E182E798E10E9489576EE57CE010
:10B280008EE698E10E9489576AEF71E18DE698E1B8
:10B290000E94895789E698E10E94A1382FEFE21AAF
:10B2A000F20A6BCF2091F00C3091F10CA9014150C2
:10B2B000510960919705709198056817790738F4DE
:10B2C0002C5F3F4F3093F10C2093F00C45CE44306F
:10B2D000510508F43DCE24503109F4CF0430110556
:10B2E00069F48091EF0C882331F083E090E0909333
:10B2F000F10C8093F00CD0E0C0E02DCFD0E0C0E0A6
:10B3000004E010E028CF109286131092851330923B
:10B31000791320927C1380937D1390937E13A093D6
:10B320007F13B093801389E293E10E94F13450922D
:10B3300086134092851381CFDF91CF911F910F919A
:10B34000FF90EF90DF90CF90BF90AF909F908F9045
:10B350007F906F905F904F903F902F900895AF92A5
:10B36000BF92CF92DF92EF92FF920F931F93CF93F2
:10B37000DF93CDB7DEB7E6970FB6F894DEBF0FBE0A
:10B38000CDBF00914B0510914C05F80101900020B4
:10B39000E9F731976F01C01AD10AF801CF01801B7C
:10B3A000910B8C159D053CF481918F32B9F7DF012B
:10B3B00011971C92F3CF8BE1E9ECF4E1DE015C968E
:10B3C00001900D928A95E1F7F12CE12CEC14FD042B
:10B3D0000CF05DC0F801EE0DFF1D8081811103C0EE
:10B3E0008FEFE81AF80A5801AE0CBF1CF5018081F6
:10B3F000882309F44CC0FFEFEF1AFF0AF801EE0DA5
:10B40000FF1D7F01E01AF10A81918111FACFCE016F
:10B410004C960E94A0B68BE1FE017C96DE0111964F
:10B4200001900D928A95E1F7B501CE0101960E9437
:10B43000AEAECE0101960E94FD2F8FE20E946838C9
:10B440008091071281113BC085EF93E00E940DB2FD
:10B450008091A91484FF1BC019821C8221E0A501E0
:10B46000BE01645E7F4FCE0101960E94E2B8811159
:10B4700029C08AE00E9468380E94754EB50184E5B3
:10B4800097E10E948957CE0101960E94FD2F8AE024
:10B490000E946838CE014C960E94FD2FE6960FB6AA
:10B4A000F894DEBF0FBECDBFDF91CF911F910F91FA
:10B4B000FF90EF90DF90CF90BF90AF90089587E01E
:10B4C00092E1C4CFCE014C960E940FB68BE1FE01F3
:10B4D0003196DE015C9601900D928A95E1F7CE01DE
:10B4E00001960E94FD2F72CF2F923F924F925F9252
:10B4F0006F927F928F929F92AF92BF92CF92DF9284
:10B50000EF92FF920F931F93CF93DF9300D000D061
:10B5100000D01F921F92CDB7DEB7B82E8091F90DE3
:10B52000843008F0D1C10E9402AA6B017C01809195
:10B53000F90D811108C080910C0D90910D0D891BA2
:10B540008F7709F4A4C681E6A82E13C08A3019F0BB
:10B550008D3009F0F6C01092F40D8091920D90910B
:10B56000930DFC01E257F24F1682892BF1F40E94F1
:10B5700010C58091F90D843008F0ECC080910C0D5D
:10B5800090910D0D891B8F7709F4E4C00E946656D7
:10B5900097FFDCCF0E94714E85EB95E00E94A138A9
:10B5A00080910C0D80930D0DE4CF1092930D1092AD
:10B5B000920D04E91DE0F8018191803209F446C042
:10B5C0008E3409F0A9C060EB75E0C8010F94DA2A47
:10B5D0004C01892B41F06EE470E0C80104960F9491
:10B5E0007B35009709F4C8014AE050E070E060E064
:10B5F00001960F944A282B013C0180918E0D909169
:10B600008F0DA091900DB091910D0196A11DB11DCE
:10B61000481659066A067B0629F060E08DE795E03A
:10B62000892851F16AE270E0C8010F94AA359C01A3
:10B63000009729F1982F901B912C992349F0915054
:10B64000F801E90FF11D80819826F7CF8F01B3CF64
:10B650004AE050E070E060E0C90101960F944A288A
:10B66000292D30E050E040E062177307840795070A
:10B6700051F060E08EE595E00E94D4F07ACF60E072
:10B6800084E395E0F9CF40928E0D50928F0D609239
:10B69000900D7092910D8091FC068130E1F067E48D
:10B6A00070E0C8010F947B350097A9F04AE050E0A4
:10B6B00070E060E001960F944A28643071058105BE
:10B6C000910548F483E994E00E94A13860E089E89C
:10B6D00094E00E941040C092A307D092A407E09289
:10B6E000A507F092A6078091940D8B3309F441CF02
:10B6F0008091F90D843008F03CCF8091FB0D8A9D3C
:10B70000C001112464E97DE08450924F0F94863586
:10B7100080E00E948EF02DCF8091A91480FFBBCFD6
:10B7200064ED7DE2C8010F94DA2A009731F0FC0144
:10B73000838180538A3008F0AECF60E08AE095E0E4
:10B740009BCF22E93DE044E95DE064EF7DE00E94AB
:10B75000661D0FCF8091A91482FFB6C01A8219828C
:10B7600071E6F72EE0E1EE2EF9E6DF2E8091F90D7D
:10B77000843008F0A9C00E949E1D8111A5C041E03F
:10B7800050E0BE016B5F7F4F8DE096E10E9462B496
:10B790000D8110E0019711F00FEF1FEF809115164A
:10B7A00090911616A0911716B09118168093A514B3
:10B7B0009093A614A093A714B093A8140E949E1D62
:10B7C0000F3F100749F4811107C00E94714E83EDAD
:10B7D00095E00E94A138CACF4091FB0D242F30E0A4
:10B7E0000A3061F00D3051F0882309F45FC089817F
:10B7F0009A81009719F001969A8389831092AE047A
:10B8000089819A81F29EF001F39EF00D1124E75098
:10B81000F24FE80FF91F1382892B69F50E9410C5BA
:10B820000E949E1D882309F4A1CF0E94DE618DE055
:10B8300096E10E940FB68091A014882391F1815067
:10B840008093A0148D9DC001112462E08C5C994FFF
:10B850000E9464BBE091A01424E0E29FF001112457
:10B86000E05DF94F60817181828193810E94B722EE
:10B870000E9417AE7BCF1A82198281E00E948EF05F
:10B880008091A5149091A614A091A714B091A8142A
:10B890008093F50D9093F60DA093F70DB093F80DEE
:10B8A000BFCF0E9418B6E092FC0660CF4F9DA0016A
:10B8B00011244450524F9E012F5F3F4F6EEA74E0B7
:10B8C000802F0E94661D52CF0E9402AA6B017C014C
:10B8D000B11004C080918B11882351F0C092DE1109
:10B8E000D092DF11E092E011F092E111BB24B39409
:10B8F0008091230590912405A0912505B0912605FE
:10B900000097A105B105B1F04091DE115091DF1112
:10B910006091E0117091E111840F951FA61FB71F70
:10B92000A7019601281B390B4A0B5B0BDA01C901F1
:10B93000B7FF92C18091130290911402A091150259
:10B94000B0911602892B8A2B8B2B09F099C10E948A
:10B9500002AA4B015C0180919E0C811108C02091CC
:10B96000F1129091F21281E0291301C080E0209140
:10B9700053123091541291E089272A3A31050CF480
:10B9800080E091E04091B3045091B4046091B5041B
:10B990007091B604452B462B472B09F490E098177D
:10B9A00089F0882309F4BDC1D501C40180569444AF
:10B9B000A24FBF4F8093B3049093B404A093B504F7
:10B9C000B093B60440907502509076026090770272
:10B9D000709078022091AF043091B0044091B1048E
:10B9E0005091B204C301B2010F945D2B882319F169
:10B9F0008091B3049091B404A091B504B091B604C1
:10BA00004092AF045092B0046092B1047092B204BC
:10BA1000892B8A2B8B2B09F449C0D501C401805690
:10BA20009444A24FBF4F8093B3049093B404A09367
:10BA3000B504B093B6048091B3049091B404A0917E
:10BA4000B504B091B6040097A105B10579F1881A43
:10BA5000990AAA0ABB0AB7FC29C01092B304109233
:10BA6000B4041092B5041092B60483E396E00E94E9
:10BA7000A13860E08FE196E00E941040809155125D
:10BA8000909156121816190624F490E080E00E9456
:10BA90006E1F8091EA119091EB111816190634F47B
:10BAA0001092EB111092EA110E9496C18091BB0492
:10BAB0009091BC04A091BD04B091BE044601570111
:10BAC000881A990AAA0ABB0AD501C401B7FDB9C1EF
:10BAD0002091F1129091F21240913502809134023E
:10BAE000291323C190912009899FC0011124880F37
:10BAF000892F881F990B91958D8380912109489FEB
:10BB0000C0011124880F892F881F990B91958E836E
:10BB10000E9402AA69837A838B839C8340E0BE01E2
:10BB20006F5F7F4FCE0105960E94B81C6D8170E05B
:10BB300089E00E94F9A841E0BE016F5F7F4FCE010E
:10BB400005960E94B81C6E8170E087E00E94F9A8FB
:10BB500080912F06882309F467C10091200210917B
:10BB60002102C801029720915512309156122817D0
:10BB700039070CF459C18090F2128F821886198609
:10BB80001A861B868091F1129F80891509F4E7C0FF
:10BB9000892D90E037E6A32EA89EF001A99EF00D16
:10BBA0001124EB5DF64F458956896789708D452BC9
:10BBB000462B472B81F4418D528D638D748D452B1F
:10BBC000462B472B41F4458D568D678D70A1452B33
:10BBD000462B472BE1F127E6B22EB89E9001B99E85
:10BBE000300D1124A9014B5D564F1A01FA016181F4
:10BBF0007281838194810F94DB344B015C01F101EC
:10BC000061A172A183A194A10F94622B2B013C012D
:10BC1000F10165A176A187A190A50F94622B9B01EC
:10BC2000AC01C301B2010F942733A50194010F9415
:10BC3000C32B4B015C01288539854A855B850F94B0
:10BC40008D34181624F488869986AA86BB868F813F
:10BC50008F5F87708F8396CF0E94714E6091A1078E
:10BC60007091A20782EE95E00E9489578AE00E94B7
:10BC7000683840E070E060E090E080E00E949B5512
:10BC80009091F1128091F212981749F0C092DE1152
:10BC9000D092DF11E092E011F092E11158CEBB207A
:10BCA00019F01092BF0453CE0E9402AA0091DE1137
:10BCB0001091DF112091E0113091E1118090130279
:10BCC00090901402A0901502B0901602080D191D54
:10BCD0002A1D3B1D601B710B820B930B97FDE1CF5F
:10BCE0008091BF04811133CE81E08093BF045F9ABD
:10BCF00080919F0C8E7F80939F0C8A9A80919F0CDD
:10BD00008D7F80939F0C8091080180958170809336
:10BD1000060180919F0C8B7F80939F0C0E94501F87
:10BD200016CE80E090E0DC0145CE2091F21257E67D
:10BD3000259F900111242B5D364FF901EF59FF4FDC
:10BD40009081899FC0011124880F892F881F990B2A
:10BD500091958D832E593F4FF9018081D0CE20914E
:10BD60001A0230911B0240911C0250911D026885FD
:10BD700079858A859B850F94C32B4B015C01B801A3
:10BD8000012E000C880B990B0F94642B9B01AC01C6
:10BD9000C501B4010F942D3269837A838B839C8310
:10BDA00040911E0250911F02B801CE0101960E94DF
:10BDB000CEC489809A80AB80BC804090B7045090FC
:10BDC000B8046090B9047090BA04A3019201C5014F
:10BDD000B4010F945D2B87FF16C028E431EE4AE7CB
:10BDE0005FE3C301B2010F94C32B20E037ED43EAB8
:10BDF0005CE30F942D32A50194010F94C32B69834A
:10BE00007A838B839C8369817A818B819C81609307
:10BE1000B7047093B8048093B9049093BA040F9454
:10BE20009933CB010E946E1FF4E6CF0ED11CE11CAA
:10BE3000F11CC092BB04D092BC04E092BD04F0920D
:10BE4000BE040E9410C58091FC06882309F4E0C15D
:10BE500080912602882309F4A3C08091FD048111FA
:10BE60009FC080918B11811108C080918C1181300D
:10BE700021F08091A91482FF93C0F894649B10C0B4
:10BE80008091220290912302A0912402B091250278
:10BE90008093FD059093FE05A093FF05B0930006E7
:10BEA0006091FD057091FE058091FF05909100065F
:10BEB000789420E030E0A9010F945D2B87FF70C0DB
:10BEC00001E00093FD0480918B11811167C088E42B
:10BED00096E00E94A1388AE00E94683884E080934E
:10BEE000060D82E08093F20C81E09AE59093401475
:10BEF00080933F148EE490E0909342148093411419
:10BF000087E08093331482E88093361484E890E0CD
:10BF1000A0E0B0E08093371490933814A0933914C4
:10BF2000B0933A1483EE93E10E94F1340E948D4065
:10BF30000093F91140E36CE876E084E799E00E9411
:10BF4000924061E088E699E00E94744010912705D4
:10BF500060E010278CE399E069F48AE796E00E949C
:10BF6000DD3F80E30E9468388AE00E94683860E024
:10BF70008DE596E00E94DD3F88E696E00E94A138BC
:10BF800080E30E9468388AE00E946838112331F00B
:10BF900083E696E09093EE0C8093ED0C0E94DE61B8
:10BFA00090910901892F80958170109100021817D6
:10BFB000C9F02091A91420622093A9148093000253
:10BFC00090FD3FC164EF71E080E090E00E945A264E
:10BFD0000E943AB68091A91483FD7CC1111133C12E
:10BFE0000E9436360E9402AA6B017C011091170252
:10BFF0001123F1F0809128058823D1F04091C004ED
:10C000005091C1046091C2047091C304460157016C
:10C01000841A950AA60AB70AB501A40177FD1AC0C9
:10C02000833009F42FC10CF01EC181300CF023C104
:10C03000212F30E0A8EEB3E00F94F531C60ED71EE5
:10C04000E81EF91EC092C004D092C104E092C2045E
:10C05000F092C30480918C11813009F073C00E946A
:10C0600002AA6B017C018091C8049091C904A0913F
:10C07000CA04B091CB04A7019601281B390B4A0BC7
:10C080005B0BDA01C901B7FD3AC0D701C601805F79
:10C09000984DAF4FBF4F8093C8049093C904A093AD
:10C0A000CA04B093CB048090C6059090C705A090B9
:10C0B000C805B090C9050E94E72BAB01BC014093B5
:10C0C000C6055093C7056093C8057093C905809154
:10C0D000AB069091AC06A091AD06B091AE06881962
:10C0E0009909AA09BB09840F951FA61FB71F809342
:10C0F000AB069093AC06A093AD06B093AE068091CC
:10C10000C4049091C504A091C604B091C70446012F
:10C110005701881A990AAA0ABB0AD501C401B7FDBA
:10C1200011C020E8C20E2EEED21E26E3E21EF11C44
:10C13000C092C404D092C504E092C604F092C70431
:10C140000E941D540E94DF390E94AA41809122055D
:10C15000882379F10E9402AA6B017C0180911E055F
:10C1600090911F05A0912005B0912105460157012E
:10C17000881A990AAA0ABB0AD501C401B7FD19C0D9
:10C180002091220530E0A8EEB3E00F94F531C60E01
:10C19000D71EE81EF91EC0921E05D0921F05E09220
:10C1A0002005F092210580E00E94F4BD8AE00E9403
:10C1B000683880911D05882359F10E9402AA6B01FD
:10C1C0007C018091190590911A05A0911B05B091F1
:10C1D0001C05A7019601281B390B4A0B5B0BDA01E2
:10C1E000C901B7FD15C020911D0530E0A8EEB3E0F0
:10C1F0000F94F531C60ED71EE81EF91EC092190520
:10C20000D0921A05E0921B05F0921C050E94D5AD54
:10C210002B960FB6F894DEBF0FBECDBFDF91CF9146
:10C220001F910F91FF90EF90DF90CF90BF90AF9054
:10C230009F908F907F906F905F904F903F902F9046
:10C2400008950E9429B6123008F0CCCE0E943636EE
:10C2500060E085EC96E056C083ED96E09093EE0C9E
:10C260008093ED0CBFCE843009F0E2CE0E94754E73
:10C270008AED96E004C00E94754E89E097E00E9426
:10C28000A138D6CE0E94754E82EF96E0F8CF80910D
:10C29000A3079091A407A091A507B091A607A701B5
:10C2A0009601281B390B4A0B5B0BDA01C901885E2A
:10C2B0009340A109B109B7FD46C98DEC95E00E94F4
:10C2C000A138C092A307D092A407E092A507F092EC
:10C2D000A60739C91230C8F48DE996E00E94A1384A
:10C2E0008AE00E9468380E94152D90E080E00E944C
:10C2F000935710920A0D1092090D1092080D60E0EC
:10C3000086EB96E00E9410406DCE123009F06ACEA6
:10C310000E9494BA882379F081E00E946ABA42EBC5
:10C3200050E06DE278E08EEA94E10E9462B48EEA19
:10C3300094E10E940FB60E94EB2F81118DCF0E94D5
:10C34000D52F0E9410BB0E9465BA4CCECF93DF93CD
:10C350008091F1129091F212891B8095877019F4E7
:10C360000E94745AF5CF8091F1128F5F8770A0916F
:10C37000F11297E6A99FD0011124FD01EB5DF64F64
:10C38000EF0119929A95E9F798E09083A65CB64F71
:10C3900090E1E3E0F3E101900D929A95E1F72091AD
:10C3A000F1129091F212291303C094E69093EE12C9
:10C3B0008093F112DF91CF910C9403309091F112A0
:10C3C0008091F212981306C080912309909124095C
:10C3D000892B21F080E00E94745AF0CF0895CF920B
:10C3E000DF92EF92FF92FC01C080D180E280F38067
:10C3F0002091C10C3091C20C4091C30C5091C40CDF
:10C40000C701B6010F94C32B0F949A3460930F1396
:10C41000709310138093111390931213C092FF1214
:10C42000D0920013E0920113F09202139091F11256
:10C430008091F212981731F0FF90EF90DF90CF903B
:10C440000C94A6610E94DE610E945A2A40910F134B
:10C4500050911013609111137091121340931F06A5
:10C46000509320066093210670932206882331F0B2
:10C47000FF90EF90DF90CF900C940330FF90EF90FF
:10C48000DF90CF9008954F925F926F927F928F923C
:10C490009F92AF92BF92CF92DF92EF92FF920F9353
:10C4A0001F93CF93DF93EC018B017A016901F901AE
:10C4B00080819181A281B381FA01408151816281A1
:10C4C0007381F80180809180A280B3804880598078
:10C4D0006A807B804092F3125092F4126092F512BF
:10C4E0007092F6128092F7129092F812A092F912BE
:10C4F000B092FA124093FB125093FC126093FD121B
:10C500007093FE128093FF1290930013A093011377
:10C51000B09302132091C10C3091C20C4091C30C16
:10C520005091C40CF60160817181828193810F94D6
:10C53000C32B0F949A344B015C012091BD0C3091B8
:10C54000BE0C4091BF0C5091C00CF701608171810D
:10C55000828193810F94C32B0F949A346B017C01D9
:10C560002091B90C3091BA0C4091BB0C5091BC0C8D
:10C57000F80160817181828193810F94C32B0F94A4
:10C580009A342B013C012091B50C3091B60C4091AE
:10C59000B70C5091B80C688179818A819B810F9486
:10C5A000C32B0F949A3460930313709304138093F6
:10C5B000051390930613409207135092081360924C
:10C5C000091370920A13C0920B13D0920C13E092CD
:10C5D0000D13F0920E1380920F1390921013A092ED
:10C5E0001113B09212139091F1128091F2129817D8
:10C5F00091F0DF91CF911F910F91FF90EF90DF901D
:10C60000CF90BF90AF909F908F907F906F905F90F2
:10C610004F900C94A6610E94DE610E945A2A4091BC
:10C620000B1350910C1360910D1370910E13009128
:10C630000713109108132091091330910A13C09029
:10C640000313D0900413E0900513F0900613C092EA
:10C650001306D0921406E0921506F0921606009387
:10C660001706109318062093190630931A06409364
:10C670001B0650931C0660931D0670931E06409186
:10C680000F13509110136091111370911213409376
:10C690001F0650932006609321067093220688237C
:10C6A00091F0DF91CF911F910F91FF90EF90DF906C
:10C6B000CF90BF90AF909F908F907F906F905F9042
:10C6C0004F900C940330DF91CF911F910F91FF9009
:10C6D000EF90DF90CF90BF90AF909F908F907F9022
:10C6E0006F905F904F9008953F924F925F926F923C
:10C6F0007F928F929F92AF92BF92CF92DF92EF92F2
:10C70000FF920F931F93CF93DF93CDB7DEB7689758
:10C710000FB6F894DEBF0FBECDBFD82E2A013B0165
:10C72000480159013E2C20E030E0A901C501B801C3
:10C730000F945D2B811110C081E08D1508F0B6C0FB
:10C7400060E070E080E793E420E030E040E752E40E
:10C750000F9427334B015C018D8A9E8AAF8AB88E75
:10C760000D2D10E0F801E653F64EE491BB24B3948E
:10C770001E160CF4B12CCC24C39420E030E0A901A7
:10C78000C301B2010F948D3418160CF0C12CBC14E7
:10C7900071F092E0D9120BC0332049F081E00F9480
:10C7A000D31B69E170E080E090E00E945A2680E0AF
:10C7B0000E94093069837A838B839C8381E00E9485
:10C7C00009306D837E838F83988782E00E940930D1
:10C7D00069877A878B879C8783E00E9409306D8701
:10C7E0007E878F87988B000F111F000F111FE1E0CC
:10C7F000F0E0EC0FFD1F0E0F1F1FF80110821182D9
:10C80000128213829E01235F3F4FAE01475F5F4F4D
:10C81000BE016B5F7F4FCE0101960E944362F8011B
:10C820004082518262827382198A1A8A1B8A1C8A08
:10C830008091230990912409892B91F4CE0141968E
:10C840007C018E010B5E1F4F9E01235F3F4FAE01A7
:10C85000475F5F4FBE016B5F7F4F40970E94F8F0CC
:10C860000E94DE61BC1451F092E0D91205C0332061
:10C8700019F080E00F94D31B0E94585668960FB6AB
:10C88000F894DEBF0FBECDBFDF91CF911F910F9106
:10C89000FF90EF90DF90CF90BF90AF909F908F90E0
:10C8A0007F906F905F904F903F90089560E070E8A8
:10C8B0008BE395E449CF4F925F926F927F928F9274
:10C8C0009F92AF92BF92CF92DF92EF92FF920F931F
:10C8D0001F93CF93DF93CDB7DEB72C970FB6F894A5
:10C8E000DEBF0FBECDBF2B013C0129873A874B87A6
:10C8F0005C8747015801F601E080F18002811381D5
:10C9000020E030E0A901B701C8010F945D2B882316
:10C9100009F488C05E2D4F2D302F212F852F942FA5
:10C92000A32FB22F89839A83AB83BC8320E030E0AE
:10C93000A901B701C8010F945D2B811108C0E090D7
:10C940004502F09046020091470210914802C7014B
:10C95000D8018D839E83AF83B887A5019401609130
:10C9600071027091720280917302909174020F941F
:10C970005D2B87FF0CC08092710290927202A09290
:10C980007302B0927402CE0101960E94352B409240
:10C99000690250926A0260926B0270926C02898501
:10C9A0009A85AB85BC8580936D0290936E02A093AF
:10C9B0006F02B0937002CE0105960E94352BA5013F
:10C9C0009401609171027091720280917302909152
:10C9D00074020F948D34181664F480927102909250
:10C9E0007202A0927302B0927402CE0101960E946C
:10C9F000352B0E94DE612C960FB6F894DEBF0FBE79
:10CA0000CDBFDF91CF911F910F91FF90EF90DF90FD
:10CA1000CF90BF90AF909F908F907F906F905F90DE
:10CA20004F90089550E040E030E820E477CFCF9277
:10CA3000DF92EF92FF920F931F936A01E0907102D1
:10CA4000F09072020091730210917402FB01208138
:10CA5000318142815381FC016081718182819381A6
:10CA60000E945B641F910F91FF90EF90DF90CF9039
:10CA70000895CF92DF92EF92FF920F931F936B0175
:10CA8000FC01E080F18002811381E9E6F2E024817B
:10CA900035814681578160817181828193810E94B5
:10CAA0005B641F910F91FF90EF90DF90CF900895FE
:10CAB0000F931F93CF93DF93EC018B0181E00F94D1
:10CAC000D31B69E170E080E090E00E945A26B80133
:10CAD000CE010E943965C091FB0680E00F94D31B04
:10CAE0001092FB0682E00E9433300E94502BC2FB62
:10CAF000CC27C0F981E08C27DF91CF911F910F9156
:10CB00000895AF92BF92CF92DF92EF92FF920F9370
:10CB10001F93CF93DF9300D01F92CDB7DEB7FC01F8
:10CB2000E080F18002811381611112C0A090710236
:10CB3000B0907202C0907302D09074029501A60169
:10CB4000B701C8010F945D2B87FF02C075018601F4
:10CB500020E030E048EC53E4B701C8010F945D2BAE
:10CB600087FD04C0E12CF12C08EC13E4C701D801C7
:10CB700089839A83AB83BC8368EF72E0CE01019610
:10CB80000E9439650F900F900F900F90DF91CF9119
:10CB90001F910F91FF90EF90DF90CF90BF90AF90DB
:10CBA00008953F924F925F926F927F928F929F92E1
:10CBB000AF92BF92CF92DF92EF92FF920F931F93AB
:10CBC000CF93DF9300D01F92CDB7DEB7382E80E031
:10CBD00090E0A0E2B1E489839A83AB83BC83C090E8
:10CBE000E812D090E912E090EA12F090EB1220E007
:10CBF00030E0A901C701B6010F945D2B87FF0CC07F
:10CC0000A701960160E070E080E291E40F942C327D
:10CC100069837A838B839C8360E0CE0101960E94B6
:10CC200081654090690250906A0260906B0270903A
:10CC30006C0280906D0290906E02A0906F02B09096
:10CC40007002332089F10E94235519821A821B82B7
:10CC50001C82E0907102F0907202009173021091B8
:10CC60007402CE0101966C01A5019401C301B201C9
:10CC70000E945B6430929F070E94D82B0F900F9008
:10CC80000F900F90DF91CF911F910F91FF90EF9038
:10CC9000DF90CF90BF90AF909F908F907F906F90DC
:10CCA0005F904F903F9008950E94E054CECF8091C6
:10CCB0009F07882319F080E00E94D16580E00895E5
:10CCC0002F923F924F925F926F927F928F929F929C
:10CCD000AF92BF92CF92DF92EF92FF920F931F938A
:10CCE000CF93DF93CDB7DEB766970FB6F894DEBF6C
:10CCF0000FBECDBFF82E282E312CF101E653F64E93
:10CD0000D49022E0821335C080919F07811103C027
:10CD100081E00E94D1650E942355811139C186ECC2
:10CD200099E10E94D71D20E030E0A9010F945D2B0E
:10CD30008823F9F06D2DDD0C770B880B990B0F9480
:10CD4000642B2B013C0186EC99E10E94D71D4B011D
:10CD50005C0120E030E040EA50E40F945D2B11E0EC
:10CD600087FF1CC0812C912C90EAA92E90E4B92E4B
:10CD700015C06D2DDD0C770B880B990B0F94642B70
:10CD80002B013C01C101880F991F880F991F825404
:10CD9000964E0E94D71D4B015C0110E0A301920149
:10CDA000C501B4010F94C32B4B015C016101CC0C94
:10CDB000DD1CCC0CDD1CC6018E54964E0E94D71D86
:10CDC000EE24E394E12620E030E040EC5FE30F94B2
:10CDD000C32BA30192010F94C32BAB01BC0100E054
:10CDE00010E098018F2D0E94746320E030E0A901CB
:10CDF000C501B4010F945D2BF601EA55F64EFA8B8E
:10CE0000E98B882309F44DC0F2E000E010E020E453
:10CE100031E4FF1619F000E010E09801B501A4011B
:10CE20007058E12C8F2D0E947463A5019401C501F7
:10CE3000B4010F942D326B8B7C8B8D8B9E8B22E0FB
:10CE4000F216E9F0F101ED55F64E6491611107C05B
:10CE50000E94754E81E899E10E94A1386AE070E075
:10CE600090E080E00F94622B9B01AC0160E070E0E9
:10CE700088E492E40F9427338B019C0104C000E006
:10CE800010E020EC30E4EE24E3944B895C896D895A
:10CE90007E898F2D0E94746332E0F312D0C00E940D
:10CEA000E05481E090E0A0E0B0E00F2C04C0880FD7
:10CEB000991FAA1FBB1F0A94D2F720919F0C282B01
:10CEC00020939F0C2091B105822B8093B105898915
:10CED0009A890E94D71DF601E759FD4F608371833F
:10CEE0008283938382E0F8121AC02091E812309175
:10CEF000E9124091EA125091EB1260917102709127
:10CF0000720280917302909174020F942C3260939C
:10CF10007102709372028093730290937402F6010F
:10CF2000EB5EF74F10821182128213828F2D0E94C6
:10CF3000F41C0E94502BF601E759FD4F808191812E
:10CF4000A281B381F601E157F84F80839183A283D8
:10CF5000B38392E0F916A9F18CE0E4ECF2E0DE0193
:10CF6000119601900D928A95E1F7E1E0F0E0EC0F67
:10CF7000FD1FEC0DFD1D80809180A280B38020E01C
:10CF800030E0A901C501B4010F945D2B81111EC0D1
:10CF900066960FB6F894DEBF0FBECDBFDF91CF917E
:10CFA0001F910F91FF90EF90DF90CF90BF90AF90C7
:10CFB0009F908F907F906F905F904F903F902F90B9
:10CFC00008950E9457668111E3CFC6CF20E030E07C
:10CFD000A901C501B4010F948D3487FF04C0B7FACD
:10CFE000B094B7F8B094F601E759FD4F6F01A30173
:10CFF0009201C501B4010F94C32B9B01AC01F60152
:10D0000060817181828193810F942C32F60160835B
:10D01000718382839383F2E080E090E0A0E4B1E446
:10D02000FF1621F080E090E0A8E4B2E48D879E87AF
:10D03000AF87B88BCE010D960E94352BA9CF81E02A
:10D0400090E0A0E0B0E00F2C04C0880F991FAA1F49
:10D05000BB1F0A94D2F720919F0C282B20939F0C82
:10D060002091B105822B8093B10589899A890E940C
:10D07000D71DF601E759FD4F608371838283938347
:10D080004ECFCF93DF9300D01F92CDB7DEB780E0B5
:10D0900090E0A0EAB0E489839A83AB83BC8361E02B
:10D0A000CE0101960E9481650F900F900F900F9016
:10D0B000DF91CF9108958F929F92AF92BF92CF92BE
:10D0C000DF92EF92FF920F931F93CF93DF93CDB731
:10D0D000DEB72C970FB6F894DEBF0FBECDBF8B0125
:10D0E00040E050E068E472E44D835E836F837887AC
:10D0F00040E050E060EA70E449875A876B877C879C
:10D100008130B9F1823009F459C020E030E040E0CC
:10D1100050E460917102709172028091730290915B
:10D1200074020F942D324B017C0120E030E048EC7A
:10D1300053E40F948D34181634F4812C912C88EC20
:10D14000E82E93E4F92EF801A084B184C284D3843C
:10D150009401A701B501C6010F948D34181614F07F
:10D1600054016701C501D60189839A83AB83BC83CF
:10D1700048C0BE01675F7F4FC80108960E943965AD
:10D18000B8016C5F7F4FAE014B5F5F4FC8010E94DB
:10D1900017650E9403312C960FB6F894DEBF0FBEC0
:10D1A000CDBFDF91CF911F910F91FF90EF90DF9056
:10D1B000CF90BF90AF909F908F900895F8012085F9
:10D1C0003185428553856091710270917202809120
:10D1D0007302909174020F942D326B017C0120E058
:10D1E00030E048EC53E40F945D2B87FD06C0C12C62
:10D1F000D12C28ECE22E23E4F22EC982DA82EB82D3
:10D20000FC82BE01675F7F4FCE010196B7CFEF92E0
:10D21000FF920F931F93CF93DF937C018B010E94AA
:10D22000FD31C9E6D2E02091790230917A02409135
:10D230007B0250917C02F701608171818281938130
:10D240000F9427332C853D854E855F850F942D32B5
:10D250006C877D878E879F87C8010E94352BDF9161
:10D26000CF911F910F91FF90EF900C94DE614F9240
:10D270005F926F927F92AF92BF92CF92DF92EF92C6
:10D28000FF920F931F93CF93DF9300D000D01F9294
:10D290001F92CDB7DEB75C0180E090E0A0E7B2E47A
:10D2A00089839A83AB83BC8380E090E0A0E8B0ECF4
:10D2B0008D839E83AF83B887BE016F5F7F4FCE01A2
:10D2C00005960E94076968E873E180E090E00E949B
:10D2D0005A26C12CD12C88ECE82E81E4F82EC98284
:10D2E000DA82EB82FC8280E090E0A0E8B0E48D83FB
:10D2F0009E83AF83B887BE016F5F7F4FCE010596D7
:10D300000E94076901EA1CE0F80140AC51AC62AC34
:10D3100073ACC0AED1AEE2AEF3AE80E090E0A0E27E
:10D32000B2E489839A83AB83BC83F50180819181C8
:10D33000A281B3818D839E83AF83B887BE016F5F67
:10D340007F4FCE0105960E940769F80140AE51AEAD
:10D3500062AE73AE129A64E670E080E090E00E94E4
:10D360005A2681E028960FB6F894DEBF0FBECDBFD7
:10D37000DF91CF911F910F91FF90EF90DF90CF90B1
:10D38000BF90AF907F906F905F904F9008951F93E4
:10D39000CF93DF93CDB7DEB72C970FB6F894DEBFEF
:10D3A0000FBECDBF182F882379F020E030E0A9010F
:10D3B0006091E9057091EA058091EB059091EC058B
:10D3C0000F945D2B8823F9F08091A00C8117D9F080
:10D3D0000E94DE618CE0E0EDF2E0DE01119601904A
:10D3E0000D928A95E1F7CE0101960E94831F8091EC
:10D3F000A00C882391F089E692E00E945C271092AD
:10D40000A00C0E94502B2C960FB6F894DEBF0FBED6
:10D41000CDBFDF91CF911F91089581E08093A00C43
:10D4200089E692E00E947021ECCF2F923F924F92BA
:10D430005F926F927F928F929F92AF92BF92CF92A4
:10D44000DF92EF92FF920F931F93CF93DF93CDB7AD
:10D45000DEB7CB54D1090FB6F894DEBF0FBECDBFF7
:10D460002DB73EB739AF28AF87E00E94854E8111B6
:10D470000BC061E086E50E94A8248DA3853060F092
:10D4800087E39EE00E94A138A8ADB9AD0FB6F8942D
:10D49000BEBF0FBEADBF40C33DA1332321F087E126
:10D4A0009EE00E94A1386AE080E50E94A824182F1F
:10D4B0008CEF810F8F3218F083EF9DE0E3CF60E0B7
:10D4C00085E40E94C424882309F448C081E08FAB1E
:10D4D000E090EC12F090ED12D7012D913D914D911D
:10D4E0005C916091690270916A0280916B029091E7
:10D4F0006C020F942D32AB01BC0188E50E94162509
:10D5000069877A878B879C87F701248135814681DB
:10D51000578160916D0270916E0280916F029091BF
:10D5200070020F942D32AB01BC0189E50E941625D3
:10D530006D877E878F87988BBE01635F7F4FCE019B
:10D5400009960E94A32E382E81110BC063E68FED41
:10D550009DE00E94104087EC9DE094CF92E09FAB4D
:10D56000B7CF8CE40E94981E082F882309F431C19C
:10D570000E9494248EA3803118F080EA9DE082CF2F
:10D58000FEA1F13009F427C160E083E50E94C424C4
:10D590008AAF882321F0011102C037E03EA38DA19C
:10D5A000833020F086E89DE00E94A1389091A00C85
:10D5B0009DAF80E00E94C7690E942D1D1D8A1E8AB2
:10D5C0001F8A188E198E1A8E1B8E1C8E83EF9FE475
:10D5D000A3ECB7E48D8F9E8FAF8FB8A383EF9FE44A
:10D5E000A3ECB7EC89A39AA3ABA3BCA3A12FB0E093
:10D5F000BCA7ABA7EDB7FEB724E0129FE019F10975
:10D6000011240FB6F894FEBF0FBEEDBF8DB79EB7C5
:10D6100001969CAF8BAF2DA14FA9BE01635F7F4FD9
:10D62000CE0109960F94B51C9B01AC010F941F35D8
:10D63000811162C20E9402AA6115710581059105DE
:10D6400011F00F94E326212C1BAA1CAA1DAA1EAAC6
:10D65000AEA1A150BB0B2C96BFAFAEAF2C97E22D65
:10D66000F0E0F8A7EFA32BA53CA5E217F3070CF019
:10D6700074C23196FEA7EDA73F932F93FF93EF93CC
:10D6800082E79DE09F938F938CE79DE09F938F931C
:10D690001F920F94F11B8DB79EB709960FB6F894A1
:10D6A0009EBF0FBE8DBF9EA1992309F458C10F9450
:10D6B00094262AE030E040E050E00F94C3310F940C
:10D6C000642B20E030E040EA50E40F948D340FEFFB
:10D6D0001FEF181614F001E010E00F94942628E6CE
:10D6E00031E040E050E00F94C3310F94642B2B01E4
:10D6F0003C010F94942627E230E040E050E00F9484
:10D70000C3316B5F7F4F8F4F9F4F0F94642B4B0143
:10D710005C01ADA1A430D1F4BC01A40184E69DE07C
:10D720000E947E41B301A2018CE59DE00E947E41F2
:10D7300086E59DE00E94A1380130110519F483E4CB
:10D740000E94683882E59DE00E94A138312CC80112
:10D75000110FAA0BBB0B2A968CAF9DAFAEAFBFAF1C
:10D760002A972C96AEADBFAD2C973A161B060CF03F
:10D77000F6C02A966CAD7DAD8EAD9FAD2A970F9405
:10D78000642B6B017C01BAADBB2341F1AC019B0161
:10D790000F942D3220E030E040E952E40F94C32B87
:10D7A0009B01AC01C301B2010F942D322B013C014E
:10D7B00020E030E044EB53E40F948D341816FCF471
:10D7C00020E030E044EB53E4C301B2010F942C326B
:10D7D000EDCF1EA2D9CE22E02EA3D6CE0F94942652
:10D7E00024E130E040E050E00F94C331675E7F4FAA
:10D7F0008F4F9F4F0F94642BA7019601CFCF20E04E
:10D8000030E0A901C301B2010F945D2B87FF0BC06B
:10D8100020E030E044EB53E4C301B2010F942D3219
:10D820002B013C01ECCF0091EC121091ED12F801AC
:10D8300024813581468157816D857E858F859889C4
:10D840000F942C3222966CAF7DAF8EAF9FAF229794
:10D850002BED3FE049E450E4C301B2010F94C32B28
:10D8600020E030E044E353E40F9427336B017C0164
:10D870000F9422336FA778AB89AB9AABD8012D9167
:10D880003D914D915C9169857A858B859C850F943E
:10D890002C3226966CAF7DAF8EAF9FAF2697A50139
:10D8A00094016FA578A989A99AA90F94C32B9B010C
:10D8B000AC0126966CAD7DAD8EAD9FAD26970F94D5
:10D8C0002D3269837A838B839C83C701B6010F94C1
:10D8D000CD34A50194010F94C32B22962CAD3DAD00
:10D8E0004EAD5FAD22970F942D326D837E838F8373
:10D8F000988740E651E070E060E0CE0101960E941A
:10D90000CEC448E651E070E060E0CE0105960E948A
:10D91000CEC4BDA1B43099F449815A816B817C8118
:10D9200086E49DE00E947E414D815E816F81788515
:10D9300081EB9FE20E947E418AE00E946838198A4A
:10D940001A8A1B8A1C8AAE014F5E5F4FBE016B5F55
:10D950007F4FCE0101960E941765339402CF20E0DD
:10D960004FA9BE01635F7F4FCE0109960F94B51C8E
:10D970004B015C01312CAC019B010F941F358111CF
:10D9800002C033243394A5019401C501B4010F945E
:10D990001F358111E2C0EFA1F8A5EE0FFF1FEE0FBA
:10D9A000FF1F2BAD3CADE20FF31F80829182A2825C
:10D9B000B382A50194016D8D7E8D8F8D98A10F94FA
:10D9C0008D34181624F48D8E9E8EAF8EB8A2A501CC
:10D9D000940169A17AA18BA19CA10F945D2B87FF73
:10D9E00004C089A29AA2ABA2BCA2A50194016BA912
:10D9F0007CA98DA99EA90F942D326BAB7CAB8DAB0E
:10DA00009EABADA5BEA5BD01BB0F880B990B0F94B6
:10DA1000642B6FA378A789A79AA79B01AC016BA978
:10DA20007CA98DA99EA90F9427332B013C014D8A17
:10DA30005E8A6F8A788EEBADFCADF8ABEFA710E095
:10DA4000C12CD12C7601AFA5B8A96D917D918D9196
:10DA50009D91B8ABAFA7A30192010F942C329B010B
:10DA6000AC010F94C32B9B01AC01C701B6010F940D
:10DA70002D326B017C011F5F211628F72FA138A5DD
:10DA800049A55AA50F9427330F94DB34698F7A8FF9
:10DA90008B8F9C8FBDA1B23068F18DA59EA50E9491
:10DAA00025EA6BA57CA581E49DE00E94A0418BE363
:10DAB0009DE00E94A13843E0C501B4010E9450BD21
:10DAC00080E20E94683881E0EDA1E3300CF480E050
:10DAD000E12C8E010F5D1F4F9E01235E3F4FAE0173
:10DAE000475E5F4FBE016B5E7F4F0E945F3F8AE0E3
:10DAF0000E9468382394B3CD0E9457660E94141D7B
:10DB00008DAD0E94C7690E94033188AD99AD0FB6F3
:10DB1000F8949EBF0FBE8DBFE8ADF9AD0FB6F89477
:10DB2000FEBF0FBEEDBFC55BDF4F0FB6F894DEBF83
:10DB30000FBECDBFDF91CF911F910F91FF90EF905E
:10DB4000DF90CF90BF90AF909F908F907F906F901D
:10DB50005F904F903F902F9008950E94576633201A
:10DB600069F280E39DE00E94A13881E0FDA11F16CB
:10DB70000CF080E0EE24E3948E010F5D1F4F9E01B8
:10DB8000235E3F4FAE01475E5F4FBE016B5E7F4F2E
:10DB90000E945F3F698D7A8D8B8D9C8D005211099B
:10DBA00026E042E00F942A269F938F938FE19DE019
:10DBB0009F938F9389E29DE09F938F931F920F9481
:10DBC000F11B2DB73EB7295F3F4F0FB6F8943EBF0C
:10DBD0000FBE2DBF93CF2F923F924F925F926F92C5
:10DBE0007F928F929F92AF92BF92CF92DF92EF92ED
:10DBF000FF920F931F93CF93DF93CDB7DEB76A9752
:10DC00000FB6F894DEBF0FBECDBF83E50E94981E0D
:10DC1000182F3090A00C882319F00E94B424382EBD
:10DC20004090690250906A0260906B0270906C02A2
:10DC300080916D0290916E02A0916F02B09170027E
:10DC40008B8B9C8BAD8BBE8B8091710290917202FD
:10DC5000A0917302B09174028F8B988FA98FBA8FA5
:10DC6000112329F0311003C080E00E94C76986E5C6
:10DC70000E94981E8A8B20E030E0A9016091E9059E
:10DC80007091EA058091EB059091EC050F945D2B66
:10DC9000882309F4C9C083E40E94981E882309F4EC
:10DCA0009DC00E94EC246B017C01ABEAB7E0B98710
:10DCB000A887BF83AE83F5E0FD831D861E8628EC12
:10DCC0002F8702EC1A86212C88EC8B8792E49C87A4
:10DCD000AE81BF81B98BA88B15E0E889F989819065
:10DCE0009190A190B190F98BE88B2A85322D4B85CC
:10DCF0005C85C501B4010F945D2B87FF04C08A8643
:10DD0000292CAB86BC862D853E854F85502FC501BD
:10DD1000B4010F948D34181624F48D869E86AF8638
:10DD20000B2D1150D1F6FD81F150FD838E819F8125
:10DD300044969F838E83F111CBCF2D853E854F85F1
:10DD4000502F6A85722D8B859C850F942D3220E093
:10DD500030E040E05FE30F94C32BA70196010F94DE
:10DD60002D324B015C012DEB37E346E855EB0F9468
:10DD70008D3487FD0AC02DEB37E346E855E3C50136
:10DD8000B4010F945D2B18164CF580E00E94C76912
:10DD900010E0E884F98400E0D7016D917D918D91C8
:10DDA0009D917D016D01B4E0CB1AD108A5019401CC
:10DDB0000F942C32F6016083718382839383602FEA
:10DDC000812F0F94C61A0F5F053031F71F5F8885CA
:10DDD00099854496998788871530D9F6AA89AA2308
:10DDE00081F020E030E0A9016091E9057091EA0539
:10DDF0008091EB059091EC050F945D2B81110E94B1
:10DE0000E7408AE50E94981E882351F00E94EC2486
:10DE100069837A838B839C83CE0101960F948E193C
:10DE2000832D0E94C7690BC0311003C09A899923C2
:10DE300041F30E94754E80E69CE00E94A138332099
:10DE400051F08091A00C811106C00E94714E81E4B6
:10DE50009CE00E94A1380E94754E83E39CE00E94E2
:10DE6000A1388091A00C0E9460410E94754E86E20C
:10DE70009CE00E94A138C090E708D090E808E090AC
:10DE8000E908F090EA0820E030E0A901C701B601F6
:10DE90000F948D3418160CF053C042E0C701B60140
:10DEA0000E9450BD8DE00E9468388AE00E94683868
:10DEB000A30192016091690270916A0280916B02E4
:10DEC00090916C020F945D2B81111FC02B893C89AE
:10DED0004D895E8960916D0270916E0280916F0232
:10DEE000909170020F945D2B81110FC02F89388D96
:10DEF000498D5A8D60917102709172028091730206
:10DF0000909174020F945D2B81110E9403316A96E7
:10DF10000FB6F894DEBF0FBECDBFDF91CF911F913A
:10DF20000F91FF90EF90DF90CF90BF90AF909F90B8
:10DF30008F907F906F905F904F903F902F900895BB
:10DF400081E29CE00E94A138B3CF8F929F92AF9262
:10DF5000BF92EF92FF920F931F93CF93DF9380E0D6
:10DF60000E94C7691092E5051092E6051092E70538
:10DF70001092E8051092E1051092E2051092E30577
:10DF80001092E4051092ED051092EE051092EF0547
:10DF90001092F0051092E9051092EA051092EB0537
:10DFA0001092EC050BEA17E0C0E0812C912C80EC7C
:10DFB000A82E8FE7B82E7801D0E0F70181929192D8
:10DFC000A192B1927F016D2F8C2F0F94C61ADF5F43
:10DFD000D53099F7CF5F0C5E1F4FC53061F7DF91E9
:10DFE000CF911F910F91FF90EF90BF90AF909F90B6
:10DFF0008F9008959091F1128091F212981308C0B9
:10E000008091230990912409892B11F40C94521FBB
:10E0100080E00E94745AEECF83E50E94E61E8823BA
:10E02000E9F00E9402AA6093DE117093DF118093E1
:10E03000E0119093E1110E94EC2420E030E04AE7E7
:10E0400054E40F94C32B0F94A03360931302709386
:10E05000140280931502909316020895809147054B
:10E0600084FD0AC08091490587FD06C080914A055C
:10E07000837011F40C94FA6F0E94DE6188E50E94AF
:10E08000981E882331F05F9A80919F0C8E7F809339
:10E090009F0C89E50E94981E882331F08A9A80910E
:10E0A0009F0C8D7F80939F0C8AE50E94981E882389
:10E0B00059F08091080180958170809306018091CC
:10E0C0009F0C8B7F80939F0C85E40E94981E81118A
:10E0D0000C94501F08952F923F924F925F926F922F
:10E0E0007F928F929F92AF92BF92CF92DF92EF92E8
:10E0F000FF920F931F93CF93DF93CDB7DEB7A69711
:10E100000FB6F894DEBF0FBECDBF8FE897E00E9438
:10E110007D2A80915D0C83FD7EC020917502309137
:10E120007602409177025091780260919B0770913E
:10E130009C0780919D0790919E070F945D2B8823EB
:10E1400009F469C010912209111161C08091670220
:10E150009091680201972091531230915412281720
:10E1600039073CF40E94754E84E599E10E94A1387C
:10E1700011E0209175023091760240917702509122
:10E18000780260919B0770919C0780919D07909108
:10E190009E070F942C326B017C0120E030E0A90136
:10E1A0000F948D3487FF04C0F7FAF094F7F8F094D9
:10E1B0002091790230917A0240917B0250917C0249
:10E1C000C701B6010F94C32B20E030E84BE354E4C1
:10E1D0000F948D341816ECF40E94754E85E399E186
:10E1E0000E94A13880919B0790919C07A0919D0768
:10E1F000B0919E078093750290937602A093770268
:10E20000B09378028BE997E00E94EF6104C010E0C0
:10E21000B0CF1111E7CF2AE037ED43E25CE3609124
:10E22000490270914A0280914B0290914C020F94E6
:10E23000C32B6B017C0160917F0270918002072EDD
:10E24000000C880B990B0F94642B9B01AC01C70148
:10E25000B6010F94C32B698B7A8B8B8B9C8B80912F
:10E26000A00C882309F18090E7089090E808A0901E
:10E27000E908B090EA08C0909707D0909807E0901E
:10E280009907F0909A0720E030E0A901C501B40198
:10E290000F945D2B8823D1F1A7019601C501B4012C
:10E2A0000F948D34181694F1C12CD12C76018E0167
:10E2B0000F5E1F4F2BE937E047E957E063E977E04E
:10E2C0008FE897E00F94680080E1EFE8F7E0A9E6B7
:10E2D000B2E001900D928A95E1F7A6960FB6F894F8
:10E2E000DEBF0FBECDBFDF91CF911F910F91FF9089
:10E2F000EF90DF90CF90BF90AF909F908F907F90E6
:10E300006F905F904F903F902F90089520916902F9
:10E3100030916A0240916B0250916C0260918F07BC
:10E320007091900780919107909192070F942C32F1
:10E330006D8B7E8B8F8B988F20916D0230916E024A
:10E3400040916F0250917002609193077091940711
:10E3500080919507909196070F942C32698F7A8F50
:10E360008B8F9C8F209171023091720240917302C9
:10E3700050917402C701B6010F942C326D8F7E8FBD
:10E380008F8F98A320917502309176024091770289
:10E390005091780260919B0770919C0780919D0736
:10E3A00090919E070F942C326B017C0120E030E0AD
:10E3B000A9016D897E898F89988D0F945D2B8111BC
:10E3C0000CC020E030E0A901698D7A8D8B8D9C8D89
:10E3D0000F945D2B882309F467CF2D893E894F89DF
:10E3E000588DCA01B9010F94C32B4B015C01298DD3
:10E3F0003A8D4B8D5C8DCA01B9010F94C32B9B01E3
:10E40000AC01C501B4010F942D324B015C012D8D7F
:10E410003E8D4F8D58A1CA01B9010F94C32B9B01AA
:10E42000AC01C501B4010F942D324B015C01A70171
:10E430009601C701B6010F94C32B9B01AC01C50126
:10E44000B4010F942D320F94DB344B015C012DEBA2
:10E4500037E346E855E30F945D2B87FF0FC020E0BC
:10E4600030E0A901C701B6010F948D344601570170
:10E4700087FF04C0B7FAB094B7F8B0942DEB37E338
:10E4800046E855E3C501B4010F945D2B87FD1CCF11
:10E4900020E030E040EA51E4C501B4010F94273395
:10E4A0000F94A0331B01672B19F422242394312CE1
:10E4B000B10190E080E00F94622B9B01AC0160E021
:10E4C00070E080E89FE30F9427332B013C01AC01FF
:10E4D0009B01C501B4010F94C32B4B015C01A30147
:10E4E00092016D897E898F89988D0F94C32B6D8BD6
:10E4F0007E8B8F8B988FA3019201698D7A8D8B8D86
:10E500009C8D0F94C32B698F7A8F8B8F9C8FA30167
:10E5100092016D8D7E8D8F8D98A10F94C32B6D8F81
:10E520007E8F8F8F98A3A3019201C701B6010F942C
:10E53000C32B69A37AA38BA39CA380E1E9E6F2E055
:10E540008E010F5F1F4FD80101900D928A95E1F760
:10E550000E9402AA2B013C0128EC420E511C611CB6
:10E56000711C0DA31EA381E0281A310809F460C0B4
:10E570000E9402AA8B019C0104191509260937097A
:10E5800037FD59C02B013C0128EC420E511C611C87
:10E59000711C80E00E94745A2D893E894F89588DE4
:10E5A00069817A818B819C810F942D3269837A8372
:10E5B0008B839C83298D3A8D4B8D5C8D6D817E8103
:10E5C0008F8198850F942D326D837E838F839887FA
:10E5D0002D8D3E8D4F8D58A169857A858B859C85C3
:10E5E0000F942D3269877A878B879C8729A13AA15E
:10E5F0004BA15CA16D857E858F8598890F942D3206
:10E600006D877E878F87988B750164018E010F5E01
:10E610001F4F9E01235F3F4FAE01475F5F4FBE011B
:10E620006B5F7F4F8DA19EA10F94680081119BCFDE
:10E63000750164013CCE0E9410C5AECF8F929F92AF
:10E64000AF92BF92CF92DF92EF92FF92CF93DF9380
:10E650008090490290904A02A0904B02B0904C02E8
:10E66000FC01C080D180E280F38020E030E0A9018D
:10E67000C701B6010F945D2B882341F0C092490277
:10E68000D0924A02E0924B02F0924C02C0917F027B
:10E69000D091800284E690E09093800280937F0284
:10E6A000C0907902D0907A02E0907B02F0907C02D8
:10E6B00080E090E0A0E8BFE38093790290937A0233
:10E6C000A0937B02B0937C020E946B7080924902FF
:10E6D00090924A02A0924B02B0924C02D0938002D8
:10E6E000C0937F02C0927902D0927A02E0927B02BC
:10E6F000F0927C02DF91CF91FF90EF90DF90CF906E
:10E70000BF90AF909F908F9008950F931F93CF93DA
:10E71000DF9300D01F92CDB7DEB79C010FE817E062
:10E7200090E1E9E6F2E0D80101900D929A95E1F7C7
:10E73000F9012081318142815381F8016085718521
:10E74000828593850F942D32F801608771878287C7
:10E75000938780E090E0A0EAB0E489839A83AB835A
:10E76000BC83CE0101960E941E730F900F900F90F4
:10E770000F90DF91CF911F910F9108952F923F92AB
:10E780004F925F926F927F928F929F92AF92BF92C1
:10E79000CF92DF92EF92FF921F93CF93DF93CDB78B
:10E7A000DEB72C970FB6F894DEBF0FBECDBF7A014F
:10E7B0001901DC012D913D914D915C912D833E839A
:10E7C0004F835887FB014080518062807380809026
:10E7D000690290906A02A0906B02B0906C02A50151
:10E7E00094016D817E818F8198850F945D2B8111BD
:10E7F0000EC011E0A301920160916D0270916E0252
:10E8000080916F02909170020F945D2B811110E046
:10E81000D1012D913D914D915C9129873A874B878C
:10E820005C87F701C080D180E280F38020910B02E9
:10E8300030910C0240910D0250910E02C701B601B9
:10E840000F945D2B882309F44EC0C0920B02D09226
:10E850000C02E0920D02F0920E02809175029091EE
:10E860007602A0917702B091780240916D025091AA
:10E870006E0260916F027091700280928F07909289
:10E880009007A0929107B0929207409393075093FC
:10E8900094076093950770939607C0929707D0925C
:10E8A0009807E0929907F0929A0780939B079093BC
:10E8B0009C07A0939D07B0939E0720E030E040E0C6
:10E8C0005FE36091CD0C7091CE0C8091CF0C909154
:10E8D000D00C0F94C32B69837A838B839C83CE01E6
:10E8E00001960E941E732D813E814F815885209391
:10E8F0008F0730939007409391075093920740926F
:10E900009307509294076092950770929607D101F1
:10E910002D913D914D915C9160919B0770919C0769
:10E9200080919D0790919E070F942D3260939B07D5
:10E9300070939C0780939D0790939E0711112FC0A1
:10E9400020E030E0A90169857A858B859C850F944C
:10E950005D2B811133C060E070E088EC92E4698344
:10E960007A838B839C83CE0101960E941E732C9622
:10E970000FB6F894DEBF0FBECDBFDF91CF911F91D0
:10E98000FF90EF90DF90CF90BF90AF909F908F90CF
:10E990007F906F905F904F903F902F9008952AEF57
:10E9A0003EE74AE25FE36091D10C7091D20C809116
:10E9B000D30C9091D40C0F94C32BD1CF60E070E0B6
:10E9C00080EA91E4CCCF0F931F93CF93DF9300D0D5
:10E9D00000D01F921F92CDB7DEB78B01FC0123A59B
:10E9E000211102C00F94A21E1D821E821F82188652
:10E9F00020E030E040E05FE36091710270917202CC
:10EA000080917302909174020F942D3269837A83FE
:10EA10008B839C839E012B5F3F4FAE014F5F5F4F07
:10EA20006DE672E089E692E00E94BE731D821E824E
:10EA30001F82188620E030E040E05FE3F801608547
:10EA40007185828593850F942D3269837A838B83B8
:10EA50009C83B8016C5F7F4F9E012B5F3F4FAE01DF
:10EA60004F5F5F4FC8010E94BE7328960FB6F8949F
:10EA7000DEBF0FBECDBFDF91CF911F910F910895E3
:10EA80009B01AC01485F5F4FBC016C5F7F4F0C94F2
:10EA9000BE732F923F924F925F926F927F928F92AE
:10EAA0009F92AF92BF92CF92DF92EF92FF920F931D
:10EAB0001F93CF93DF93CDB7DEB7A6970FB6F89429
:10EAC000DEBF0FBECDBF8C011B015A874987409026
:10EAD000690250906A0260906B0270906C028090A4
:10EAE0006D0290906E02A0906F02B0907002DB01F8
:10EAF0008D919D910D90BC91A02D8B8B9C8BAD8B9E
:10EB0000BE8B9C01AD01C301B2010F942C326B018D
:10EB10007C01D10114968D919D910D90BC91A02DF9
:10EB20008F8B988FA98FBA8F9C01AD01C501B4015D
:10EB30000F942C326B8F7C8F8D8F9E8FA985BA8519
:10EB40008D919D910D90BC91A02D8B879C87AD8759
:10EB5000BE879C01AD01C301B2010F942C326F8FAF
:10EB600078A389A39AA3A985BA8514968D919D91BE
:10EB70000D90BC91A02D8F87988BA98BBA8B9C018F
:10EB8000AD01C501B4010F942C326BA37CA38DA3FE
:10EB90009EA3A7019601C701B6010F94C32B6B0179
:10EBA0007C012B8D3C8D4D8D5E8DCA01B9010F947A
:10EBB000C32B9B01AC01C701B6010F942D324B0151
:10EBC0005C012B893C894D895E896B857C858D85AF
:10EBD0009E850F942C322B013C012F89388D498D55
:10EBE0005A8D6F85788989899A890F942C326B01A7
:10EBF0007C01A3019201C301B2010F94C32B2B012D
:10EC00003C01A7019601C701B6010F94C32B9B01DC
:10EC1000AC01C301B2010F942D320F94DB346B01B0
:10EC20007C012F8D38A149A15AA1CA01B9010F94C5
:10EC3000C32B2B013C012BA13CA14DA15EA1CA011C
:10EC4000B9010F94C32B9B01AC01C301B2010F9416
:10EC50002D329B01AC01C501B4010F948D341816FF
:10EC6000B4F520E030E0A901C701B6010F948D345E
:10EC700087FF2AC0C701B601905820E030E040EA83
:10EC800050E40F948D34181614F5A10169857A8526
:10EC9000C8010E944975A6960FB6F894DEBF0FBE54
:10ECA000CDBFDF91CF911F910F91FF90EF90DF903B
:10ECB000CF90BF90AF909F908F907F906F905F901C
:10ECC0004F903F902F900895C701B601D6CF20E016
:10ECD00030E040E050E4C501B4010F948D341816C3
:10ECE00024F4B101C8010E94E37419821A821B82C4
:10ECF0001C82BE016F5F7F4FC1010E9440752DECE9
:10ED00003CEC4CEC5CE3C701B6010F94C32B9B01B8
:10ED1000AC01F80160817181828193810F94C32BD2
:10ED20006D837E838F839887D8019B968C919B9768
:10ED30008823C9F02AE939E949E95FE314966D911E
:10ED40007D918D919C9117970F94C32B69837A8342
:10ED50008B839C83BE016F5F7F4F8FE897E00E949B
:10ED60004075F80113A6BE016B5F7F4F89859A85B8
:10ED70000E94407590CF3F924F925F926F927F9228
:10ED80008F929F92AF92BF92CF92DF92EF92FF92BB
:10ED90000F931F93CF93DF93CDB7DEB76C970FB66A
:10EDA000F894DEBF0FBECDBFDB010C91142F100F06
:10EDB000153008F067C11196DC90C22ECD0CB4E07E
:10EDC000BC1508F45FC1ED2DF0E0E25FFA4F8080E2
:10EDD000912CB12CA12C002E04C0B694A79497942A
:10EDE00087940A94D2F780FE4DC1EC2DF0E0E25FEB
:10EDF000FA4F8080912CB12CA12C012E04C0B69426
:10EE0000A794979487940A94D2F780FE3BC1322E40
:10EE1000642F7C014090E1055090E2056090E3058D
:10EE20007090E4058091E9059091EA05A091EB05C9
:10EE3000B091EC05898F9A8FAB8FBC8F660F770BE3
:10EE4000072E000C880B990B0F94642B4B015C016F
:10EE5000602F000F770B880B990B0F94642B298D73
:10EE60003A8D4B8D5C8D0F94C32BA30192010F94AF
:10EE70002D32A50194010F942D326D877E878F87E7
:10EE8000988B612F110F770B880B990B0F94642BC4
:10EE9000298D3A8D4B8D5C8D0F94C32BA30192016C
:10EEA0000F942D32A50194010F942C3269837A833B
:10EEB0008B839C834090E5055090E6056090E705C4
:10EEC0007090E8058091ED059091EE05A091EF0519
:10EED000B091F005898F9A8FAB8FBC8F632D660F31
:10EEE000770B072E000C880B990B0F94642B4B01AA
:10EEF0005C016D2DDD0C770B880B990B0F94642B47
:10EF0000298D3A8D4B8D5C8D0F94C32BA3019201FB
:10EF10000F942D32A50194010F942D32698B7A8BB9
:10EF20008B8B9C8B6C2DCC0C770B880B990B0F94D7
:10EF3000642B298D3A8D4B8D5C8D0F94C32BA301CF
:10EF400092010F942D32A50194010F942C326D8300
:10EF50007E838F839887F70180859185A285B3850D
:10EF600089879A87AB87BC878D8B9E8BAF8BB88F39
:10EF700047E651E061E070E0CE0141960E94CEC4C8
:10EF800047E651E061E070E0CE0105960E94CEC4F4
:10EF90004FE551E061E070E0CE010D960E94CEC4D5
:10EFA0004FE551E061E070E0CE0101960E94CEC4D1
:10EFB00089889A88AB88BC8827E137EB41ED58EB0C
:10EFC000C501B4010F948D3487FD5CC023E030E0AF
:10EFD00044EB53E4C501B4010F945D2B18160CF4F7
:10EFE00051C08D849E84AF84B88827E137EB41ED12
:10EFF00058EBC501B4010F948D3487FD43C023E065
:10F0000030E040EB53E4C501B4010F945D2B1816BA
:10F01000CCF18D809E80AF80B88427E137EB41ED45
:10F0200058EBC501B4010F948D3487FD2BC023E04C
:10F0300030E044EB53E4C501B4010F945D2B181686
:10F040000CF189809A80AB80BC8027E137EB41EDE1
:10F0500058EBC501B4010F948D3487FD13C023E034
:10F0600030E040EB53E4C501B4010F945D2B18165A
:10F070004CF0AE014F5F5F4FBE01635F7F4FC70132
:10F080000E9449756C960FB6F894DEBF0FBECDBFD7
:10F09000DF91CF911F910F91FF90EF90DF90CF9074
:10F0A000BF90AF909F908F907F906F905F904F90A8
:10F0B0003F9008952F923F924F925F926F927F926E
:10F0C0008F929F92AF92BF92CF92DF92EF92FF9278
:10F0D0000F931F93CF93DF93CDB7DEB7CC58D109F1
:10F0E0000FB6F894DEBF0FBECDBF80E19CE00E945A
:10F0F000A13887E00E94854E81116EC084E50E9490
:10F10000E61E882329F00E94D92481110E943EBD69
:10F1100080E090E0A0E8BFE389839A83AB83BC835F
:10F120008D839E83AF83B8878DEC9CECACE4BEE30B
:10F1300089879A87AB87BC8780E090E0A0E2B1E442
:10F140008D879E87AF87B88B8CE390E09A8B898BF5
:10F150008DEC90E09C8B8B8B8DEC9CECACECBEE34F
:10F160008D8B9E8BAF8BB88F80E090E0A0EEBFE3DD
:10F17000898F9A8FAB8FBC8F1BA61CA64AE959E9D1
:10F1800069E97EE38FE40E9416256D8F7E8F8F8F55
:10F1900098A360E083E40E94C42489A360E08BE428
:10F1A0000E94C4248AA382E40E94E61E882381F17F
:10F1B0000E94D924009761F19C012852310925361B
:10F1C000310520F16CE870E082EE9BE00E94A041E6
:10F1D0008DED9BE00E94A138C457DF4F0FB6F89425
:10F1E000DEBF0FBECDBFDF91CF911F910F91FF907A
:10F1F000EF90DF90CF90BF90AF909F908F907F90D7
:10F200006F905F904F903F902F9008959A8B898BCD
:10F210008CE40E94E61E8823E1F00E94EC246B013E
:10F220007C01C986DA86EB86FC8620E030E0A90105
:10F230000F948D3487FD0AC020E030E040E050E4B8
:10F24000C701B6010F945D2B18161CF485EB9BE0EB
:10F25000C1CF81E50E94981E882331F18091170566
:10F2600090911805892BE9F00E94EC246B017C0138
:10F27000CD82DE82EF82F8862DEC3CEC4CE45DE33F
:10F280000F948D3487FD0AC020E030E040E751E460
:10F29000C701B6010F945D2B181634F484E89BE087
:10F2A00099CF89E59BE096CF83E50E94E61E8823EF
:10F2B000E9F00E94EC246B017C01CD8ADE8AEF8AA2
:10F2C000F88E2DEC3CEC4CEC5DE30F948D3487FD17
:10F2D0000AC020E030E040E050E4C701B6010F94DE
:10F2E0005D2B18161CF482E39BE074CF80E50E942E
:10F2F000981E882341F18091170590911805892B5C
:10F3000019F48AEF9AE066CF8BA58F5F8BA70E94D6
:10F31000EC246B017C01CD86DE86EF86F88A20E046
:10F3200030E0A9010F948D3487FD0AC020E030E061
:10F3300048EC51E4C701B6010F945D2B18161CF47C
:10F3400082ED9AE047CF86E40E94E61E8823E9F02A
:10F350000E94EC246B017C01C98EDA8EEB8EFC8E50
:10F3600020E030E040E85FE30F948D3487FD0AC071
:10F3700020E030E040E850E4C701B6010F945D2B77
:10F3800018161CF489EA9AE025CFC98CDA8CEB8C2C
:10F39000FC8C8D889E88AF88B88CA7019601C70128
:10F3A000B6010F94C32B9B01AC0160E070E084E4D4
:10F3B00090E40F94273329813A814B815C810F942B
:10F3C000C32B2B013C01A5019401C501B4010F948D
:10F3D000C32BA70196010F94C32B2CEE31E548EB0C
:10F3E0005DE30F9427339B01AC01C301B2010F947D
:10F3F000C32B69837A838B839C8388E40E94E61EF7
:10F40000882379F00E94D924009759F09C01255A4D
:10F4100031092838310518F08BE79AE0DBCE9C8B58
:10F420008B8B85E50E94981E8823C9F00E9402AA52
:10F43000611571058105910511F00F94E326809106
:10F44000170590911805892B91F00E94EC24609388
:10F45000130570931405809315059093160582E5A6
:10F460000E94981E811108C087E49AE0B3CE60E044
:10F4700070E088E492E4EBCF809117059091180535
:10F48000892B61F00E94D924AD969FAF8EAFAD97C6
:10F49000181619064CF083E19AE09CCE2AE130E080
:10F4A000AD963FAF2EAFAD9789E50E94E61E88234B
:10F4B00081F10E94EC242091EF083091F0084091F6
:10F4C000F1085091F2080F942C326B017C0188E511
:10F4D0000E94E61E882331F10E94EC242091EB0863
:10F4E0003091EC084091ED085091EE080F942C32C9
:10F4F0006BA37CA38DA39EA3CFA2D8A6E9A6FAA650
:10F50000CE0183960E94571E811115C089EE99E0A5
:10F5100061CEC0906D02D0906E02E0906F02F090CC
:10F520007002D5CF6091690270916A0280916B027E
:10F5300090916C02DDCF84E40E94981E91E08927AF
:10F540000E94C76980E090E0A0EAB0E48DA79EA782
:10F55000AFA7B8AB60E0CE018D960E948165309177
:10F560001408CD57DF4F3883C358D0401092140889
:10F570000E94511C88EC99E00E94A13889899A89DF
:10F580008A3191050CF044C08B899C890E946E1FC2
:10F5900061E080E00E94DEBF811142C06FEF8DED1F
:10F5A00099E00E9410408CA5811104C0CE01019603
:10F5B0000F94A21E80E090E0A0EAB0E48093970749
:10F5C00090939807A0939907B0939A071DA61EA63B
:10F5D0001FA618AABE01635D7F4F8FE897E00E94C7
:10F5E0004075CD57DF4F5881C358D0405093140811
:10F5F0000E94511C8AA18111EFCD1092EB11109243
:10F60000EA110E9496C190E080E00E946E1FE4CD56
:10F610000E94AC2281E00E9467BE8111B5CFBECFAF
:10F620001092750210927602109277021092780270
:10F6300085E792E00E94EF618BA5882309F452C010
:10F6400020E030E040E751E46091D10C7091D20CA1
:10F650008091D30C9091D40C0F9427336DA77EA783
:10F660008FA798AB80E1E9E6F2E0AFE8B7E0019060
:10F670000D928A95E1F72D853E854F8558896091D9
:10F680009B0770919C0780919D0790919E070F9416
:10F690002D3260939B0770939C0780939D079093F6
:10F6A0009E07CE018D960E941E732D853E854F8547
:10F6B000588960919B0770919C0780919D0790915C
:10F6C0009E070F942C3260939B0770939C07809346
:10F6D0009D0790939E078CA5811104C0CE010196D1
:10F6E0000F94A21EEEE0F5E085E0DF011D928A9501
:10F6F000E9F780E1E9E6F2E0AFE8B7E001900D92CA
:10F700008A95E1F789859A85AB85BC8580939707B3
:10F7100090939807A0939907B0939A071DA61EA6E9
:10F720001FA618AABE01635D7F4F8FE897E00E9475
:10F730004075BE01635E7F4F8FE897E00E94407581
:10F7400089A1882309F41CC42091690230916A02BE
:10F7500040916B0250916C02E5962CAF3DAF4EAFDD
:10F760005FAFE59780916D0290916E02A0916F025C
:10F77000B0917002E1968CAF9DAFAEAFBFAFE19795
:10F78000312C212C9FEFA4969FAFA497AFEFA896A2
:10F79000AFAFA897BFEFC158DF4FB883CF57D04066
:10F7A000EFE4C058DF4FE883C058D040F3ECCF57A8
:10F7B000DF4FF883C158D04027E4CE57DF4F28836E
:10F7C000C258D04081E090E0A0E0B0E0022C04C03C
:10F7D000880F991FAA1FBB1F0A94D2F7CC57DF4F7F
:10F7E00088839983AA83BB83C458D040AEE0B5E038
:10F7F000E796BFAFAEAFE79710E000E09101032CB2
:10F80000000C440B550BC857DF4F288339834A83BC
:10F810005B83C858D040C457DF4F2882CC58D040B3
:10F82000E796AEADBFADE7978D91E796BFAFAEAFB0
:10F83000E79790E0B0E0A0E0CC57DF4F2881398116
:10F840004A815B81C458D04082239323A423B523EB
:10F85000892B8A2B8B2B09F024C1C857DF4F688175
:10F8600079818A819B81C858D0400F94642B209164
:10F87000E9053091EA054091EB055091EC050F94B4
:10F88000C32B2091E1053091E2054091E3055091B1
:10F89000E4050F942D32EB966CAF7DAF8EAF9FAF2A
:10F8A000EB97B801012E000C880B990B0F94642B79
:10F8B0002091ED053091EE054091EF055091F00556
:10F8C0000F94C32B2091E5053091E6054091E705A3
:10F8D0005091E8050F942D326B017C01EB962CAD15
:10F8E0003DAD4EAD5FADEB97E5966CAD7DAD8EADAC
:10F8F0009FADE5970F942C322B013C01A701960197
:10F90000E1966CAD7DAD8EAD9FADE1970F942C323D
:10F910004B015C01A3019201C301B2010F94C32BFF
:10F920002B013C01A5019401C501B4010F94C32B27
:10F930009B01AC01C301B2010F942D320F94DB3453
:10F940004B015C01EB962CAD3DAD4EAD5FADEB9741
:10F950006BA17CA18DA19EA10F942C322B013C01A7
:10F96000A70196016FA178A589A59AA50F942C32BD
:10F970006B017C01A3019201C301B2010F94C32B5F
:10F980002B013C01A7019601C701B6010F94C32BBF
:10F990009B01AC01C301B2010F942D320F94DB34F3
:10F9A00020E030E040E751E40F942733A5019401B3
:10F9B0000F942D326B017C018090130590901405FB
:10F9C000A0901505B090160520E030E040E85FE318
:10F9D000C501B4010F948D341816F4F4C501B401B7
:10F9E0000F9499334B015C0160E070E0CB01181477
:10F9F00019041A041B0434F40F949426A5019401ED
:10FA00000F94C3310F94642B9B01AC01B601C70165
:10FA10000F942D326B017C01C158DF4F2881CF57E5
:10FA2000D040C058DF4F3881C058D040CF57DF4F4B
:10FA30004881C158D040CE57DF4F5881C258D0407E
:10FA4000B601C7010F945D2B87FF2BC0A4960FAFA3
:10FA5000A497C457DF4F3881CC58D040A8963FAF09
:10FA6000A897EC96CFAEEC97ED96DFAEED97EE96BD
:10FA7000EFAEEE97EF96FFAEEF97C158DF4FC8821B
:10FA8000CF57D040C058DF4FD882C058D040CF5752
:10FA9000DF4FE882C158D040CE57DF4FF882C258BE
:10FAA000D0400F5F1F4F0530110509F0B9CE4FEF61
:10FAB000241A340A55E02516310409F083CEA496A1
:10FAC0008FADA497E82FF0E0E25FFA4F208181E04C
:10FAD00090E0A0E0B0E0A8960FACA89704C0880F13
:10FAE000991FAA1FBB1F0A94D2F7822B8083A89666
:10FAF0009FADA8976A969FAF6A97A496AFADA4975B
:10FB00006B96AFAF6B97EC968FADEC97ED969FAD84
:10FB1000ED97EE96AFADEE97EF96BFADEF976F9680
:10FB20008CAF9DAFAEAFBFAF6F97A896BFADA89794
:10FB3000BF3F09F409C2A496EFADA497EF3F09F4C3
:10FB400003C26B2FBB0F770B880B990B0F94642BA1
:10FB50002091E9053091EA054091EB055091EC05C3
:10FB60000F94C32B2091E1053091E2054091E3050C
:10FB70005091E4050F942D32162F072F382E292E81
:10FB8000862F902FA32DB22D65968CAF9DAFAEAF73
:10FB9000BFAF6597A496FFADA4976F2FFF0F770BAC
:10FBA000880B990B0F94642B2091ED053091EE0595
:10FBB0004091EF055091F0050F94C32B2091E5057E
:10FBC0003091E6054091E7055091E8050F942D32FC
:10FBD0006B017C016996CCAEDDAEEEAEFFAE6997EF
:10FBE000CE018F5A9F4F0E94571E882309F4B0C13F
:10FBF00020E030E040EA50E4612F702F832D922DF9
:10FC00000F942D324B015C01CB01D50121968CAFB5
:10FC10009DAFAEAFBFAF21972596CCAEDDAEEEAEB9
:10FC2000FFAE2597A8962FADA8972111E3C1A49602
:10FC30003FADA4973111B3C120E030E040EA50E479
:10FC4000C701B6010F942D326B017C01A4964FAD14
:10FC5000A497442309F4C5C1A4968FADA49784301A
:10FC60000CF0BFC122ED422E23E5522E2BE7622E6F
:10FC700021E4722E21968CAC9DACAEACBFAC21972A
:10FC800025968CAD9DADAEADBFAD2597A7968CAF3B
:10FC90009DAFAEAFBFAFA7979C01AD0169966CADAC
:10FCA0007DAD8EAD9FAD69970F942C32AB966CAF46
:10FCB0007DAF8EAF9FAFAB97A501940165966CADFC
:10FCC0007DAD8EAD9FAD65970F942C322D966CAFA8
:10FCD0007DAF8EAF9FAF2D97AB962CAD3DAD4EADAA
:10FCE0005FADAB9761962CAF3DAF4EAF5FAF619705
:10FCF000A50194016091690270916A0280916B0282
:10FD000090916C020F942C324B015C01A7962CADA4
:10FD10003DAD4EAD5FADA79760916D0270916E02E3
:10FD200080916F02909170020F942C32A7966CAF65
:10FD30007DAF8EAF9FAFA797812F902FA32DB22DB0
:10FD40008DA79EA7AFA7B8ABC9AADAAAEBAAFCAA4F
:10FD5000C984DA84EB84FC84CDAADEAAEFAAF8AECB
:10FD60002DEC3CEC4CEC5CE3C301B2010F94C32BD3
:10FD700029813A814B815C810F94C32B20917502BC
:10FD80003091760240917702509178020F942D3293
:10FD900069AF7AAF8BAF9CAFA5019401C501B401E7
:10FDA0000F94C32B4B015C01A7962CAD3DAD4EAD1E
:10FDB0005FADA797CA01B9010F94C32B9B01AC019A
:10FDC000C501B4010F942D3220E030E040E050E452
:10FDD0000F948D341816ACF420E030E040E05FE37F
:10FDE000C701B6010F942D3229966CAF7DAF8EAF4F
:10FDF0009FAF2997BE01635C7F4FCE0101960E94A1
:10FE0000E37489859A85AB85BC8529968CAF9DAFB7
:10FE1000AEAFBFAF2997A3961CAE1DAE1EAE1FAEF0
:10FE2000A397BE01615A7F4FCE01CD960E944075C7
:10FE30008CA58823C1F02AE939E949E95FE36D819E
:10FE40007E818F8198850F94C32BA3966CAF7DAF75
:10FE50008EAF9FAFA397BE01615A7F4F8FE897E0A7
:10FE60000E9440751CA6E090C90CF090CA0C00914D
:10FE7000CB0C1091CC0CA090C50CB090C60CC090CF
:10FE8000C70CD090C80C9501A601B701C8010F940A
:10FE90008D34181614F475018601809049029090F3
:10FEA0004A02A0904B02B0904C022DEC3CEC4CEC82
:10FEB0005DE3B701C8010F94C32B609349027093AF
:10FEC0004A0280934B0290934C0240E0BE01675B74
:10FED0007F4FCE018D960E9450C980E1E9E6F2E0A5
:10FEE000AFE8B7E001900D928A95E1F78092490260
:10FEF00090924A02A0924B02B0924C0220E04FEF47
:10FF0000BE01675A7F4FCE0101960E94BB7620E06A
:10FF100041E0BE01675A7F4FCE0101960E94BB7639
:10FF20002FEF40E0BE01675A7F4FCE0101960E943D
:10FF3000BB7621E040E0BE01675A7F4FCE010196BB
:10FF40000E94BB760E94DE6180910C0D80930D0DA6
:10FF5000AD964EAD5FADAD9741505109AD965FAFD7
:10FF60004EAFAD97452B09F419CB6A968FAD6A97C2
:10FF700087FD14CB6B968FAD6B9787FFE1CB0ECBD4
:10FF80002BA13CA14DA15EA1E5962CAF3DAF4EAF9C
:10FF90005FAFE5978FA198A5A9A5BAA5EBCB812F57
:10FFA000902FA32DB22D21968CAF9DAFAEAFBFAFDA
:10FFB000219720E030E040EA50E4C701B6010F94F9
:10FFC0002C3225966CAF7DAF8EAF9FAF2597A49650
:10FFD0005FADA49754300CF42FCE182D092D3A2C78
:10FFE0002B2C92ED492E93E5592E9BEF692E90E430
:10FFF000792E40CEA8969FADA89794300CF452C0AD
:020000021000EC
:10000000A496AFADA497A4300CF120E030E040EA14
:1000100050E4612F702F832D922D0F942C32219656
:100020006CAF7DAF8EAF9FAF219720E030E040EA0C
:1000300050E4C701B6010F942C326B017C01A496E9
:10004000EFADA497E4300CF40DCECBCF812F902FE1
:10005000A32DB22D21968CAF9DAFAEAFBFAF219730
:1000600020E030E040EA50E4C701B6010F942D32A1
:1000700025966CAF7DAF8EAF9FAF2597A496BFAD91
:10008000A497B111D2CF20E030E040EA50E4612FD4
:10009000702F832D922D0F942C32162F072F382E70
:1000A000292E9FCFA496FFADA497F1110DC020E09B
:1000B00030E040E251E4B401C5010F942C32162F18
:1000C000072F382E292ECECDA4962FADA4972430FD
:1000D0009CF020E030E040E251E4B401C5010F940F
:1000E0002C3221966CAF7DAF8EAF9FAF2197182D2C
:1000F000092D3A2C2B2CB6CD182D092D3A2C2B2C52
:1001000082ED482E83E5582E8BEF682E81E4782E01
:10011000B1CD2F923F924F925F926F927F928F92CA
:100120009F92AF92BF92CF92DF92EF92FF920F9386
:100130001F93CF93DF93CDB7DEB7C054D1090FB66D
:10014000F894DEBF0FBECDBF8091A00C888B87E5F1
:100150000E94981E882309F423C120E030E0A90101
:100160006091E9057091EA058091EB059091EC05AD
:100170000F945D2B811108C00E94714E8DE09DE0AF
:100180000E94A13810E01FC18AE50E94E61E882364
:1001900039F10E94EC242091F3083091F408409149
:1001A000F5085091F6080F942C326B017C0120E089
:1001B00030E040E251ECC701B6010F948D3487FD69
:1001C0000AC020E030E040E251E4C701B6010F94DC
:1001D0005D2B181674F40E94714E80E09DE0D0CF24
:1001E000C0907102D0907202E0907302F09074029D
:1001F000DECF40E050E060EC7FE788E50E94162506
:100200002091EB083091EC084091ED085091EE08F8
:100210000F942C322B013C0140E050E060EC7FE772
:1002200089E50E9416252091EF083091F008409151
:10023000F1085091F2080F942C324B015C016FEFE2
:1002400089E40E94A824182F6FEF8AE40E94A82452
:10025000082FA3019201C301B2010F941F35811130
:100260006EC0A5019401C501B4010F941F35811121
:1002700066C08BA19CA1ADA1BEA18BAB9CABADAB6D
:10028000BEAB2091E1053091E2054091E30550912C
:10029000E405C301B2010F942C322B013C0120E094
:1002A00030E040E05FE36BA97CA98DA99EA90F9483
:1002B000C32B9B01AC01C301B2010F942D322BA9BA
:1002C0003CA94DA95EA90F9427330F949933162F9B
:1002D0004FA058A469A47AA42091E5053091E605C1
:1002E0004091E7055091E805C501B4010F942C3207
:1002F0004B015C0120E030E040E05FE3C301B2016C
:100300000F94C32B9B01AC01C501B4010F942D3296
:10031000A30192010F9427330F949933062F812F55
:10032000012E000C990B97FD33C005979CF5802F8B
:10033000002E000C990B97FD2FC005977CF515300A
:1003400008F020CF053008F01DCF80E00E94C7697B
:1003500095E01902F0011124E00FF11D07FDFA9557
:10036000EE0FFF1FEE0FFF1FE555F84FC082D18241
:10037000E282F382602F812F0F94C61A88890E942F
:10038000C7698889882309F4FDCE0E940331FACE1B
:1003900010E0CDCF14E0CBCF00E0D1CF04E0CFCF41
:1003A0008AE40E94981E182F811128C070E060E036
:1003B00086E50E94DD249A838983059710F18BEDF1
:1003C0009CE00E94A138812FC05CDF4F0FB6F894EB
:1003D000DEBF0FBECDBFDF91CF911F910F91FF9078
:1003E000EF90DF90CF90BF90AF909F908F907F90D5
:1003F0006F905F904F903F902F9008950E94A56F4F
:10040000C1CE60E084E40E94C4248F8740E050E0C5
:10041000BA018AE50E9416256BA77CA78DA79EA727
:1004200040E050E86BE376E483E50E94162520E087
:1004300030E040E752E40F94273360934502709315
:1004400046028093470290934802E090EC12F090AD
:10045000ED12D7014D905D906D907C9020E030E0E2
:10046000A901C301B2010F942D32962E872E382E8A
:10047000292E20E030E040E450E40F945D2B87FF0C
:1004800006C0912C812CB0E43B2E00E4202E20E00D
:1004900030E040EB53E4C301B2010F942D326BAB5B
:1004A0007FAB88AF99AF20E030E84EEA53E40F9479
:1004B0008D3418163CF41BAAB0E8BFABEEEAE8AFE7
:1004C000F3E4F9AFD70114964D905D906D907C9058
:1004D000179720E030E0A901C301B2010F942D323B
:1004E0005B016C0120E030E040EE51E40F945D2BA5
:1004F00087FF06C0A12CB12CF0EECF2EA1E4DA2E9E
:1005000020E030E044EB53E4C301B2010F942D32FC
:100510007B01082F9AAF20E030E046EA53E40F94C5
:100520008D3418162CF4E12CF12C06EAB3E4BAAFA2
:1005300088E40E94981E882309F41AC20E94EC24C1
:100540000F9499332B0177FF02C06F5F7F4F759532
:100550006795EE27FF27E61BF70B2196FFAFEEAF5F
:100560002197BF016C547F4F072E000C880B990B0D
:100570000F94642B6BAF7CAF8DAF9EAF9501A6013E
:100580000F948D34181624F0ABAEBCAECDAEDEAEFB
:1005900021966EAD7FAD219760557F4F072E000CE1
:1005A000880B990B0F94642B5B016C01292D382D5E
:1005B000432D522D0F948D34181624F0A92CB82CED
:1005C000C32CD22CC501D6018B8B9C8BAD8BBE8BE3
:1005D0008BAD9CADADADBEAD8F8B988FA98FBA8F13
:1005E000B201550C880B990B0F94642B2B013C0125
:1005F000AC019B016BAD7CAD8DAD9EAD0F942D32EA
:100600001B014C019701402F5AAD0F945D2B87FFC2
:1006100003C07101082D9AAEA3019201B501C60174
:100620000F942D325B016C012BA93FA948AD59AD48
:100630000F945D2B87FF04C0ABAABFAAC8AED9AE8A
:100640008BA99FA9A8ADB9AD8B8F9C8FAD8FBE8FA5
:10065000C701A02FBAAD8F8F98A3A9A3BAA3BE01DB
:10066000695E7F4FCE0143960E94A32E882309F432
:10067000ADC1BE01615E7F4FCE014B960E94A32E9D
:10068000E82E882309F4A2C12F89388D498D5A8D0F
:100690006F8D78A189A19AA10F942C3220E030E0CF
:1006A00040E85EE30F94C32B4B015C012B893C892E
:1006B0004D895E896B8D7C8D8D8D9E8D0F942C3236
:1006C00020E030E040E85EE30F94C32B6BA37CA3F3
:1006D0008DA39EA38FA298A6A9A6BAA689819A8166
:1006E0001816190674F489EA9CE00E94A1388F85D7
:1006F000882321F08FE99CE00E94A1388AE00E94C3
:1007000068380E94DE610E942D1D80E00E94C7694A
:1007100080E090E0A0E2B1E48FA798ABA9ABBAABC0
:1007200060E0CE018F960E9481652091E9053091AD
:10073000EA054091EB055091EC056BA17CA18DA1E0
:100740009EA10F945D2B811130C02091ED05309159
:10075000EE054091EF055091F0056FA178A589A5B0
:100760009AA50F945D2B811120C02091E105309155
:10077000E2054091E3055091E4056B897C898D8900
:100780009E890F945D2B811110C02091E505309159
:10079000E6054091E7055091E8056F89788D898DD0
:1007A0009A8D0F945D2B8823A9F00E94A56F88E095
:1007B000FE01B396A9EEB5E001900D928A95E1F79E
:1007C00088E0FE017396A1EEB5E001900D928A9546
:1007D000E1F7188A60E085E40E94C424882309F4C4
:1007E000F8C0F1E0FBAB1B861C861D861E861A8AAC
:1007F0009E2C4FE6C42E4CE0D42E5DE7A52E5CE087
:10080000B52E1A8915300CF0F4C06B857C858D856A
:100810009E859B01AC010F941F358111EAC0992080
:1008200009F4DAC031E03FAB35E0232E91E09926A0
:10083000F12EFF0CFF0CF10EF394898B19896A8954
:10084000121509F4D2C0062E000C770B880B990BF9
:100850000F94642B2FA138A549A55AA50F94C32B3B
:100860002F89388D498D5A8D0F942D322B013C01E3
:10087000612F110F770B880B990B0F94642B2BA111
:100880003CA14DA15EA10F94C32B2B893C894D89BE
:100890005E890F942D326B837C838D839E834F8280
:1008A000588669867A8689819A81892B79F06F2D9D
:1008B0008BE89CE00E94764169E170E089E89CE069
:1008C0000E94A04186E89CE00E94A1381F9299E115
:1008D0009F931F92FF92DF92CF92BF92AF921F928F
:1008E0000F94F11B29814BA9BE01695F7F4FCE0197
:1008F00003960F94B51C2B013C014B865C866D86DC
:100900007E860FB6F894DEBF0FBECDBFAC019B0153
:100910000F941F35811166C089883A8825E0382DEB
:10092000320380011124030D111D37FC1A95000FAD
:10093000111F000F111F0555184FA30192016BA540
:100940007CA58DA59EA50F942D32D8016D937D9326
:100950008D939C931397632D882D0F94C61A188A34
:1009600081E00E94745AF3948989BFA98B0F65CFE7
:10097000A501B60186E40E9416252B013C01492DF4
:10098000582D632D722D8CE40E9416256B8B7C8B69
:100990008D8B9E8B4F8A588E698E7A8EA701602F21
:1009A0007AAD82E40E9416256B017C014BA95FA9F8
:1009B00068AD79AD82E50E9416256B8F7C8F8D8F97
:1009C0009E8FCF8ED8A2E9A2FAA249CE8FEB9CE0EF
:1009D000F8CC22E02BAB07CF8FEF8FAB22242A94E9
:1009E00084E024CF88890E94C7698A898F5F8A8BB7
:1009F00008CF0E94D7ED0E945766882359F0888956
:100A00000E94C76980E090E0A0ECBFE78B879C87DD
:100A1000AD87BE876B857C858D859E859B01AC01EE
:100A20000F941F35811159C08F85811126C082E036
:100A3000F82E02E094E0C92E12E0DC2CD11A21E05D
:100A400041E0612F802F0E94C52221E04FEF612FEE
:100A50008F2D0E94C5222FEF41E06D2D802F0E9427
:100A6000C5222FEF4FEF6D2D8F2D0E94C522115003
:100A700020F70150F3940F3FF9F60E94E7400E94DF
:100A8000F31E8F85811124C081E792E00E94DD1D55
:100A90004B015C0189E692E00E94831F9B01AC013F
:100AA000C501B4010F94C32B9B01AC01609171028D
:100AB0007091720280917302909174020F942C32A3
:100AC0006093710270937202809373029093740228
:100AD0008F858111E888E092A00C0E94141D8091FE
:100AE000A00C81110E94502B0E9441680E9403318A
:100AF0006B857C858D859E8511E09B01AC010F94F3
:100B00001F35811160CC3ECB8F929F92AF92BF92E6
:100B1000CF92DF92EF92FF920F931F93CF93DF93C9
:100B200000D01F92CDB7DEB75C016B017A01122FA6
:100B30000023E1F10E94754E88E999E00E94A138F6
:100B400061E0812F0E94953A9090280583E0809380
:100B5000280581E080939E0C0E948D4082E0809366
:100B6000F91140E368E879E084E799E00E94924057
:100B700040E069E171E18DE699E00E94924061E018
:100B800088E699E00E9474408AE799E00E948122F9
:100B900080919E0C882341F060E0812F0E94953A5D
:100BA00081E00E94745AF4CF9092280520E030E052
:100BB000A901F50160817181828193810F945D2B80
:100BC000882371F080E090E0A0ECB0E489839A8300
:100BD000AB83BC83BE016F5F7F4FC5010E94076975
:100BE00020E030E0A901F60160817181828193816A
:100BF0000F945D2B882351F18090D90C9090DA0CE2
:100C0000A090DB0CB090DC0C80E090E0A0E7B1E4B9
:100C10008093D90C9093DA0CA093DB0CB093DC0C8E
:100C200080E090E0A0EAB1E489839A83AB83BC833F
:100C3000BE016F5F7F4FC6010E9407698092D90C89
:100C40009092DA0CA092DB0CB092DC0C20E030E049
:100C5000A901F70160817181828193810F948D34A4
:100C6000181674F480E090E0A0E4B0E489839A83DD
:100C7000AB83BC83BE016F5F7F4FC7010E940769D2
:100C80008091FD0429E131E1882311F029E439E064
:100C900047E559E061E679E081E00E94B5400E94B5
:100CA0008D4081E00F900F900F900F90DF91CF91CA
:100CB0001F910F91FF90EF90DF90CF90BF90AF907A
:100CC0009F908F900895CF93C82F80915D0C83FDE6
:100CD00014C080912209811110C080916702909107
:100CE00068029C01215031094091551250915612D1
:100CF0004217530714F40E946E1FCC2329F061E0C1
:100D000080E0CF910C94DEBF8091220991E0892789
:100D10008093440280914402882389F08091531289
:100D2000909154122091551230915612821B930BC0
:100D300097FF03C0919581959109029744F4109211
:100D4000440280915D0C83FF06C0C1E01AC080E0C0
:100D50000E94745ADFCFC0912209C11112C0809144
:100D600067029091680201972091551230915612B6
:100D70002817390754F70E94754E8BE299E00E94BC
:100D8000A1388C2FCF910895AF92BF92CF92DF926E
:100D9000EF92FF920F931F93CF93DF93CDB7DEB700
:100DA00064970FB6F894DEBF0FBECDBF0E94744F9C
:100DB00087FDAFC08AE50E94E61E882309F4BAC009
:100DC00040E050E0BA018AE50E9416257B018C01C3
:100DD000209171023091720240917302509174021D
:100DE00060E070E088EC93E40F942C325B016C01BE
:100DF0009701A8010F948D34181614F0750186011F
:100E000020E030E0A901B701C8010F948D34181615
:100E100024F4E12CF12C00E010E0B701C8010F949C
:100E20009933072E000C880B990B0F94642B698B58
:100E30007A8B8B8B9C8B20E030E0A9010F945D2B8B
:100E4000882321F0CE0141960E94857380E090E0D6
:100E5000A0EAB1E48D879E87AF87B88B19861A8682
:100E60001B861C868CE40E94981E882309F467C0A8
:100E70000E94EC246B017C0120E030E0A901C70155
:100E8000B6010F948D3487FF04C0F7FAF094F7F899
:100E9000F094CD82DE82EF82F88620915512309157
:100EA00056122430310574F08091531290915412EF
:100EB000821B930B97FF03C091958195910901E0E7
:100EC00004970CF400E080E00E946386882359F0C8
:100ED00022E0AE01435F5F4FBE016B5F7F4FCE01EB
:100EE00009960E94848569897A898B899C898B01FE
:100EF0009C01305809831A832B833C8320E030E027
:100F0000A9010F945D2B882321F0CE0101960E9448
:100F1000857364960FB6F894DEBF0FBECDBFDF9128
:100F2000CF911F910F91FF90EF90DF90CF90BF90E6
:100F3000AF900895E12CF12C00E211E449CFC0906C
:100F4000DC05D090DD05E090DE05F090DF0594CF64
:100F50007F928F929F92AF92BF92CF92DF92EF9249
:100F6000FF920F931F93CF93DF9300D000D01F9277
:100F70001F92CDB7DEB76C015B014A01722E78017A
:100F8000009129060E947A1F809155129091561265
:100F90008E159F051CF4C7010E946E1F80E00E9401
:100FA0006386882331F0272DA401B501C6010E9474
:100FB00084851E141F043CF4C7010E946E1F60E06C
:100FC00080E00E94DEBF81E00E94638680E090E0C6
:100FD000A0E7B2E489839A83AB83BC8380E090E08E
:100FE000A0E8B0EC8D839E83AF83B887BE016F5FAE
:100FF0007F4FCE0105960E94076987E00E94672A0D
:10100000811158C08091710290917202A091730277
:10101000B09174024091020550910305609104055E
:1010200070910505C090FE04D090FF04E09000058B
:10103000F0900105C0928F07D0929007E09291073F
:10104000F09292074093930750939407609395070B
:10105000709396078093970790939807A0939907AA
:10106000B0939A0780E090E0A8E4B2E489839A8381
:10107000AB83BC83CE0101960E941E73809106054E
:1010800090910705A0910805B091090580939707F5
:1010900090939807A0939907B0939A0780E090E007
:1010A000A0EAB0E489839A83AB83BC83CE01019626
:1010B0000E941E73C12CD12C80E7E82E82E4F82E0A
:1010C000C982DA82EB82FC8280E090E0A0E8B0E4A2
:1010D0008D839E83AF83B887BE016F5F7F4FCE0144
:1010E00005960E94076920E030E0A90160910A0599
:1010F00070910B0580910C0590910D050F945D2B5F
:1011000087FF0BC0C982DA82EB82FC82BE016F5F6F
:101110007F4F8AE095E00E94076980910A059091CF
:101120000B05A0910C05B0910D058093750290936D
:101130007602A0937702B093780280939B079093F6
:101140009C07A0939D07B0939E078BE997E00E94B0
:10115000EF618091E00581110F940C1A61E087EB3B
:1011600099E00E94DD3F80918B11815080938B111B
:101170004AE958E16FEB79E085E00E94E5EB809168
:101180008B11882339F00E9417AE80918B1181500A
:1011900080938B1180E00F94D31B0E94FD318091CE
:1011A0008C11823011F40E94AF380E94D7ED28963E
:1011B0000FB6F894DEBF0FBECDBFDF91CF911F9168
:1011C0000F91FF90EF90DF90CF90BF90AF909F90E6
:1011D0008F907F900895CF92DF92EF92FF920F93BE
:1011E0001F93CF93DF9300D01F92CDB7DEB77C0162
:1011F0006B018A0161E08CE399E00E94DD3F4AE9DE
:1012000058E163E479E085E00E94E5EB90918B1171
:1012100081E0890F80938B118091A91482FF06C011
:101220008B7F8093A9149E5F90938B110E94A139AC
:1012300080E1E9E6F2E0AEEFB4E001900D928A952C
:10124000E1F70E94DE6181E00F94D31B20E030E0E3
:10125000A901F70160817181828193810F945D2BD7
:101260008823F1F08091220981110CC080916702DE
:1012700090916802019720915312309154122817CF
:10128000390774F080E090E0A0E7B2E489839A83A4
:10129000AB83BC83BE016F5F7F4FC7010E940769AC
:1012A00087E00E94672A811103C0B6010E945B6833
:1012B00020E030E0A901F801608171818281938191
:1012C0000F945D2B882341F080E00E946386882381
:1012D00019F0C8010E943769129A64E670E080E054
:1012E00090E00E945A2681E00F900F900F900F908F
:1012F000DF91CF911F910F91FF90EF90DF90CF90F2
:101300000895CF92DF92EF92FF92CF93DF936B011C
:101310007C01D42FC091280583E08093280581E0CB
:1013200080939E0CC114D104E104F10431F00E94B9
:1013300002AAC60ED71EE81EF91E80919E0C8823B5
:1013400089F0C114D104E104F10421F48D2F0E942D
:10135000745AF3CF0E9402AA6C197D098E099F0965
:1013600097FDF4CF10929E0CC0932805DF91CF918A
:10137000FF90EF90DF90CF9008950F931F93CF933E
:10138000DF93C82F162F0E94754EC11194C0CFE86D
:10139000D8E0CE010E94A13861E0812F0E94953AE9
:1013A0000E9402AA685370458F4F9F4F6093250695
:1013B000709326068093270690932806109229069C
:1013C0000091280583E08093280530E020E049E182
:1013D00051E16DE179E082E00E94B5408DE199E054
:1013E0000E94812281E080939E0C80919E0C882334
:1013F00009F464C060E0812F0E94953A809129062B
:10140000882309F454C00E94754E83E099E00E943D
:10141000A13830E020E04DEE58E064EF78E082E063
:101420000E94B54084EF98E00E94812241E060E094
:1014300070E0CB010E94818930E020E050E040E084
:1014400060EE78E085E00E94B54080EE98E00E9472
:1014500004360E947A1F80E00E9463860E94754EC7
:10146000CE010E94A1380E9402AA685370458F4F96
:101470009F4F6093250670932606809327069093CE
:1014800028061092290630E020E049E151E164EDA0
:1014900078E082E00E94B54083EC98E00E948122CF
:1014A00081E080939E0C61E0812F0E94953A81E05B
:1014B0000E94745A9ACFC4EAD8E06BCF00932805F3
:1014C000DF91CF911F910F910895CF92DF92EF920C
:1014D000FF920F931F93CF93DF93CDB7DEB7A09703
:1014E0000FB6F894DEBF0FBECDBF0E94744F87FDCC
:1014F000CCC085E40E94981E882309F4D5C00E94C0
:10150000EC246B017C0120E030E0A9010F948D34C4
:1015100087FF04C0F7FAF094F7F8F094F7FAF09424
:10152000F7F8F094CD8EDE8EEF8EF8A28CE0ECED25
:10153000F2E0DE01119601900D928A95E1F78AE5BD
:101540000E94E61E882351F040E050E0BA018AE58F
:101550000E94162569877A878B879C8788E50E9479
:10156000E61E882351F040E050E0BA0188E50E9471
:10157000162569837A838B839C8389E50E94E61E06
:10158000882351F040E050E0BA0189E50E94162519
:101590006D837E838F83988785E50E94981E8823BC
:1015A00009F489C00E94EC246B017C0120E030E04A
:1015B000A901C701B6010F948D3487FF04C0F7FA63
:1015C000F094F7F8F094F7FAF094F7F8F094C98EE5
:1015D000DA8EEB8EFC8E1D8A1E8A1F8A188E8CE492
:1015E0000E94981E882309F46FC00E94EC246B01AE
:1015F0007C0120E030E0A901C701B6010F948D34D1
:1016000087FF04C0F7FAF094F7F8F094C98ADA8AF1
:10161000EB8AFC8A62E070E082E40E94DD24F82E0E
:1016200080918B11811131C021E0AE01475E5F4F87
:10163000BE016F5F7F4FCE014D960E94EB888823DD
:1016400021F16F2D81E00E94BD8982E50E94E61E96
:10165000882309F442C00E94D92440E050E060EAA7
:1016600071E44D875E876F87788B20918B112223E1
:1016700061F08C012F2DAE01435F5F4FBE016F5EA5
:101680007F4FCE0145960E94A887A0960FB6F8948A
:10169000DEBF0FBECDBFDF91CF911F910F91FF90A5
:1016A000EF90DF90CF900895C12CD12C80E8E82EE8
:1016B00080E4F82E33CFC090D805D090D905E090C3
:1016C000DA05F090DB0572CFC090DC05D090DD0527
:1016D000E090DE05F090DF058CCF90E080E0BDCF9C
:1016E000CF92DF92EF92FF920F931F93CF93DF93EE
:1016F000CDB7DEB76C970FB6F894DEBF0FBECDBF87
:101700008CE40E94981E882309F4B0C00E94EC2447
:101710006B017C0120E030E0A9010F948D3487FF3C
:1017200004C0F7FAF094F7F8F094F7FAF094F7F8A9
:10173000F094C98EDA8EEB8EFC8E8CE0ECEDF2E04C
:10174000DE01119601900D928A95E1F788E50E94DD
:10175000E61E8823A1F040E050E0BA0188E50E942F
:1017600016252091EB083091EC084091ED0850913E
:10177000EE080F942C3269837A838B839C8389E5EE
:101780000E94E61E8823A1F040E050E0BA0189E5FE
:101790000E9416252091EB083091EC084091ED084D
:1017A0005091EE080F942C326D837E838F8398873F
:1017B0008AE50E94E61E882351F040E050E0BA011D
:1017C0008AE50E94162569877A878B879C871D8604
:1017D0001E861F86188A80918B11811138C020E0E7
:1017E000AE01435F5F4FBE016F5F7F4FCE014996F1
:1017F0000E94EB88882359F18091E00581110F94B4
:101800000C1A60E080E00E94BD89898D9A8DAB8DB5
:10181000BC8DB0588D8B9E8BAF8BB88F198A1A8A6E
:101820001B8A1C8A1D861E861F86188A80918B1132
:10183000882369F010E000E020E0AE014B5E5F4FCE
:10184000BE016F5E7F4FCE010D960E94A8876C96F9
:101850000FB6F894DEBF0FBECDBFDF91CF911F91C1
:101860000F91FF90EF90DF90CF900895C12CD12C75
:1018700080E8E82E80E4F82E58CF2F923F924F92C6
:101880005F926F927F928F929F92AF92BF92CF9210
:10189000DF92EF92FF920F931F93CF93DF93CDB719
:1018A000DEB7E5970FB6F894DEBF0FBECDBF8DABA8
:1018B000209128052CAB81E0809328058091460576
:1018C0008D3409F4C6C4843511F40C949CA087347B
:1018D00009F091C180914405909145058B319105A6
:1018E00009F4DDC108F079C18430910508F030C1F8
:1018F0002091FC068230910508F48EC1213009F058
:1019000091C111E0029709F010E00E942D25198283
:101910001A821B821C821D821E821F82188682E50B
:101920000E94E61E882309F490C10E94EC246B01FA
:101930007C0120E030E0A9010F945D2B882309F49D
:10194000EAC04090690250906A0260906B02709009
:101950006C0280916D0290916E02A0916F02B09125
:1019600070028CA79DA7AEA7BFA780908F0790900D
:101970009007A0909107B090920780919307909163
:101980009407A0919507B091960788AB99ABAAAB45
:10199000BBABA5019401C301B2010F945D2B811172
:1019A0000DC028A939A94AA95BA96CA57DA58EA55A
:1019B0009FA50F945D2B882309F4ADC0A30192016C
:1019C000C501B4010F942C3220E030E040E05FE329
:1019D0000F94C32B68A779A78AA79BA72CA53DA521
:1019E0004EA55FA568A979A98AA99BA90F942C3255
:1019F00020E030E040E05FE30F94C32B2B013C017B
:101A000020E030E0A901C701B6010F945D2B881FCB
:101A10008827881F181709F40FC180E090E0A0E81C
:101A2000BFEB8CA79DA7AEA7BFA728A539A54AA540
:101A30005BA5CA01B9010F94C32B4B015C01A30143
:101A40009201C301B2010F94C32B9B01AC01C501EC
:101A5000B4010F942D320F94DB344B015C01AC01C7
:101A60009B01C701B6010F942C3268AB79AB8AABEE
:101A70009BABA5019401C701B6010F942D329B01C8
:101A8000AC0168A979A98AA99BA90F94C32B6B0102
:101A90007C0120E030E0A9010F948D3487FDD1C096
:101AA000C701B6010F94DB346B017C01C301B201A5
:101AB0009058A50194010F9427332CA53DA54EA560
:101AC0005FA50F94C32BA70196010F94C32B28A5E4
:101AD00039A54AA55BA50F942D3269837A838B8340
:101AE0009C83A501940168A579A58AA59BA50F945F
:101AF00027332CA53DA54EA55FA50F94C32BA701A9
:101B000096010F94C32BA30192010F942D326D8384
:101B10007E838F83988720E030E0A90169817A81F4
:101B20008B819C810F945D2B8111A3C020E030E05C
:101B3000A9016D817E818F8198850F945D2B811124
:101B400098C00E94714E8BEB9FE00E94A1386AC042
:101B50008531910509F466C08A31910509F49CC06C
:101B6000049709F048C080E50E94E61EC12CD12CE4
:101B70007601882321F00E9466246B017C0183E5B5
:101B80000E94E61E882361F00E94EC2420E030E0F1
:101B90004AE754E40F94C32B0F94A0336B017C01EC
:101BA0000E94DE6180918D11811105C060E081EDA0
:101BB0009FE00E9410400E9402AAC60ED71EE81E97
:101BC000F91E0E9402AA6C197D098E099F0997FFD0
:101BD00029C080E00E94745AF4CF8A32910509F43A
:101BE000ADC160F48D31910509F4D6C008F470C020
:101BF0004E9709F429C10F94781C14C08B359105B8
:101C000009F47FC28C35910509F47FC28A359105AC
